:020000022000DC
:106000000000042091860200ED660700E76C07009F
:10601000ED660700ED660700ED6607000000000072
:10602000000000000000000000000000ED66070016
:10603000ED66070000000000ED660700ED66070052
:1060400085850200ED660700E5890200C18802002F
:10605000D1880200ED660700ED810200ED660700C1
:10606000ED660700C5890200D5890200618602003D
:10607000ED660700ED660700ED660700ED660700B8
:10608000358E020071860200ED660700ED6607009E
:10609000ED660700ED66070031890200ED66070036
:1060A000ED660700ED660700ED660700ED66070088
:1060B000ED660700ED66070000000000000000002C
:1060C000ED660700ED660700ED660700E188020057
:1060D00081860200ED660700ED660700058A020072
:1060E000F5890200ED660700ED66070009890200E8
:0860F00000000000ED6607004E
:1070000040F8044B40F8045B40F8046B40F8047B04
:1070100040F8048B40F8049B40F804AB40F804BBF4
:1070200040F804CB40F804DB6846704781F000412B
:1070300002E000BF83F0004330B54FEA41044FEA5D
:10704000430594EA050F08BF90EA020F1FBF54EAF8
:10705000000C55EA020C7FEA645C7FEA655C00F094
:10706000E2804FEA5454D4EB5555B8BF6D420CDD65
:107070002C4480EA020281EA030382EA000083EAE8
:10708000010180EA020281EA0303362D88BF30BD88
:1070900011F0004F4FEA01314FF4801C4CEA1131DE
:1070A00002D0404261EB410113F0004F4FEA03333D
:1070B0004CEA133302D0524263EB430394EA050FC8
:1070C00000F0A780A4F10104D5F1200E0DDB02FA37
:1070D0000EFC22FA05F2801841F1000103FA0EF2CB
:1070E000801843FA05F359410EE0A5F120050EF191
:1070F000200E012A03FA0EFC28BF4CF0020C43FAC2
:1071000005F3C01851EBE37101F0004507D54FF0CE
:10711000000EDCF1000C7EEB00006EEB0101B1F51E
:10712000801F1BD3B1F5001F0CD349085FEA300064
:107130004FEA3C0C04F101044FEA445212F5800F6F
:1071400080F09A80BCF1004F08BF5FEA500C50F10C
:10715000000041EB045141EA050130BD5FEA4C0CEF
:10716000404141EB0101013C28BFB1F5801FE9D24C
:1071700091F0000F04BF01460020B1FA81F308BF6F
:107180002033A3F10B03B3F120020CDA0C3208DD3B
:1071900002F1140CC2F10C0201FA0CF021FA02F116
:1071A0000CE002F11402D8BFC2F1200C01FA02F186
:1071B00020FA0CFCDCBF41EA0C019040E41AA2BFAB
:1071C00001EB0451294330BD6FEA04041F3C1CDA73
:1071D0000C340EDC04F11404C4F1200220FA04F093
:1071E00001FA02F340EA030021FA04F345EA03013D
:1071F00030BDC4F10C04C4F1200220FA02F001FAFF
:1072000004F340EA0300294630BD21FA04F0294680
:1072100030BD94F0000F83F4801306BF81F4801119
:107220000134013D4EE77FEA645C18BF7FEA655C8C
:1072300029D094EA050F08BF90EA020F05D054EA5E
:10724000000C04BF1946104630BD91EA030F1EBF63
:107250000021002030BD5FEA545C05D14000494167
:1072600028BF41F0004130BD14F580043CBF01F55A
:10727000801130BD01F0004545F0FE4141F4700140
:107280004FF0000030BD7FEA645C1ABF194610461B
:107290007FEA655C1CBF0B46024650EA013406BF1C
:1072A00052EA033591EA030F41F4002130BD00BFDB
:1072B00090F0000F04BF0021704730B54FF4806498
:1072C00004F132044FF000054FF0000150E700BF19
:1072D00090F0000F04BF0021704730B54FF4806478
:1072E00004F1320410F0004548BF40424FF0000165
:1072F0003EE700BF42004FEAE2014FEA31014FEAA8
:1073000002701FBF12F07F4393F07F4F81F06051F6
:10731000704732F07F4208BF704793F07F4F04BF41
:1073200041F40021704730B54FF4607401F000451E
:1073300021F000411CE700BF50EA010208BF70477E
:1073400030B54FF000050AE050EA010208BF70476F
:1073500030B511F0004502D5404261EB41014FF4D8
:10736000806404F132045FEA915C3FF4D8AE4FF0E0
:1073700003025FEADC0C18BF03325FEADC0C18BFC3
:10738000033202EBDC02C2F1200300FA03FC20FA14
:1073900002F001FA03FE40EA0E0021FA02F1144461
:1073A000BDE600BF4FEA4102B2F1E04324BFB3F5AE
:1073B000001CDCF1FE5C0DD901F0004C4FEAC0026C
:1073C0004CEA5070B2F1004F40EB830008BF20F050
:1073D0000100704711F0804F21D113F13872BCBF0A
:1073E00001F00040704741F480114FEA5252C2F15F
:1073F0001802C2F1200C10FA0CF320FA02F018BFA8
:1074000040F001004FEAC1234FEAD32303FA0CFCFA
:1074100040EA0C0023FA02F34FEA4303CCE77FEA89
:10742000625307D150EA01331EBF4FF0FE4040F4D3
:107430004000704701F0004040F0FE4040F4000082
:10744000704700BF80F0004002E000BF81F00041C3
:1074500042001FBF5FEA410392EA030F7FEA226CFA
:107460007FEA236C6AD04FEA1262D2EB1363C1BF8A
:10747000D218414048404140B8BF5B42192B88BFF9
:10748000704710F0004F40F4000020F07F4018BF1C
:10749000404211F0004F41F4000121F07F4118BF3C
:1074A000494292EA030F3FD0A2F1010241FA03FCE4
:1074B00010EB0C00C3F1200301FA03F100F00043CC
:1074C00002D5494260EB4000B0F5000F13D3B0F194
:1074D000807F06D340084FEA310102F10102FE2A03
:1074E00051D2B1F1004F40EBC25008BF20F0010073
:1074F00040EA03007047490040EB0000013A28BF12
:10750000B0F5000FEDD2B0FA80FCACF1080CB2EB94
:107510000C0200FA0CF0AABF00EBC2505242184312
:10752000BCBFD0401843704792F0000F81F40001B7
:1075300006BF80F400000132013BB5E74FEA41038A
:107540007FEA226C18BF7FEA236C21D092EA030FF6
:1075500004D092F0000F08BF0846704790EA010F70
:107560001CBF0020704712F07F4F04D1400028BF9D
:1075700040F00040704712F100723CBF00F500007F
:10758000704700F0004343F0FE4040F400007047B5
:107590007FEA226216BF08467FEA23630146420261
:1075A00006BF5FEA412390EA010F40F48000704774
:1075B0004FF0000304E000BF10F0004348BF40421A
:1075C0005FEA000C08BF704743F0964301464FF056
:1075D00000001CE050EA010208BF70474FF00003B2
:1075E0000AE000BF50EA010208BF704711F00043F3
:1075F00002D5404261EB41015FEA010C02BF8446C3
:107600000146002043F0B64308BFA3F18053A3F521
:107610000003BCFA8CF2083AA3EBC25310DB01FA68
:1076200002FC634400FA02FCC2F12002BCF1004FEC
:1076300020FA02F243EB020008BF20F0010070477D
:1076400002F1200201FA02FCC2F1200250EA4C00D1
:1076500021FA02F243EB020008BF20EADC70704717
:107660007BB972B90029BEBF00204FF0004106E08F
:1076700008BF00281CBF6FF000414FF0FF3000F042
:1076800081B9ADF1080C6DE904CE002909DB002BAE
:107690001ADB02F04FFDDDF804E0DDE9022304B05F
:1076A0007047404261EB4101002B1BDB02F042FDC1
:1076B000DDF804E0DDE9022304B0404261EB410162
:1076C000524263EB43037047524263EB430302F0C1
:1076D00031FDDDF804E0DDE9022304B0404261EB56
:1076E00041017047524263EB430302F023FDDDF892
:1076F00004E0DDE9022304B0524263EB4303704728
:1077000053B94AB9002908BF00281CBF4FF0FF3108
:107710004FF0FF3000F036B9ADF1080C6DE904CE42
:1077200002F008FDDDF804E0DDE9022304B0704753
:1077300070B54FF0FF0C4CF4E06C1CEA11541DBF07
:107740001CEA135594EA0C0F95EA0C0F00F0DEF8D2
:107750002C4481EA030621EA4C5123EA4C5350EAB7
:10776000013518BF52EA033541F4801143F4801308
:1077700038D0A0FB02CE4FF00005E1FB02E506F099
:107780000042E0FB03E54FF00006E1FB03569CF0EE
:10779000000F18BF4EF0010EA4F1FF04B6F5007FF4
:1077A00064F5407404D25FEA4E0E6D4146EB060666
:1077B00042EAC62141EA55514FEAC52040EA5E50EF
:1077C0004FEACE2EB4F1FD0C88BFBCF5E06F1ED899
:1077D000BEF1004F08BF5FEA500E50F1000041EBD0
:1077E000045170BD06F0004646EA010140EA02007D
:1077F00081EA0301B4EB5C04C2BFD4EB0C0541EA9F
:10780000045170BD41F480114FF0000E013C00F3B3
:10781000AB8014F1360FDEBF002001F0004170BDD7
:10782000C4F10004203C35DA0C341BDC04F11404F0
:10783000C4F1200500FA05F320FA04F001FA05F27C
:1078400040EA020001F0004221F0004110EBD37049
:1078500021FA04F642EB06015EEA430E08BF20EA75
:10786000D37070BDC4F10C04C4F1200500FA04F318
:1078700020FA05F001FA04F240EA020001F00041AA
:1078800010EBD37041F100015EEA430E08BF20EA1D
:10789000D37070BDC4F1200500FA05F24EEA020E65
:1078A00020FA04F301FA05F243EA020321FA04F094
:1078B00001F0004121FA04F220EA020000EBD3704B
:1078C0005EEA430E08BF20EAD37070BD94F0000F4B
:1078D0000FD101F00046400041EB010111F4801F7F
:1078E00008BF013CF7D041EA060195F0000F18BF30
:1078F000704703F00046520043EB030313F4801F6C
:1079000008BF013DF7D043EA0603704794EA0C0F25
:107910000CEA135518BF95EA0C0F0CD050EA41063B
:1079200018BF52EA4306D1D181EA030101F00041B8
:107930004FF0000070BD50EA410606BF10461946E0
:1079400052EA430619D094EA0C0F02D150EA0136EC
:1079500013D195EA0C0F05D152EA03361CBF10462D
:1079600019460AD181EA030101F0004141F0FE41CC
:1079700041F470014FF0000070BD41F0FE4141F450
:10798000780170BD704700BF4A0011D212F5001295
:1079900011D20DD56FF47873B3EB62520ED44FEA67
:1079A000C12343F0004343EA505323FA02F07047E7
:1079B0004FF00000704750EA013002D14FF0FF3025
:1079C00070474FF00000704730B5144685B017A3DC
:1079D000D3E90023FFF744FE054601A9284647F0F6
:1079E000F1FB9DF807309DF806200F491B0443EA80
:1079F00042539DF8082043EAC2239DF8092043EA38
:107A000042139DF80A2043EA5203BDF8042025F0F2
:107A10000105A2F2BC7243EA4263A5FB01012360A7
:107A200005B030BDAFF3008000CA9A3B00CA9A3B54
:107A300000000000182A2DE9F74F054621D0202A22
:107A400022D00A200423C5F8002185F8040185F816
:107A50000531284600F0AAFC0022034695F80541AE
:107A6000A24214D3DFF8DCC0DFF8DCE000EB8403D3
:107A700095F804210132B4EB820F1AD303B0BDE8AC
:107A8000F08F0C200623DEE70E200823DBE711F839
:107A9000044B03F8044B11F8034C03F8034C11F8A2
:107AA000024C03F8024C11F8014C03F8014C01326E
:107AB000D4E795F80521B4FBF2FA02FB1A4913F852
:107AC000041C13F8038C13F8027C13F8016C019268
:107AD000B9F1000F0BD11CF808B01CF807801CF896
:107AE00006701CF801601EF80A108BEA0101D5F837
:107AF0000021202A0CD1B9F1040F09D1DFF84490FC
:107B000019F8011019F8088019F8077019F80660BB
:107B1000019AA21A043310F8229000EB820281EA43
:107B2000090103F8041C517888EA010803F8038C62
:107B300091784F4003F8027CD278564003F8016CEC
:107B4000013495E77F3B0A00743B0A002DE9F04FB2
:107B5000044685B0084600F029FC89460246804666
:107B6000214600204EF09FFD231D019304F11003D8
:107B70000125029322462146002311F82300324EAC
:107B8000305C01F823000133042BF6D1019B013155
:107B90008B42F1D1617963786170617A6171617B47
:107BA0006172A17A6373A378A170A17BA372A37998
:107BB000A171E17BA373E378E170E17AE173E1798C
:107BC000E172E37199F80431AB4234D092F800B01D
:107BD0005678917892F803A08BEA060081EA0A03AE
:107BE00080EA0307039366F0DEF98BEA0000784031
:107BF000107086EA010066F0D6F946407E40567065
:107C0000039866F0D0F94140794091708BEA0A0000
:107C100066F0C9F98AEA000A029B87EA0A07D77068
:107C200004329342D2D128464246214601354EF0D5
:107C30003AFDEDB29EE742462146284605B0BDE832
:107C4000F04F4EF030BD00BF7F3B0A002DE9F04FF2
:107C5000504C904603F003029B101F2B04EB821440
:107C600089469E464C49A8BF4FF01F0E1C2B1D464F
:107C7000A8BF1C2551F822206168033587B025EA8A
:107C8000E575294101920391E268A1688446294182
:107C900000202A410290049105925CF8045B3F4A5F
:107CA000154225F0004111D106AA02EB810151F8DD
:107CB000102C002D40EA0200B8BF5242B8F1010872
:107CC00049F8042BE9D107B0BDE8F08F344A1542DA
:107CD00009D154F82120002BBABFCEF100018A400F
:107CE00042FA0EF2E5E72F4A154214D110392E4A16
:107CF000019E52F8212082FB0616AEF10302002AF3
:107D000044DA51426FF0004242FA01F7B742D0DB49
:107D100006FA01F2CDE74A04B2F1006FB6BF4A0598
:107D200000210421B2F1005FB8BF92001F4EB8BF1E
:107D30000231B2F1804FBCBF52000131B242C7BF25
:107D40001B4F1C4E1C4F1D4E924687FB0ABA77688C
:107D50005744924687FB0ABAB7685744924687FB56
:107D60000ABAF768BA448AFB027236691644144AA2
:107D700052F8212086FB0272019ED20082FB067619
:107D8000104A52F82120AEEB0202B8E746FA02F29E
:107D90008FE700BFE8740A00D8740A00FCFFFF7F79
:107DA000F0FFFF7FC0FFFF7F18740A009979825AA5
:107DB00063218510B0730A00A9BDA029C4730A000D
:107DC000F8730A00D8730A002DE9F74F00F5A048B0
:107DD0004FF0000A476D88F8B4AD88F8AEADB1F148
:107DE000000B816DC0F820A04FF0FF3304464362C2
:107DF0000CBFFF220C22CB1BD019013B04F5DA7615
:107E00008842C8BF1A46236C0092314604F15400E0
:107E10009847009A8242054613D1002F68D1A549A0
:107E20000522304659F067FA78B1A3490522304659
:107E300059F061FA48B10823E361002003B0BDE8BE
:107E4000F08F0623F8E70123F6E7B4F8BA31236090
:107E5000A360B4F8BC316360E36094F8BE31C3F34F
:107E600002120132A261BBF1000F40F0BB8194F815
:107E7000BF2188F8B02D180688F8AFBD4BD503F0A8
:107E8000070B0BF1010B4FF0030A05F5DA710AFA43
:107E90000BFA236C5246214404F1540098470544E0
:107EA00098F8B50D01282DD804F58D520221123213
:107EB00001FA0BF1A44611449CF8C1319CF8C2E1CF
:107EC000DB084FEA9E0EDB0243EA4E139CF8C3E147
:107ED00043EADE0300B15BBA22F8023F91420CF1A3
:107EE000030CE9D14FF0030A0AFA0BFA0AF10D0A62
:107EF00016F80A302C2B00F0E3803B2B0ED1072321
:107F0000E3616FE104F58D50524604F2C111143063
:107F100059F005FAEAE74FF00D0AE9E7212B40F0A6
:107F20009B8006EB0A020AF102015378FE2B68D00F
:107F3000FF2B21D0012B5ED0F92B84D1735C042B55
:107F400013D1D17888F8AF1D5079137903EB002352
:107F50000A204343012BD8BF64232362C90744BFCF
:107F6000937988F8B13D0AF108018A46C0E70AEB27
:107F70000301BAF1000FF8D016F801A04B1CA5EBD5
:107F8000030B0AF11F025A4515DB01F2B5115A46DF
:107F900021443046009359F0EDF9009B0BF5DA715E
:107FA0001F440AF12002236C214404F15400984735
:107FB00000230BEB0005BAF10B0FD8D106EB030B36
:107FC0003E4900935246584659F095F9009B03F1FB
:107FD0000B010028D0D19BF80B30032BCCD19BF8A0
:107FE0000C30012BC8D19BF80E209BF80D3003EB11
:107FF00002236362C0E7735C4A1C9918002BFAD114
:10800000B3E716F801A04B1CA5EB030B0AF11F0206
:108010005A4515DB01F2B5115A462144304600930A
:1080200059F0A8F9009B0BF5DA711F440AF1200200
:10803000236C214404F15400984700230BEB000506
:10804000A26B1AB9DA19A263A4F83CA00AEB0301E7
:10805000BAF1000FD5D188E7A36DDB1B202BB4BF8D
:1080600007230123E8E604F5A55006EB0B011430C5
:10807000009259F054F9009A93447EE0009259F02E
:108080004EF9009A616B236C114461635144ABEB70
:108090000202214404F1540000929847636B009A55
:1080A00029461A4494E0636C394404F1540098471B
:1080B00098E000BF672409006D24090066220900CA
:1080C00006EB0A030AF10A0B99785A7802EB0122AF
:1080D00022611979DA7802EB0122626199795A7981
:1080E00002EB01222260197ADA7902EB0122626046
:1080F0005B7A88F8B33D1A0644D503F007030133D1
:1081000005F5DA7103229A4001932144236C009211
:1081100004F15400984798F8B51D009A01290544C8
:10812000A1D8019B04F5A5524FF0020C12324FF07A
:10813000010B0CFA03FC04EB0A000BFA03FB94445A
:1081400090F8BE3190F8BFE1DB084FEA9E0EDB02EB
:1081500043EA4E1390F8C0E143EADE0301B15BBA93
:1081600022F8023F944500F10300E9D10BF1FF3BF7
:108170000BEB4B0B0AF10D0AD34404F5A04301228B
:1081800083F8B42D16F80B30174A04F5A0480BF10C
:10819000010188F8B23DD35CA3610023636341F21F
:1081A000B47A8D421EDD16F801B0606B4B1CEA1AE2
:1081B00050449345204406EB03013FF75FAF5A4616
:1081C000009359F0ACF8626B009B5A440BEB03012F
:1081D0006263BBF1000FE4D101238D4288F8AE3D0C
:1081E0003FF761AF012029E6F8700A002DE9F04F52
:1081F00000248BB0CDE90444664B674867490122EF
:1082000025461E6846B1D0F80463164204D01D60AE
:108210001E680296029E144304338B424FEA4202C8
:10822000EFD15D4BD3F87C218AB10022C3F87C21C9
:10823000D3F87C310393039B4FF0A04344F00044F8
:10824000D3F810350493564BD3F810350593E3B2A9
:10825000D3B1544F01260025344210D0AB0003F1B6
:10826000804303F5C043D3F81005D3F8101557F831
:10827000253023B1C1F30141C0F3052098470135F2
:10828000082D4FEA4606E7D1002C7FDA0DF1200BCE
:1082900000230893CBF80430DFF804914FF0FF334C
:1082A000069307930025404B0193A846019A12F9C3
:1082B000013F01925A1C50D0C3F3C20000F12802C2
:1082C0000DEB020C03F007011CF8102CCA40D70775
:1082D000DCB203F03F0640D5324A17463244A409C7
:1082E00092F9282057F822A0BAF1000F0AD1032CE6
:1082F00033D11BF800E001228A4042EA0E020BF85B
:10830000002001E0032CF4D01F2E8BBF03F01F03CD
:1083100033464A464FF0A04203F5E07352F823304B
:108320001CF8182CCA40D207C3F3014305D5022B11
:1083300013D1032C0BD1214604E0032B0DD1032CC8
:1083400005D10221304637F021FD0135EDB2BAF1F9
:10835000000F02D021463046D04708F10103022B1E
:108360004FF00108A2D18DB14FF0A0430499D3F88A
:108370001025D9F81035914202D10599994205D0BE
:108380000492089ACDE90532099B8AE70BB0BDE853
:10839000F08F00BF0061004000600040206100409D
:1083A0000003005054610120AB610120D0F800317E
:1083B000103B102B07D8054A22FA03F313F0010FE4
:1083C00008BF002070470020704700BF0101010076
:1083D0002DE9F04F04468DB00846FFF7E7FF0D4644
:1083E00001900246214695F804014EF05CF995F89B
:1083F0000461231D013E099304F11003F6B20A93B0
:10840000627A637B62736279627262786271A27A65
:108410006370A378A270A27BA372A379A271E279A0
:10842000A373E378E270E27AE271E27BE272E373D3
:1084300025462246002312F823105148415C02F8D9
:1084400023100133042BF6D1099B01329342F1D161
:10845000019A214630464EF026F9002E00F08C801D
:1084600095F80080AB780093404665F09CFD029043
:1084700065F099FD039065F096FD6F780B90384696
:1084800065F091FD024665F08EFD049065F08BFD70
:108490008246009895F803B065F085FD059065F07B
:1084A00082FD069065F07FFD8146584665F07BFDB4
:1084B000079065F078FD089065F075FDDDE9023103
:1084C00083EA010C0B9B069983EA0C0C82EA0C0CE4
:1084D0008AEA0C0C81EA0C0C89EA0C0C009980EAFF
:1084E0000C0C87EA0C0C81EA0C0C04995A404A40A7
:1084F00005998AEA02024A40089989EA02024A403A
:108500004240009988EA02024A408BEA02026A70FD
:10851000039A05995A408AEA02024A4006994A405B
:10852000079989EA02024A40424088EA02027A40F8
:108530008BEA0C0C8BEA020B85F800C085F802B0C0
:10854000029A5340049A53408AEA030A089A89EA35
:108550000A0981EA09035340584000990A9B88EAB6
:10856000000887EA08077940E9700435AB427FF4D8
:1085700077AF013EF6B243E70DB0BDE8F08F00BF24
:10858000743A0A0010B54FF08043D3F804436207F1
:1085900007D54FF4847060F0D7F810B11E4B1B68FC
:1085A0009847A30608D54FF48A7060F0CDF818B14B
:1085B0001A4B00201B689847600608D54FF48C7052
:1085C00060F0C2F818B1154B01201B6898472106CE
:1085D00008D54FF48E7060F0B7F818B1104B00203A
:1085E0001B689847E20508D54FF4907060F0ACF82E
:1085F00018B10B4B01201B689847A3050AD54FF40F
:10860000927060F0A1F828B1054BBDE810401B68DE
:108610000220184710BD00BFE4620120E86201207B
:10862000EC620120DFED0A7A9FED0A7ADFED0A6A3B
:10863000A0EE277ADFED097AE7EE007AB7EE007A4E
:10864000A0EE267A67EE807A87EE870A704700BF31
:108650006BD30DBCBA132FBDAEE534BF75AA2A3E4D
:1086600002480322002122F0DFBE00BF00B000401C
:1086700002480422012122F0D7BE00BF00100140B1
:1086800002480422022122F0CFBE00BF0040024077
:1086900008B57E4A7E4B7F498B42C0F0BF807E4B3F
:1086A0007E4A00219342C0F0BE804FF08053D3F841
:1086B0003021082A4ED14FF080420021C2F80C111F
:1086C000C2F81011C2F8381502F54042D3F804146C
:1086D000C2F82015D3F80814C2F82415D3F80C14E6
:1086E000C2F82815D3F81014C2F82C15D3F81414B6
:1086F000C2F83015D3F81814C2F83415D3F81C1486
:10870000C2F84015D3F82014C2F84415D3F8241445
:10871000C2F84815D3F82814C2F84C15D3F82C1415
:10872000C2F85015D3F83014C2F85415D3F83414E5
:10873000C2F86015D3F83814C2F86415D3F83C14A5
:10874000C2F86815D3F84014C2F86C15D3F8443455
:10875000C2F8703555F088FF18B1514B514AC3F833
:108760008C2655F081FF18B14F4BFB22C3F818251A
:1087700055F07AFF58B14FF080424FF08051D2F857
:10878000E43ED1F8581261F30303C2F8E43E55F019
:108790006BFF20B1454B4FF40072C3F840264FF0F9
:1087A0008053D3F83031082B09D14FF08043D3F8F0
:1087B0000024D10744BF6FF00102C3F800243C4AF3
:1087C000D2F8883043F47003C2F88830BFF34F8F7B
:1087D000BFF36F8F4FF01023D3F80C22D20725D5AB
:1087E000344B0122C3F80425D3F80024002AFBD01F
:1087F0004FF01022D2F80C3223F00103C2F80C32F1
:108800002C4BD3F80024002AFBD00022C3F8042507
:10881000D3F80024002AFBD000F0ACFC52F8040B83
:1088200043F8040B38E743F8041B3BE7D3F8002276
:10883000002A03DBD3F80432002B22DA1D4B01227D
:10884000C3F80425D3F80024002AFBD04FF01022EF
:108850001221C2F80012D3F80024002AFBD04FF0F6
:1088600010231222C3F80422124BD3F80024002A4A
:10887000FBD00022C3F80425D3F80024002AFBD043
:10888000CAE70D4B0D4A1A6041F082F91C7F0A00BD
:1088900000000120DC050120000601201C6F0120E2
:1088A000005000404881030000F00040009002406A
:1088B00000ED00E000E00140000001200090D00346
:1088C0000149024847F09ABD18620120003000407B
:1088D00002494FF0402047F091BD00BF4C6201209B
:1088E00008B50748D0F8183143B14FF48C715FF0E8
:1088F00023FFBDE80840034857F06CBA08BD00BF2D
:1089000000300240B861012008B50748D0F818319E
:1089100043B14FF48C715FF00FFFBDE8084003488E
:1089200057F058BA08BD00BF00F00240DC610120DA
:1089300073B51F4C022501A861F0BAFC052812D1BD
:108940001C4D4FF40C741C48ADF802400DF10201AF
:1089500061F03AFC08B30C2803D1184918485AF0C2
:10896000F5FB02B070BD019B032B14D004D8022B81
:10897000E1D100232370DEE7A3F10902022ADAD84D
:108980000A2B06D0092B14BF0120022047F0FCFB64
:10899000D1E70020FAE72570CDE7D5F8B430002BF9
:1089A000D1D01E680448D3E9011290473346F6E758
:1089B000FE6E0120F4620120245F01205320090093
:1089C000546409000149024857F0FABF00620120CF
:1089D000009000400149024857F0F2BF0C620120AC
:1089E00000A000400149024864F021BA80620120E1
:1089F000002000400149024864F019BAA462012035
:108A0000008002402DE9F04FBC4BBD4AD3F8001363
:108A1000002385B01C4601201D4621FA03F6F60707
:108A20000BD552F8236046B100FA03F6344342F8FE
:108A30002350BFF36F8FBFF34F8F0133192BECD14E
:108A4000E10738D5AD4B0122C3F81425C3F8102532
:108A500000221546930003F1804303F51C330132D5
:108A6000082A5D609D62F5D1A44BA6485D629D64B5
:108A7000C3F85851D3F80024D3F800140A43C3F8BC
:108A80000024D3F80023C3F808239F4AC3F8042323
:108A900000214FF4927258F083FC9A4A8DF80850E6
:108AA00040231383138101214FF4807301A8ADF893
:108AB000043018F0E5F814F4006F924D07D08F4B96
:108AC000D3F8A836A5F81631012385F81C31A20287
:108AD00004F4800635D5894AD2F8143513F480732E
:108AE00008D01EB1D2F80034DB0702D408204BF0C6
:108AF00015FD0123814AD2F81015CF0540F14A81B6
:108B000095F81C318BB1002385F81C31B5F816316E
:108B10009BB24FF4E06203930121882301A8ADF8D2
:108B20000420ADF8083018F0ABF8744B4FF44072E5
:108B3000D3F820350293012101A8ADF8042018F0E4
:108B40009FF87EB36D4BD3F8006440F2017232405F
:108B5000F005C3F8002409D50121C3F82C1501A89C
:108B60004FF48063ADF8043018F08AF871050FD522
:108B7000624B0122C3F808259A65D3F8002312F44A
:108B8000001208BFC3F854214FF40012C3F80423A5
:108B9000B20507D54FF4A063012101A8ADF8043058
:108BA00018F06EF823022ED5544BD3F88014D3F866
:108BB0008424D3F888E4D3F88CC4D3F89074D3F821
:108BC0009464D3F89804D3F89C3411F07F0FD2B298
:108BD00001D1052A17D04FF4C0688DF808108DF820
:108BE0000E00012101A8ADF804808DF809208DF850
:108BF0000AE08DF80BC08DF80C708DF80D608DF8C3
:108C00000F3018F03DF8414B23403BB1BFF35B8F71
:108C10003F4B4FF000021A70BFF35B8F394FDFF804
:108C2000DCB00026B8464FF0140AB14606F10C033A
:108C300024FA03F3D80726D50AFB06B305EB461141
:108C4000D3F80827D8F8003013FA82F3C8F80030B8
:108C5000B1F806C090B2082E1CFA82F24FEA461311
:108C6000CA8000F0A480B8F80820824240F09F80BB
:108C7000CA88B8F8041092B2914240F2988016B9AE
:108C800024481AF0B7FE0136092E08F12008CDD18C
:108C9000214B2340002B00F09480184BD3F86C84B8
:108CA000C3F86C84BFF36F8FBFF34F8F14F48064ED
:108CB0001CBFD3F88044D3F88064DFF848A01DBF00
:108CC000C6F3C016C4F3C01486F0010626464FF062
:108CD00000094FF4E06B28FA09F1CA0703D4B9F18F
:108CE000000F31D184B3054B142202FB09315FFA26
:108CF00089F0D1F80836DAF810100FE00070024061
:108D000000710240E82101200514C001FCFB1F0096
:108D1000082301204C7002400004000151FA83F145
:108D2000CAF8101005EB4911B1F816E05EFA83FCA1
:108D3000A1F816C0B1F816C0BAF814E01FFA8CFCFE
:108D4000E6455ED94BF0CAFB09F10109B9F1080FFC
:108D50000AF1200ABFD100244FF0010904F11003E9
:108D600028FA03F3DB0701D474B96EB105EB4412A2
:108D70006301D17A002955D0D288B98892B2914244
:108D800050D9E0B24BF0CAFB0134082C07F12007A0
:108D9000E4D116E0002B7FF4C8AE95F82131002B0A
:108DA0007FF4C3AE4FF40013C2F80833BDE62B4482
:108DB000DA7A8AB94FF0E023D3F8F03DD90700D52D
:108DC00000BE1A4A1A4B136010460023536005B0C8
:108DD000BDE8F04F07F0E8BEDA88A8F8042083F871
:108DE0000B90DB888DF808609BB24FF4E0620121A4
:108DF00001A8ADF8042003938DF8099017F040FF07
:108E000041E7C98AADF804B089B260F07F000391F0
:108E100000218DF808008DF8091001A8012117F034
:108E20002FFF91E72B4483F80A90ADE7BC6801203F
:108E3000DBD0080010B5074CD4F800314BB1064B1D
:108E40005B68984720464FF48071BDE810405FF0A2
:108E500073BC10BD00000140C8620120022A2DE948
:108E6000F04159D13B4B826883FB02423A4D846901
:108E700085FB046422440A60DFF8F0C042688CFB82
:108E80000242364EC46986FB047422444A6002687A
:108E900083FB0242046A85FB046422448A60304EEC
:108EA000026886FB02422F4C056A84FB05752A4442
:108EB000CA604FF06045426885FB0272C76985FB56
:108EC00007E73A440A61826884FB0272876986FB7D
:108ED00007E73A444A61426983FB02728A61026988
:108EE0008CFB0272CA61C26883FB02720A62C368A9
:108EF00086FB03234B62036985FB03238B62436973
:108F000084FB0323CB620023C1E91033C1E90E3394
:108F1000C1E90C33BDE8F081134B902404FB02320D
:108F200002F1480E02F18C0501F14406683250F856
:108F3000043B55F804795EF804CB1C468CFB048492
:108F400041F8044B87FB0343AA4246F80439EED1AB
:108F5000E0E700BFD8E3CEB8281C3107CD3C410D77
:108F60009A615FC9669EA0F670710A0033C3BEB2F3
:108F70002DE9F8431C4E04468846914600254FF4DF
:108F8000004746F00106B4F85E20ABB29A4205D81D
:108F900094F83400BDE8F84336F00CBF03F00F033B
:108FA00047FA03F313EA090F14BF012100212046F9
:108FB0004EF0DCF9B4F85E30AAB2A3EB08039A4293
:108FC00003DD94F8340036F023FF94F8610036F0A6
:108FD0001FFF4020B04794F8610036F0EBFE4020C0
:108FE000B0470135CFE700BF00210A00F8B590F87F
:108FF0006530013B80F86B3090F866305A1E80F87F
:109000006C20012B88BF90F86C304FF000058CBFAE
:1090100003F1FF33012380F86D30044680F86E5071
:109020000127856540F2033694F86330EAB2934233
:109030003CD82368314A934257D002F5805293427C
:1090400055D002F58052934253D002F580329342BC
:1090500051D002F5805293421ED10423284850F883
:10906000332000EBC300002590F90430012151604A
:10907000002BC2F80455D160C2F80855C2F810554B
:109080004FF48035C2F8045306DB5A0903F01F037E
:1090900099401C4B43F82210236801224FF47A7147
:1090A0005A60DA60C3F840151A60F8BDA36C03EB90
:1090B00002131B7B1F2B86BF03F01F0312494FF0C7
:1090C000A04103F5E07341F82360A36C94F86D10A0
:1090D00003EB02133942187B04D036F099FE7F006F
:1090E0000135A1E736F066FEF9E70023B6E7012374
:1090F000B4E70223B2E70323B0E700BF00800040DB
:10910000CC6B0A0000E100E00003005000280CDBFB
:109110004309064900F01F0020330122824041F834
:109120002320BFF34F8FBFF36F8F704700E100E044
:109130004309064900F01F0020330122824041F814
:109140002320BFF34F8FBFF36F8F704700E100E024
:109150000028ABBF00F16040054B00F5614000F016
:109160000F004FEA4111B4BF195480F80013704743
:1091700014ED00E0BFF34F8F0549064BCA6802F4B7
:10918000E0621343CB60BFF34F8F00BFFDE700BF2A
:1091900000ED00E00400FA05014B1868704700BFBD
:1091A0005400012007EE900AF5EEC07AF1EE10FAB5
:1091B00001D400F009B808B580F0004000F004F8D0
:1091C000404261EB410108BD70B5FEF793F80C4BCE
:1091D000002204460D46FEF7ABFAFEF7D5FB064625
:1091E000FEF766F8074B0022FEF7A2FA02460B468E
:1091F00020462946FDF71EFFFEF7C6FB314670BD2F
:109200000000F03D0000F04170B510EE105A25F05E
:1092100000440123B4F1FF4FB0EE403A064603602C
:1092200004D320EE003AB0EE430A70BD34B9DFED4E
:10923000D07AB7EE007A87EE273AF4E7B4F1E45F2C
:109240000BD2002DBEBF4FF0FF330360B1EE400ADA
:1092500024F084FDB1EE403AE5E7002D80F2C682AD
:10926000B4F1964FE3D2B4F17A5F9FEDC25A78D24F
:10927000DFEDBF0A20EE050A002000F015FEF0EE3B
:10928000402AF5EE402AF1EE10FAD0D023EE220A61
:10929000B0EEC00A85EE000A24F060FDF5EEC02AAB
:1092A000F1EE10FAB0EE402A40F1B9804FF0FF33F2
:1092B000B4F17E5F336000F09382B4F1804F00F030
:1092C0008F82B1EE433A6B0000F1DE81AA4B9C42E3
:1092D00000F2F580B0EE430A24F040FDA74B9C421B
:1092E000B1EE400A40F29D80B7EE007A37EE437A45
:1092F00067EE077ADFEDA26A9FEDA26A9FEDA23AC0
:10930000A7EEA66ADFEDA16AE6EE276A9FEDA06AE6
:10931000A6EEA76ADFED9F6AE6EE276A9FED9E6ADA
:10932000A6EEA73ADFED9D6AE7EE866A9FED9C6A9E
:10933000A6EEA76ADFED9B6AE6EE276A9FED9A6AC2
:10934000A6EEA76ADFED996AE6EE276A23EE073AF2
:10935000A6EEA73AF6EE007AA7EE673A33EE003AA9
:10936000FFE0B1EE407AB0EE470A1DF063FAB4EECA
:10937000407AF1EE10FA19D0F6EE007A27EE277A4D
:10938000B0EE470A1DF056FA37EE400A30EE000AFA
:10939000F0EE407AFEEECF7A17EE903A062B39D8EF
:1093A000DFE803F02312121F1F2B2B00DFED807A62
:1093B00077EEC37A17EE903A03F0010307EE903A86
:1093C0009B00B8EEE70AE9E7F6EE007A37EEC00A4E
:1093D000DFED670A20EE050A00F036FBF1EE402AC9
:1093E0004FE7F7EE007A37EEC00ADFED610A20EEB4
:1093F000050A002000F058FDF0E7F7EE087A30EE9D
:10940000670ADFED5B0A20EE050A00F01DFBB1EEF6
:10941000400AE3E7F0EE007A30EE670AE5E7012361
:1094200046E7644B9C4264D99FED637A33EE477AFA
:1094300067EE074A9FED616ADFED616ADFED615A11
:109440009FED615A9FED613A64EE877AE7EE866A96
:109450009FED5F6AA6EEA76ADFED5E6AE6EE276A19
:109460009FED5D6AA6EEA76ADFED5C6AE7EEA65A9D
:10947000DFED5B6AE5EEA76ADFED5A5AE6EEA75A22
:10948000DFED596AE5EEA76ADFED585AA7EEA55A57
:10949000DFED575AE5EE275A9FED565AA5EEA75A2B
:1094A000DFED555AE5EE275AE5EE876AA6EEE73A74
:1094B000DFED527A94EE863A33EE673A4EE7504B40
:1094C0009C4206D9B0EE007A37EE437A9FED280A27
:1094D0000EE74C4B9C4206D99FED4B7A9FED240A38
:1094E00033EE477AA4E7F7EE007A33EE673A9FED62
:1094F000200A9FED467ADFED467ADFED466AE3EE1D
:10950000077A9FED457AA7EE837ADFED447AE7EE9E
:10951000037A9FED437AA7EE837ADFED4D7AE7EE8B
:10952000037A9FED407AE3EE076A9FED3F7AA6EE5D
:10953000837ADFED3E6AE7EE036A9FED3D7AA6EEA1
:10954000837AF7EE006AE7EE036A67EE837A87EEC6
:10955000A67AFEEE006AF0EE477AE3EE267A37EE60
:10956000803A002DBFF65FAE32EE433A5BE600BFB5
:1095700000000000DB0F49406666663F1F4A3B3F24
:10958000A283D337679767393F239E3DA1549C3A06
:109590007E02F23B01F0893D752C3C384584E2386F
:1095A00034B6053AC66E3D3B1599A83C661AA53EF1
:1095B0000000004B07336D3E0C5BEC3E6B7BA53926
:1095C00076F4B7BA67F8663A85300DBA521CE631C0
:1095D00007E7C73B474D06BD5EB9F73E27F9A3B97C
:1095E000FE7771BB3D37933C3C2117BEF7E9AF399D
:1095F0009916143BFEFC28BC155A843DCDCDF83D90
:1096000017A6DD3F1FA69D3FC316BB3F5E3C5B3CDC
:1096100078756A3EAF72D53DB24B7A3FE73ABA3FB2
:10962000F400223FDBD5523BDFEF443F2D390840A9
:10963000BE2E1D4067FF0538B435F13ABDD7F5366B
:10964000E440DA3CE6DC153E7ACCA63E5A245C3E89
:109650003F239EBDD6EE4B3A54BF983C6E0F303E32
:10966000C5D0383F3B2DB23FE8C4D5BAD23D5B3AB6
:109670005C061CBAFD0C503A610B36BBABAAAA3D86
:109680001D7FD63E00000000B4F1824FF7EE002AA5
:1096900075D2FDEEC35A1FED197A5FED196A1FED01
:1096A000196AF8EEE57A15EE903A73EE677A033BA5
:1096B000E7EE876A1FED1E7AA6EEA77A5FED1F6AB6
:1096C000E7EE276A1FED207AA6EEA77A5FED216A02
:1096D000E7EE276A1FED227AA6EEA77A5FED236AEE
:1096E000E7EE866A1FED246AA6EEA76A5FED256A9B
:1096F000E6EE276A1FED266AA6EEA76A5FED276AE7
:10970000E6EE276A27EE277AE6EEA72A87EE223AC8
:10971000B6EE007AA7EE873A042B3FF622AFDFE8D9
:1097200003F02B2825220300B1EE087A37EE877A62
:10973000F1EE046A77EEA66A66EE876AB1EE007A09
:1097400037EE877A27EE267AB0EE080A37EE800ADF
:1097500020EE070AB0EE007A77EE877A27EE800ACD
:1097600024F0FCFAFAE5B7EE007AE1E7F7EE006ADA
:10977000E4E7B7EE007AE7E7B7EE000AEAE7B0EE13
:10978000430A24F0EBFAB4F1B94F30EE620A24D266
:10979000C2EE836A5FED4C5A1FED4C6A66EEA67A04
:1097A000B6EE007AA7EEA56A5FED4F5AE6EE275AAD
:1097B0001FED506AA5EEA76A5FED515AE6EE275AF3
:1097C0001FED526AA5EEA76A33EE477A1FED543AB1
:1097D000A6EE263AA7EE003AC3E623EE003AC0E62C
:1097E0001FED583AC0E61FED593A1CE5B4F17E5F13
:1097F000F9D0B4F1804FF6D01FED5E2A63E500BFCB
:109800007FB510EE105A834A25F000439342044678
:1098100005D8002380ED000A4360002022E07E4A44
:1098200093423AD825F00043002DDFED7C7A7C4A44
:1098300023F00F0318DD934230EE670A09BFDFED16
:10984000797A9FED797A9FED797A30EE670A70EE3A
:10985000477A30EE670AC0ED007A30EE470A80EDB5
:10986000010A012004B070BD934230EE270A09BFFF
:10987000DFED6C7A9FED6C7A9FED6C7A30EE270A03
:1098800070EE077A30EE670AC0ED007A30EE070A14
:1098900080ED010A4FF0FF30E4E7654A93426DD84E
:1098A0009FED647AB0EEC00AF6EE007AE0EE077A39
:1098B000FDEEE77AF8EEE76A17EE900ADFED577AE9
:1098C000A6EEE70A1F28DFED587A66EEA77A30EE9B
:1098D000677A09DC5849461E25F0004251F82610E7
:1098E00022F0FF028A4207D117EE102AC2F3C752B4
:1098F000C2EBD352082A02DC84ED007A1BE09FED14
:10990000497AB0EE406AA6EEC76A70EE467AE6EE95
:10991000C77A9FED467AD6EE877A36EE677A17EEEB
:10992000102AC2F3C752C2EBE353192B15DC84EDA6
:10993000007AB0EE460A30EE470A002D30EE670A94
:1099400084ED010A8EDAB1EE477AB1EE400A84ED79
:10995000007A84ED010A404284E79FED387AB0EE48
:10996000460AA6EEC70A76EE407AE6EEC77A9FED83
:10997000347AD6EE877A30EE677ABDE7B3F1FF4FDF
:1099800006D330EE400A80ED010A80ED000A44E77C
:10999000DA15863AA3EBC25307EE903ABDEEE77AAA
:1099A000DFED286AB8EEC77A77EEC77A8DED017AD7
:1099B00067EEA67ABDEEE77AB8EEC77A77EEC77A99
:1099C0008DED027A67EEA67AF5EE407AF1EE10FAA6
:1099D000CDED037A19D1B5EE407AF1EE10FA16D03A
:1099E0000223214601A800F089F8002DBFF63AAF06
:1099F000D4ED007AF1EE677AC4ED007AD4ED017A05
:109A0000F1EE677AC4ED017AA5E70323E9E70123C4
:109A1000E7E700BFD80F493FE3CB1640800FC93FAF
:109A2000D00FC93F004435374344353708A3852E4E
:109A3000800F494384F9223F04660A0000A3852E63
:109A400032318D240000804310EE103A23F00043A1
:109A5000B3F1485FB7EE007A04D2FDEEC07A17EE9C
:109A6000902ABAB360EE006ADFED1C5A9FED1C6AC3
:109A70001C4AA6EEA56A9342DFED1B5AE6EE265A73
:109A80009FED1A6AA5EEA66ADFED195AE6EE265A90
:109A90009FED186AA5EEA66A60EEC00A26EE266A59
:109AA000F6EE007AE6EE860A66EEA77A04D877EE3E
:109AB000E07A37EE670A70470F4A93429ABF03F184
:109AC0007F4306EE903AF5EE026A37EE667A77EE5D
:109AD000E67AECE7B0EE470A704700BF4ED747ADD5
:109AE000F6740F319999993E7CF293B4010DD037F9
:109AF000610BB6BAABAA2A3D0000483F2DE9F04FF2
:109B00009246033A48BF0AF10402D7B0D2109B46EE
:109B1000551C2DB202910BF1FF31EB0080460DF187
:109B20006809501A0BF1090CC24F0393AAEBC50543
:109B300000EB0C064C460028AABF3B5CDFEDC17A67
:109B400007EE903A00F10100A8BFF8EE677AB04244
:109B5000E4EC017AEFD142AF08EB8B0309EB8B0405
:109B60000193BE46DFEDB77A26464046F0EC016A27
:109B7000019B36ED017A9842E6EE877AF6D1013103
:109B80008C45EEEC017A04F10404EBD1A949DFED38
:109B9000AA6A9FEDAA6A531809240593A3000493A7
:109BA00056AB03EB840212ED140A07EB840006A9FE
:109BB0002246002A45DC28463EF01AF9B0EE407AEB
:109BC000B4EE000A27EE000A1CF034FEF2EE007A32
:109BD000A0EE677A002DFDEEC77A17EE906AF8EED8
:109BE000E77A37EE677A3EDD06AA601EC5F1080EF9
:109BF00052F8203043FA0EF10E4401FA0EF1591AD0
:109C000042F82010C5F10702114100293ADD002277
:109C100001360DF1180E1346944255DC002D03DD7C
:109C2000012D62D0022D6AD002292BD1B7EE000A95
:109C300030EE477A33B328463EF0DAF837EE407A12
:109C400020E060EE267A013AFDEEE77AF8EEE77A58
:109C5000A7EEC60ABDEEC00AA1EC010A30ED010A6A
:109C600037EE800AA5E705D1621E06A951F8221039
:109C70000912CAE7F6EE007AB4EEE77AF1EE10FACE
:109C800020DA0021B5EE407AF1EE10FA40F084803F
:109C9000601E00230DF1180E082838DC002B56D169
:109CA0000FA9012251F8040DB0B3049B3E1D04EB33
:109CB0000B01601C1E4409EB8101224490422DDD02
:109CC00014466BE70221A2E7DEF8000053B920B189
:109CD000C0F58070CEF80000012001320EF1040EB4
:109CE000034699E7C0F1FF00F4E704F1FF3E06A840
:109CF00050F82E2002F07F0240F82E2094E704F165
:109D0000FF3E06A850F82E2002F03F02F4E75EF86E
:109D1000202001381343BFE70132C3E7059B1B5CDA
:109D200007EE903AF8EE677A4446E1EC017ADFED0F
:109D3000457A8C46F4EC015A019B3CED017A9C4239
:109D4000E5EE877AF6D1E6EC017A0130B6E7013C20
:109D5000083D06AA52F82430DBB12846B7EE000AC7
:109D60003EF046F89FED347A381D4FEA840800EB48
:109D70008400234606AD002B3CDA2346002B63DB30
:109D8000DFF8BCE0DFED2F7A07EB830C0025E01A4B
:109D900047E0013C083DDDE7039BB0EE470AA3EB3B
:109DA0000A003EF025F89FED257AB4EEC70AF1EEE1
:109DB00010FA19DBDFED207A60EE277A06AAFDEEB5
:109DC000E77A0835F8EEE77AA7EEC70AFDEEE77AFC
:109DD000BDEEC00A10EE103A42F8243017EE903A69
:109DE000013442F82430B8E7BDEEC00A06AA10EEEE
:109DF000103AF6E755F8232007EE902AF8EEE77AB6
:109E0000013B67EE807A20EE070A60ED017AB2E747
:109E1000FEEC016ABCEC017A01350A2DE6EE877A88
:109E200001D08542F4DD56AA02EB800040ED287A8D
:109E3000013BA3E784660A000000803B00008043EA
:109E40004C670A00000000002FA81FED027A00EB0B
:109E500008032246002A17DAE1B1F1EE477A029BA5
:109E6000C3ED007ADDED2E7A77EEC77A01239C42AE
:109E700013DA09B1F1EE677A029B06F00700C3ED31
:109E8000017A57B0BDE8F08F73ED017A013A37EEF1
:109E9000277ADFE7F0EE477AE1E7B0EC017A0133A9
:109EA00077EE877AE3E700BF10EE103A23F0004325
:109EB000B3F1485F04D2FDEEC07A17EE903A5BB37F
:109EC00020EE007ADFED157A9FED156AA7EE276A7E
:109ED000DFED147AE6EE077A9FED136AA7EE876A44
:109EE000DFED127A60EE076AE6EE077A30B99FED91
:109EF000106AA7EE276AA6EE260A704767EEE67A92
:109F0000B6EE006AE0EE867AD7EE870ADFED097AD0
:109F1000E6EEA70A30EE600A704700BFD3C92E2FC5
:109F2000342FD7B21BEF3836010D50B98988083C61
:109F3000ABAA2ABEABAA2A3E10EE103A23F000428A
:109F4000B2F1465FF0EE407A14D2BDEEC07A17EE61
:109F5000101A29BB431C134306D1F0EEC07AB7EEAA
:109F6000007A87EE270A7047012800F09B80BFEE39
:109F7000007AF6E74C498A4212D3002B9FED4B7AC8
:109F8000B8BFF1EE407A37EE677ADFED497AB8BFB5
:109F9000F1EE600A77EEE07ADFED460A77EE877A37
:109FA00067EEA76ADFED445A9FED446A9FED445A7D
:109FB0003D4926EEA67A67EEA64AA7EE256A8A42B2
:109FC000DFED405AE6EE075A9FED3F6AA5EE876A3D
:109FD000DFED3E5AE6EE075A9FED3D6AA5EE876A31
:109FE000DFED3C5AE7EE055A9FED3B5AA5EE875A46
:109FF000DFED3A5AE5EE075A9FED395AA5EE875A3A
:10A00000DFED385AE5EE075AB0EE467AA5EEA67AAD
:10A01000B0EE606AA7EE246A9FED337AE6EE260A78
:10A02000E4EE870A37EEA00A1DD307EE100AF8EE19
:10A03000C76A60EE005A30EE260A9B1785EE806AEA
:10A0400003F00203C3F1010307EE103A36EE606A33
:10A05000B8EEC77A77EEC67AB0EE006AE7EEC66A67
:10A0600026EE870A704701281CD010EE103A6FF3D5
:10A070000B0306EE903A76EEE77A70EEE70AFFEE13
:10A08000007A87EE807AF7EE007A17EE103A6FF3D7
:10A090000B0300EE103AE6EE807AE0EE807AA7EE4F
:10A0A000870A7047704700BF40A12C3FDA0F493F35
:10A0B00068212233000000005FAE9BB745F4A3384F
:10A0C0008453D937C8261A3A16696B3BA427B33C88
:10A0D0008988083E7AC09538B937813948DEBE3A5A
:10A0E0001F37113CD10D5D3DABAAAA3E42084B087B
:10A0F00002F0553203F05533801AC91A8A088308D2
:10A1000001F0333100F0333002F0333203F03333F7
:10A110000344881803EB131300EB101003F00F3304
:10A1200000F00F30184400EB002000EB0040000E60
:10A13000704700BF2DE9F04782B00646DDF828E001
:10A140000846B4460D46002B4ED18A4214466DD9BE
:10A15000B2FA82F242B1C2F12003954026FA03F32B
:10A1600094401D4306FA02FC260CA7B2B5FBF6F19B
:10A170004FEA1C4306FB115543EA054301FB07F078
:10A18000984209D9E31801F1FF3580F00381984224
:10A1900040F20081023923441B1A1FFA8CFCB3FBE6
:10A1A000F6F006FB10334CEA034C00FB07F3634563
:10A1B0000AD914EB0C0C00F1FF3580F0ED806345FB
:10A1C00040F2EA80A444023840EA0140ACEB030CC0
:10A1D0000021BEF1000F04D02CFA02F30022CEE9D8
:10A1E000003202B0BDE8F0878B4209D9BEF1000F02
:10A1F00001D0CEE900610021084602B0BDE8F08739
:10A20000B3FA83F1174600294DD1834202D3B242FB
:10A2100000F20F81B6EB070C60EB030301201D4633
:10A22000BEF1000FDDD0CEE900C5DAE7002A00F06C
:10A2300098801A46B4FA84F3002B40F0AF800B1BD1
:10A24000270CA6B20121B3FBF7F54FEA1C4007FB30
:10A25000153340EA034306FB05F8984507D9E31890
:10A2600005F1FF3002D2984500F2E8800546A3EBE5
:10A2700008031FFA8CFCB3FBF7F007FB10334CEA22
:10A28000034C06FB00F3634508D914EB0C0C00F1FA
:10A29000FF3602D2634500F2CE803046ACEB030CB1
:10A2A00040EA054095E7C1F120058B4022FA05FC04
:10A2B0004CEA030C00FA01F426FA05F3E84002FA2E
:10A2C00001F943EA04084FEA1C4206FA01FAB0FB1E
:10A2D000F2F71FFA8CF602FB17004FEA184444EA23
:10A2E000004407FB06F0A0420AD91CEB040407F166
:10A2F000FF3380F09C80A04240F29980023F64448A
:10A30000241A1FFA88F3B4FBF2F002FB104443EA6C
:10A31000044300FB06F69E4209D91CEB030300F13F
:10A32000FF3480F082809E427FD90238634440EA45
:10A330000740A0FB09749B1BA3423E46A04664D382
:10A3400061D0BEF1000F0AD0BAEB060263EB08033E
:10A3500003FA05F5CA401543CB40CEE9005300216E
:10A360003FE7730843EAC1734A08190C41EA024106
:10A370004FEAC67C9BB2B2FBF4F02646A0462746C5
:10A380001F2243EA0143B1FBF4F1A3EB080341EAC6
:10A39000004158E72946FFE6284615E71A46C3F16B
:10A3A00020019C4026FA01F320FA01F1904003437A
:10A3B000270C06FA02FCB1FBF7F0A6B207FB10155A
:10A3C000190C41EA054100FB06F58D423BD96118A5
:10A3D00001D28D4220D8491B0138B1FBF7F5019518
:10A3E00005FB06F8019D9BB207FB151143EA0143EB
:10A3F000434526D2E31805F1FF31C6D24345C4D206
:10A40000A91E2344C1E7BA459BD2B7EB090664EB0A
:10A410000C040138A04694E7651B29440238B1FBBF
:10A42000F7F5019505FB06F8DCE720467FE71F46B8
:10A4300066E70846F4E6A44402382FE7023D2344C9
:10A4400015E70199A1E7491BB1FBF7F5019505FB5C
:10A4500006F8C7E72DE9F0410D4606464FF0AAFA87
:10A46000294640F2FF4058F07EFE06F108070446F8
:10A4700090B1436828469847A36801219B69054627
:10A48000984710B1294846F0B5FBA36839462846DD
:10A490009B68BDE8F04118472549284657F09DFFC5
:10A4A000044618B390F85030D906EBD443F01003AB
:10A4B00080F85030394653F0D1FE96F82A3003F038
:10A4C0000C03002B94F8513014BF0122002223F01A
:10A4D000060343EA420384F8513005D194F8503022
:10A4E00043F0020384F85030BDE8F081114928465A
:10A4F00057F073FF0446B0B190F82A309A07C1D4E0
:10A5000043F00203394680F82A3053F04AFC96F8AB
:10A510002A1001F00C010039204618BF0121BDE8C6
:10A52000F04153F025BC0448ADE700BF624A090082
:10A53000B8C509001CC60900554A09002DE9F743B2
:10A540000746002608466A4601A9019658F08FFB87
:10A550000199022902D8234846F038FB7868012285
:10A5600089001DF0B3FC7E6080463E81019BB4B241
:10A57000A34206D85B00C7F804803B8103B0BDE866
:10A58000F083009B184953F8245040F2EA422846D1
:10A5900025F0FAFD686840F2EA42022125F0B2FD9A
:10A5A000A86840F27B6125F01DFE40F27B6347F610
:10A5B000FF720E49814657F07FF8E86840F28161EA
:10A5C00025F010FE094940F2816347F6FF72054607
:10A5D00057F072F828F8249008EB8404013665805F
:10A5E000C4E700BFF3470900FC2809000080FFFF13
:10A5F0002DE9F04F2DED028B91468DB0C268BDF86C
:10A6000064B0DDF86880BDF86C701D9C06468A4613
:10A610001D46B0EE408A82B980F845204BEA070318
:10A620001F2B14D8BAF1000F40F08980002F00F0E2
:10A63000B28054464FF0040A13E043689A4200F097
:10A64000B380002380F845300FF0B2FEE6E7BAF1A0
:10A65000000F40F09580002F00F0968054464FF098
:10A66000080AB9F1000F00F09C8040F20122ADF819
:10A670001820002D00F093806A1CADF81A200022EB
:10A68000079206A85FF0CCFD8146002851D1182220
:10A6900001460DEB020056F083FEDFED457A9FED9B
:10A6A000457A454B8DF818A028EE278A5D43C8EE01
:10A6B000077A42F210734F4508BFC846B5FBF3F561
:10A6C0004846189BADF82450012507948DF82D506D
:10A6D0000293ADF80CB0CDF81080ADF81470B6EE62
:10A6E000007A77EE877AFCEEE77ACDED087A4DF0C6
:10A6F0002BFC8146E8B9314C06AA02A920465FF03E
:10A7000069FD8146A8B92E49324606F128000BF0B2
:10A7100025F89DF97020217828465FF08BFD814651
:10A7200038B9207829465FF057FD814608B9189B53
:10A73000F36048460DB0BDEC028BBDE8F08F3CB332
:10A74000F0EE0C7AB4EEE78AF1EE10FA6946204694
:10A7500010D807EE905A9FED1B7AF8EE677AF4EE68
:10A76000C77AF1EE10FA05D84DF0B2F86C464FF00A
:10A77000020A76E74DF0ACF80C464FF0030A70E79A
:10A7800000244FF0060A6CE73C464FF00A0A68E7DF
:10A790004FF0010A65E73C464FF0050A61E72A469B
:10A7A0006BE7CDE906996CE74FF01109C1E700BFEF
:10A7B0000024744900401C4440420F00B9050120A8
:10A7C0002D8007006666A63F2DE9F8434160994653
:10A7D0004B680B9F90469A790A9B80F82C20038542
:10A7E0008D7D044605F0300605F0060572B34B6812
:10A7F000D8684EF0F3FBE0842DB10023C4E9028950
:10A80000C4E90433A361002384F82D3084F82A308E
:10A81000A384089BE361099B23621AB3EFB11B4930
:10A82000224638460AF09AFF5DB115F0040118BFC0
:10A83000012160681ABF84F82B10002201220FF05A
:10A8400061FFDEB1B20616D4012315E04FF6FF73A7
:10A85000C3842B4635461E46CEE70C4821460AF0F7
:10A8600061FFE1E767B10A49224638460AF076FF00
:10A8700026B17307E8D4022384F82B30BDE8F883AF
:10A88000034821460AF04EFFF2E700BFAD8A0800F8
:10A89000178B080037B504464FF6FF70236100237D
:10A8A000A080A160E271A371E3608B88ADF80430F1
:10A8B000501C8B798DF80630221D01A9C0B25FF0C3
:10A8C000D7FC054678B9094AA18813888B4228BF6E
:10A8D0000B461380064A13888B4238BF0B46084646
:10A8E000138000F08BF8284603B030BDA00501208E
:10A8F000D06A01202DE9F04F89B081469DF848606B
:10A9000015465FFA81F81C46002B36D043681A7949
:10A910001B680621C3F800151D4B342101FB0233CF
:10A9200086F00106022283F82D207201194E4FF0A5
:10A93000000AB4F5806F274603A928BF4FF480674B
:10A940004846CDE9047ACDE9065A8DF80CA08DF879
:10A950000D80019200F0C2FDB042834603D1E41B9A
:10A96000019A3D44E5D1D9F8040035F08FFD5846F1
:10A9700009B0BDE8F04F45F01FBD414610F010F999
:10A98000A0420CBF6FF01200204609B0BDE8F08F66
:10A99000186201200000AD0B074A002311688142B4
:10A9A00001D1184670470133082B02F10402F5D19A
:10A9B0004FF0FF30704700BF0C4701200C4B187858
:10A9C00001280DD10B4B1B78FF2B0BD10A4B1868BC
:10A9D000C20708D4C30308D4800C00F004007047F9
:10A9E0000228F3D17047052070470120FAE700BF25
:10A9F000446F01204C6F0120006701202DE9F041D8
:10AA0000094D0746884600244FF6FF7635F81400B6
:10AA1000B04203D0424639465FF02EFC4434B4F5D0
:10AA2000AA7FF3D1BDE8F081A0090120034B53F8C0
:10AA3000203013B19A6801329A607047E4200120F7
:10AA400038B5144B53F82040ECB1207935F0D0F9EB
:10AA50000546607935F0CCF9A2790F49E37940EAEF
:10AA6000450000F0030040EA8202A0718A5C1344B2
:10AA700094F908205BB29342E37105DBE36801338C
:10AA8000E3600023E37138BD52429342FBDCE3688C
:10AA9000013BF5E72C470120ED200A002DE9F04F9E
:10AAA0000546A7B08A460146002058F05CFB09AC79
:10AAB000002841D1CDE913000CAA7E21284629F0B7
:10AAC00061FEA94B0F9301224023CDE9102316AB61
:10AAD00012930FAB0E93A54B09940A9300260820FE
:10AAE000CDE9050656F02CFB07902046CDE903661C
:10AAF0008DF8206055F0CBFFDFF880B23746354641
:10AB00009DF85490B9F1000F13D0204655F0BFFFC7
:10AB1000B9F15D0F00F092804AD8B9F13A0F3BD8F5
:10AB2000B9F11F0F14D8B9F10A0F31D8B9F1080FD4
:10AB3000E6D88F4846F05EF80121284629F014F83F
:10AB400043680A93002309950B938DF85430C5E7A9
:10AB5000A9F12002D2B20123934013EA0B0F40F077
:10AB60000F81844A1340CBD1B9F1220FE1D1069372
:10AB70009DF854100029DCD0222940F0A480204602
:10AB800055F085FFDDE906102CF000FA81462CE037
:10AB9000B9F10D0FB4D0CCE7B9F15B0FC9D10020EA
:10ABA00022F030FE8146002D3AD04FF0010821E01E
:10ABB000B9F1740F70D039D8B9F1660F4FD0B9F12F
:10ABC0006E0FB6D19DF85430752BB2D1204655F09A
:10ABD0005EFF6C28ADD1204655F059FF6C28A8D1F6
:10ABE000204655F054FF4FF00E09002D00F00E8165
:10ABF0004FF00008604B9F4240F0F58049462846E0
:10AC000057F0FFFFB8F1000F3FF47AAF049B002B21
:10AC100040F0F780012101A82BF08CFF049B1D6000
:10AC200048462BF09FF84D46074669E7B9F17B0F80
:10AC300000F0D580B9F17D0F7FF47BAF002D3FF49C
:10AC400078AF039B002B00F00081013B049A039333
:10AC500052F8235028462BF085F8074650E79DF818
:10AC60005430612B7FF465AF204655F010FF6C28FF
:10AC70007FF45FAF204655F00AFF73287FF459AF89
:10AC8000204655F004FF65287FF453AF204655F069
:10AC9000FEFE4FF01E09A8E79DF85430722B7FF49A
:10ACA00048AF204655F0F3FE75287FF442AF2046AA
:10ACB00055F0EDFE65287FF43CAF204655F0E7FEE9
:10ACC0004FF03E0991E75C290CD1204655F0DFFE9C
:10ACD0007528014606D86D2808D8622840D0662815
:10ACE00008BF0C2105A862F075FD35E0A0F16E03E8
:10ACF000072BF7D801A252F823F000BF1DAD0200C8
:10AD0000E5AC0200E5AC0200E5AC020065AD020076
:10AD1000E5AC020021AD020025AD02000A21E1E709
:10AD20000921DFE74FF000084FF00409204655F0F5
:10AD3000AEFE40F02000A0F130025738D2B2C0B2CF
:10AD4000092A88BF0246B9F1010942EA0818EDD183
:10AD5000414605A862F050FD204655F098FE07E7F1
:10AD60000821BFE70D21BDE7385E0900410A080050
:10AD70004E35090001100004A45D09000020FF0306
:10AD8000002306939846494605A862F023FD9DF8E6
:10AD90005490B9F12E0F17D009F0DF03452B13D0D3
:10ADA000B9F12B0F12D0B9F12D0F0FD0484645F055
:10ADB00059FE024650B9DDE90610B8F1000F09D07E
:10ADC000134658F03EF9E1E64FF00108204655F0F1
:10ADD0005EFED8E743460A222DF08EFFD6E600201D
:10ADE0002BF07AFFDEE62EB9B8F1000F7FF4A1AEAA
:10ADF0004E4685E631464A46284657F047FB002630
:10AE000000E7294601A857F0FCFE09E7BAF1000F58
:10AE100011D0B9F1000F3FF48CAE039B002B7FF4EF
:10AE200088AE05A862F04DFD484627B0BDE8F08F1A
:10AE3000204655F02CFE9DF85450284645F026FE3D
:10AE40000028F5D1002DE4D073E6A946BAF1000F31
:10AE5000F1D0E2E7C20713B5044603D5C0F34700BB
:10AE600002B010BD830707D102680E4B9A4203D18E
:10AE70002AF066FFC0B2F3E7204657F08FFE48B1D4
:10AE800020462AF0E5FEFCEEC07ACDED017A9DF871
:10AE90000400E5E720462AF065FF5E22C1880248EB
:10AEA00045F09CFEC0320900CA4009002DE9F04F70
:10AEB0000546E3B058484FF09CF8061E09DB574C96
:10AEC0006388B3F57F7F08D340F2512323803DF0A0
:10AED000FFFB002063B0BDE8F08F1A1DAA4200F20C
:10AEE0009880591E251D4E486A5C2F2A4FF000029B
:10AEF0000CBF6A54EA5405A954F094FD494B074627
:10AF0000186010B11BF050F920B940F25133238082
:10AF10003046DCE707F18000059A06A953F019FFD7
:10AF200040F2511345F8043C0023C4E901330746BD
:10AF3000E36010B103236370EAE71AAD294606A85F
:10AF400053F0F3FF08B9AB7E93B9002106A853F084
:10AF5000ECFF4FF00009A7604F450FD106A853F052
:10AF6000F9FB0023A26863806260E360A361CFE71E
:10AF7000294606A853F0D9FF0137E3E7294606A87A
:10AF800053F0D3FF6B892989C4F8049003F01F02A2
:10AF90005200480A0192C3F344120092DB0A01F006
:10AFA0001F0200F2BC70C1F3431161F0B8FA1E4BEE
:10AFB000A0FB0303C4E904032B7B13F0100318BFA9
:10AFC00001230DF1820B15BFE360E36000232B68C2
:10AFD000A361584660F0F6FB6080824630463DF043
:10AFE00077FB4FF00008C24502D809F10109B3E729
:10AFF000AAEB0802042A4FF0000328BF04220BEB3F
:10B0000008010548009303920FF062FC039A9044F4
:10B01000E9E701205EE700BF18500120E051012060
:10B02000E4510120DC50012000CA9A3BF8B5284BBE
:10B030001D68284B1B681A68012151641B68264A49
:10B04000D3F844650023146814B12179814230D0CB
:10B050000133082B02F10402F5D1F8BD6369A06940
:10B06000E289218AEB1A89B211FA82F2301AA18997
:10B07000B2FBF1F7C3EB034303444FF6FF7001FB50
:10B0800017228342A16828BF034621F81230238A81
:10B09000A2899BB2934203D2238A0133238214E014
:10B0A000E3899BB20133B3FBF2F102FB1133E3817D
:10B0B0000BE0E379002BD1D034F09AFE637900F0F5
:10B0C0000100834201D00023E3716561A661C4E7FA
:10B0D000F0660120A06801200C4701202DE9FF4106
:10B0E00004460F464EF066FC6368DB6853F8275051
:10B0F00040F2FF40294658F036F8064600285CD05A
:10B10000436828469847B36801A95B68804698471A
:10B11000B36800219B68054640469847B368002104
:10B120009B694046984763682849DB6853F82700C5
:10B1300057F053F9C0B190F85030B0F9382023F0EF
:10B14000100380F85030B0F93C309A421FBFADF880
:10B150000830C38F826BADF80A304FF000031ABF7E
:10B16000019201250025836263681949DB6853F861
:10B17000270057F032F9064668B190F82A3023F0DC
:10B18000020301A980F82A3017F002FF00210546CA
:10B19000304652F006FE6DB194F82A30DB070ED42B
:10B1A000019BA361029BE36194F82A3043F0010301
:10B1B00084F82A3004B0BDE8F0810546B3E704F115
:10B1C000180201A9104651F070FFEDE7B8C509005B
:10B1D0001CC609002DE9F74F404B01900020187064
:10B1E0003F4BDFF820A1DFF820C1FF2002EB8109EF
:10B1F00018703C493C48144615464FF001084FF082
:10B20000FF32A94520D1013204D0019B002B51D13E
:10B2100014F066FD354E364800220023C6E90023AF
:10B2200000231A46A5424BD15AB193ED017ADFEDC6
:10B23000317A67EE277A17EE900AFDF7B3FFC6E979
:10B24000000103B0BDE8F08F55F8047BBB07D8D1EF
:10B250003B685345D5D17B681A79A2F12003C2F12E
:10B26000200628FA06F608FA03F333433E7A08FA72
:10B2700002FEAEB1DCF804600096DCF8006046EA3D
:10B280000E0B009E1E43CCE900B67E7A002EB8D08D
:10B29000D1E9007647EA0E071E43C1E90076B0E720
:10B2A00046680096066846EA0E0B009E1E43C0E9FB
:10B2B00000B6EAE7104A00231360104A1370A9E7AA
:10B2C00021688F0708D10F68874205D112B10C4859
:10B2D00045F090FC0B4601220434A3E7446F0120A3
:10B2E0004C6F0120200D0120100D0120280D0120A0
:10B2F0009C8E090000007A4400670120F96E01204D
:10B300004A480900B88E0900000D0120242B2DE9C0
:10B31000F047884601D8012B06D1FDF73DFF1623E3
:10B3200003600020BDE8F087344E0D46294615F82D
:10B33000014B375D17F00807F8D12D2C10D12C7870
:10B3400001278D1C33F0100115D1302C0DD1297837
:10B3500001F0DF01582908D16C78023510230AE08A
:10B360002B2C04BF2C788D1CECE7002BF6D1302C55
:10B3700014BF0A23082307F1004E0EF1FF3E0021FF
:10B38000BEFBF3F90E4603FB19EAA4F1300CBCF145
:10B39000090F10D86446A3421EDDB1F1FF3F07D06C
:10B3A000B14516D301D1A24513DB06FB03460121AB
:10B3B00015F8014BE9E7A4F1410CBCF1190F01D8D4
:10B3C000373CE8E7A4F1610CBCF1190F04D8573CF5
:10B3D000E1E74FF0FF31EBE74B1C05D1222303607F
:10B3E000764632B930469DE707B17642002AF9D059
:10B3F00009B105F1FF38C2F80080F3E7197E0A00B1
:10B400002DE9F043344E86460D46284615F8014B8B
:10B41000375D17F00807F8D12D2C10D12C780127B3
:10B42000851C33F0100015D1302C0DD1287800F098
:10B43000DF00582808D16C78023510230AE02B2C45
:10B4400004BF2C78851CECE7002BF6D1302C14BF00
:10B450000A2308234FF0FF380026B8FBF3F803FB5C
:10B4600008F96FEA09093046A4F1300CBCF1090F64
:10B4700010D86446A3421EDDB6F1FF3F07D08045D9
:10B4800016D301D1A14513DB00FB0340012615F8BB
:10B49000014BE9E7A4F1410CBCF1190F01D8373C8D
:10B4A000E8E7A4F1610CBCF1190F04D8573CE1E7BF
:10B4B0004FF0FF36EBE7731C06D12223CEF80030A5
:10B4C000304632B9BDE8F08307B14042002AF9D0D6
:10B4D00006B1691E1160F5E7197E0A002DE9F74FE4
:10B4E00080460D46019260F062FAD8F80430AC4F05
:10B4F00001225A72D8F804301E791C68342303FBE9
:10B500000677002387F82E30EB6803F06043B3F131
:10B51000005F81468B4607D0A248D8F8043000224D
:10B520005A7203B0BDE8F08F9F4BC4F8083397F808
:10B530002F3003F0FF0A23B1BB689C48C4F80433E2
:10B54000EBE787F82F20AE46BEE80F0007F10C0CA2
:10B55000ACE80F00DEF80030CCF8003087F830A0FF
:10B560006B78C4F888354FF4827120465DF0E4F8BA
:10B570004FF4927120465DF0DFF8C4F850A5C4F88E
:10B5800040A52B78032B00F2B380DFE803F0729A1A
:10B5900052022B6903F06043B3F1005FBCD14FF45A
:10B5A0008073C4F800326B68EA68C4F844254FF42D
:10B5B000A871C4F8483520465DF0BEF84FF4B0716C
:10B5C00020465DF0B9F84FF4A47120465DF0B4F860
:10B5D00001232362A360D4F85031002BFBD04FF439
:10B5E000A87120465DF0A8F8AB682A69C4F8442524
:10B5F000C4F848356A4B342202FB06336C4A9A6021
:10B600004FF4827308226B4F2978654D03291CBFC4
:10B610000121A15034227243A918AA58002A79D0D6
:10B620008B68C4F80433634B9F4200F0A8806248E3
:10B6300073E76B68EA68C4F84425C4F848352B6999
:10B6400003F06042B2F1005F7FF466AFAA68C4F80D
:10B6500034354FF48453C4F83825C4F80032504BC5
:10B66000342202FB063340F202229A600123236255
:10B67000C6E701996B68EA68C4F84425C4F8483500
:10B680003422474B89B102FB06334FF48071C4F872
:10B690000012474A9A604FF4A47120465DF04CF8BE
:10B6A0004FF4A47301222262ACE702FB06334FF48D
:10B6B000007140F20222C4F800129A604FF48273C3
:10B6C000F0E76B68EA68C4F83425C4F838354FF4FD
:10B6D0008053C4F80032324B342202FB063340F26E
:10B6E00002229A600123236200224FF482738AE7C8
:10B6F000314F4FF48273082286E7D4F8242152B1E7
:10B700004FF4927120465DF017F8012323626361C4
:10B710004FF4827323441A68002AEED03422D4F8FE
:10B72000C434C4F8C43402FB0651002281F82F202F
:10B730008BB1224A224813F0010F08BF104613F0C4
:10B74000020F02F5803218BF104613F0040F1D4B94
:10B7500018BF1846E1E6204648F044FF00287FF471
:10B7600062AF1648D9E660F022F9814574EB010119
:10B7700009D2D8F80430144800225A72D1E619F5DB
:10B780007A794BF10004D8F804305A7A002AEAD1C9
:10B790009B7A042B96BF0D4A084852F82300C0E656
:10B7A000186201200A00AD0B02029C010B00AD0BD8
:10B7B000000204000000AD0B0400AD0B0100AD0B56
:10B7C0000000AE0B0200AE0B0700AD0B30220A00EA
:10B7D000F8B590F82A309B0704462DD4F8BDDB68F5
:10B7E00053F8256040F2FF40314657F0BCFC074655
:10B7F00068B1436830469847BB6804F108019B680C
:10B800009847013563689A689542E8D3E6E70B49A3
:10B81000304656F0E2FD20B104F1080152F01EFD61
:10B82000EFE70749304656F0D8FD0028E9D004F18B
:10B83000080152F0B6FAE4E70025E3E7B8C50900CD
:10B840001CC6090090F950301F4A10B5002B836ABE
:10B85000B4BF418A018AB0F90C40002B08BF1346DF
:10B860000C44997B8289B9B193F9051011FB02F15F
:10B870005A88114409B2A0F8461093F905205B8854
:10B8800012FB04331BB29942D2BFA0F84A30A0F891
:10B890004A10A0F8463010BD93F9041011FB02F1D4
:10B8A0001A88114409B2A0F8441093F904201B88A7
:10B8B00012FB04331BB29942D2BFA0F84830A0F863
:10B8C0004810A0F84430E6E7A205012090F9503076
:10B8D0001F4A10B5002B836AB4BF018A418AB0F9B0
:10B8E0000E40002B08BF13460C44997BC289B9B1A6
:10B8F00093F9041011FB02F11A88114409B2A0F85F
:10B90000441093F904201B8812FB04331BB29942A4
:10B91000D2BFA0F84830A0F84810A0F8443010BDBD
:10B9200093F9051011FB02F15A88114409B2A0F8ED
:10B93000461093F905205B8812FB04331BB2994231
:10B94000D2BFA0F84A30A0F84A10A0F84630E6E787
:10B95000A205012008B510EE103A23F00042B2F122
:10B960007E5FF0EE405A10D308D19FED2F0ADFED35
:10B970002F7A002BB8BFB0EE670A08BD70EE405AB0
:10B98000DFED297A87EEA50AF7E7B2F17C5F11D2E5
:10B99000B2F14A5F9FED266A42D920EE000AFCF719
:10B9A00041FEDFED247AE0EE657A75EEE75A36EE79
:10B9B000650AE2E7002BB7EE000AF6EE007A14DA29
:10B9C00075EE805A25EEA70AB1EEC06AFCF72AFE92
:10B9D000DFED197AE0EE067A9FED150A77EE867AAA
:10B9E00030EE670A30EE000AC7E730EE650A20EE57
:10B9F000270AB1EEC05AB0EE407A15EE103A6FF356
:10BA00000B0305EE903AA5EEE57A75EE257A87EE02
:10BA1000276AFCF707FEA0EE056A36EE250AE1E785
:10BA2000B0EE460AA9E700BF00000000DA0F494067
:10BA3000DA0FC93F6821A2336821A2B308B510EE1E
:10BA4000103A5A00F0EE407A0FD4B7EE007A70EE5A
:10BA5000477ABDE8084037EEA77AA7EEA77AB1EE9D
:10BA6000C70A37EE800A22F0CDB823F00043B3F1C5
:10BA70008B4F13D2FFEE006AE0EE006ABDE808408B
:10BA8000B1EEE67AF7EE006A37EE007A86EE870AC4
:10BA9000B0EE007A97EE870A22F060B922F05EF9E4
:10BAA000DFED027A30EE270A08BD00BF1872313F81
:10BAB00030B589B0084611461A4602AB0193194BBE
:10BAC0000093032355F0C5FD1749029D0C2057F044
:10BAD00025F99DF80C30037245609DF8103004463E
:10BAE000EBB128460EF060F8606805AA4FF49F613C
:10BAF00028F048FE237A5B0043F0010305AA0021E9
:10BB00000120079355F0EEFE57F054F805466068A3
:10BB10004EF0E9F81DB9217A044845F073F8204643
:10BB200009B030BD44240A00F4CC09007A49090068
:10BB300010B58EB003AB51F8044B0193194B009331
:10BB40000138032324F03AFA40F21C51606806AA37
:10BB500028F018FE237A5B0043F001030893039B4F
:10BB6000099340F626130A93049B5B0043F00103FC
:10BB70000B93059B6FF0004293421FBF40F2E642D9
:10BB80005B000C9243F0010314BF0221012106AABD
:10BB90004FF0020018BF0D9355F0A4FE0E200EB01A
:10BBA00010BD00BF2C240A0010B58EB003AB51F8B5
:10BBB000044B0193194B00930138032324F0FEF941
:10BBC00040F27961606806AA28F0DCFD237A5B0008
:10BBD00043F001030893039B099340F626130A934D
:10BBE000049B5B0043F001030B93059B6FF0004245
:10BBF00093421FBF40F2E6425B000C9243F0010308
:10BC000014BF0221012106AA4FF0020018BF0D93B4
:10BC100055F068FE0E200EB010BD00BF14240A00BF
:10BC200010B596B003AB51F8044B01932D4B009324
:10BC30000138062324F0C2F909AA606840F27A614B
:10BC400028F0A0FD237A5B0043F001030B93039BD4
:10BC50000C93049B0D9344F646430E93059B5B00A7
:10BC600043F001030F93069B6FF00042934235D0DF
:10BC70005B0043F0010344F616421193109209232E
:10BC8000032116AA02EB830244F2061042F8340C98
:10BC900016AA02EB8300079A520042F0010240F814
:10BCA000302C089A6FF00040824210D016A800EBAA
:10BCB000830044F2D60440F82C4C16A800EB830312
:10BCC000520042F00102013143F8282CC9B209AAFE
:10BCD000032055F007FE0E2016B010BD07230221E9
:10BCE000CFE700BFE4230A00F0B58BB00846114649
:10BCF0001A4603AB01931B4B0093072355F0A9FC95
:10BD0000DDE903600E2816D010F0030203D10168AC
:10BD1000154B99420CD02AF025F8C388009313489C
:10BD200040F28F134FF4917240F2FF2144F056FF1E
:10BD300001214EF073FA0E49182056F0EFFF9DF8DE
:10BD400020409DF824109DF81C50069F049A9DF8F1
:10BD500014300573C0E90167447381730261037590
:10BD60000BB0F0BDE4240A00F4C609006C510900D0
:10BD7000D8CC090030B58BB004466A464068244DE3
:10BD800040F2236128F0FEFC00216A46084655F087
:10BD9000A9FD56F00FFF002831D060686A4640F2D6
:10BDA0001F3128F0EFFC42F6D6330293A3685B0004
:10BDB00043F00103039344F6C6630493237B5B00C3
:10BDC00043F00103059344F6C6530693637B5B007F
:10BDD00043F00103079342F6C6421123CDE908233D
:10BDE00004216A46002055F07DFD23690E2B03D007
:10BDF000217D58684EF0FEF960680BB030BD04F04C
:10BE00000FFFAB6A002BBFD0012027F0D5FFBBE7A7
:10BE1000F46201202DE9F743054601F134000E4696
:10BE200004F0C2FE2B88102B05D0112B5FD0002010
:10BE300003B0BDE8F083404C002388224FF6FF7129
:10BE400002FB03F7E05B884205D00133052BF7D1F5
:10BE50004FF408770423882101FB03F0B5F804C0F0
:10BE600024F800C022180E20D065002082F85A0065
:10BE7000A2F87600EA7B01FB0343022A14BF96F87E
:10BE800045200122DA704FF000084FF6FF7207F1EB
:10BE90000800A3F8582041465022204483F87880B7
:10BEA00004EB070983F8798055F07AFA07F160000E
:10BEB0004A462044214909F051FCC6F818802869F7
:10BEC00069696C373C4403C468465EF0A5F9BDF867
:10BED00000302A8A9A4202D86A8A9A4203D2A888F3
:10BEE00069465EF081F90023F3600120A0E7AB888A
:10BEF000114F0024882202FB04F1785A984205D0A1
:10BF00000134052CF7D14FF40871042439440B484F
:10BF100009F03AFC88235C433A194FF6FF733B5310
:10BF2000002382F85A30D26D0E2A1EBF5360297A40
:10BF30001172B361D9E700BFA009012009FE030017
:10BF40002DE9F0418AB0084611461A4605AB019327
:10BF5000234B0093052355F07CFB0522059802A98D
:10BF600027F0B0FD039EA6F11002102A03D81D4B46
:10BF7000D340DB0702D41C4844F03CFE069C022C54
:10BF800004DC002C04DC194844F0D8FD062CFAD15E
:10BF90000798DDF80880A0B9074615494FF48A7064
:10BFA00056F0BCFE089B80F80C41C0F810313246B8
:10BFB0003B46414605464DF04EFF28460AB0BDE8D7
:10BFC000F081012202A927F07DFD0028E4D003982A
:10BFD00040F26512102124F095F8029FDDE700BFC2
:10BFE0008C240A00010101007B4A09002D47090049
:10BFF00094CC090070B588B003AB51F8045B019391
:10C00000184B00930138022323F0D8FF0522039830
:10C0100005A927F057FD069CA4F11002102A03D8A9
:10C02000114BD340DB0702D4104844F0E3FDDDE9B7
:10C03000040640B903462846224631464DF00BFF20
:10C040000E2008B070BD012205A927F03BFD002895
:10C05000F0D0069840F26512102124F053F8059BA9
:10C06000E9E700BF7C240A00010101007B4A0900C6
:10C0700010B50446084656F07EFA022804DC002873
:10C0800004DC044844F05AFD0628FAD184F80C0177
:10C090000E2010BD2D4709001FB503AB01930F4BB8
:10C0A0000093054601230E46002023F087FF31460A
:10C0B000284646F055FF03982AF00EFD441004D0A0
:10C0C000074840F2F44144F041FD29460120324640
:10C0D000FFF780F80348214660F08FFF78250A00BB
:10C0E0004A52090054250A0070B505460E4600283C
:10C0F00044D046F035FF324629460020FFF76AF863
:10C1000000F0A4F900231A4642F082F81C4B9C6A06
:10C1100094BB4DF0BFFE78B3FEF750FC012818D059
:10C1200002280BD1174A234656F82340A10702D113
:10C130002168914203D001339D42F5D10E2420465F
:10C140003CF0C8FE00F060F820463CF0C3FE2046FC
:10C1500070BD0D4B0D491A78234656F82340A007B1
:10C1600006D12068884203D1606800799042E6D009
:10C1700001339D42F1D1E1E70E24E3E70E24E6E727
:10C18000F46201209C8E09004C6F0120B88E0900DA
:10C1900010B586B0084611461A4602AB0193114B02
:10C1A0000093042355F055FA4FF49C61029861F016
:10C1B000FFF80D4904460C2056F0B0FD9DF8102004
:10C1C00012B10A4844F016FD22792F2A01D95DF0F8
:10C1D00032FA9DF814209DF80C10017244604272EE
:10C1E00006B010BD34250A00B88E0900D04D0900F4
:10C1F00010B5044C23781BB913F072FD0123237092
:10C2000010BD00BFF96E0120F8B5344C344A2368E4
:10C210006FF3172393421CD04FF4807200213148F2
:10C2200055F0BEF8304A00231370304A4FF44031C5
:10C2300013701A0102F180420133082BC2F804196D
:10C24000F7D14FF080434FF47C12C3F88429244B7C
:10C250002360274E274D0024D5E90001D6E900329E
:10C26000C4F1200703430A430120A4F1200100FA8E
:10C2700001F120FA07F73943A04003400A40134375
:10C2800008D0E0B23AF0BEF9204633F0C7FE2046AF
:10C2900033F0B2FF0134402CDED117491748002299
:10C2A0000023C6E90023C5E90023C1E900234FF4B8
:10C2B0000033C0F84833D0F80423920308D5C0F8FF
:10C2C0000833D0F844311BB14FF4A2715CF034FA5A
:10C2D0000B4B00200021C3E90001F8BD486F01208D
:10C2E000AF0000AD4D6F0120446F01204C6F012065
:10C2F000000D0120100D0120200D01200040024002
:10C30000280D0120F0B50E4687B000251446002AFE
:10C310005ED08A075FD10A68414B9A425BD16A4678
:10C320004FF4807057F05CF810B93E4844F006FCBA
:10C33000DDE90035042CA5EB030536D0A30732D187
:10C340002368394A934208D0384A934205D0384A84
:10C35000934202D0374A934225D1052203A92046B1
:10C3600027F0B0FB049BAB4202D0334844F042FCC0
:10C370009DF81410039C0022402023F063FF012845
:10C3800001D02E48F2E7009B5A19B2F5807F07D8FA
:10C390002B482A462146184454F0C1FF0E2417E0CA
:10C3A000284844F0F5FB2848C0E7284654F0C8FE6A
:10C3B000009B5A19B2F5807F044604D820492A46CA
:10C3C000194454F0ACFF214628462AF035FC0446B7
:10C3D000204607B0F0BD3246006800234FF480715C
:10C3E00027F08EFB042C064600F1010708D1B7F5B3
:10C3F000807F9CBF124B1D5C6D0045F00104E7E798
:10C40000204656F0B8F84223FF220021044655F09A
:10C4100053F9B7F5807FC3D8094B9C55BEE700BFE1
:10C42000885C0900E9370900FC650900385E0900ED
:10C43000585D090004620900DB460900654F0900E8
:10C440004D6F0120994409000B42090038B5084B93
:10C45000D3E9004554EA050305D05FF0A8FA201A95
:10C4600065EB010138BD4FF0FF300146FAE700BF30
:10C47000280D012010B52DED028B88B0084611461D
:10C480001A4603AB01932E4B0093022355F0E1F8BB
:10C49000DDE90304B0F10E0218BF0122B4F10E036E
:10C4A00018BF01239A4202D1264844F0A3FB0E286C
:10C4B00038D029F0CDFBB0EE408A5FF078FAFBF778
:10C4C00089F8DFED217A07EE100A0E2CC7EE278AD5
:10C4D00021D04FF46571049823F084FE04463AF0AD
:10C4E000FDFF05A93FF0A4F89DF81A3001939DF8CF
:10C4F000193000939DF817209DF818309DF81610FC
:10C50000BDF8140042F036FE231A08EE103AB8EED9
:10C51000C88A38EE288AB4EEE88AF1EE10FA04D51B
:10C520000A48C2E79FED0A8AC7E70A49082056F081
:10C53000F5FB80ED018A08B0BDEC028B10BD00BF99
:10C5400024250A007C46090000007A449B45090026
:10C55000000000009C8E09001FB5084611461A46CF
:10C5600003AB0193084B0093012355F072F84FF48D
:10C570009C61039860F01CFF0449082056F0CEFB34
:10C58000002044F0DBFA00BF1C250A00808E090061
:10C5900010B5094B094C1B6823B1A34202D00848CF
:10C5A00044F0F6FAC0220021064854F0F9FE054B8B
:10C5B00043F8044C181F10BD045601205C640900A8
:10C5C000694509000856012010B5084C20681EF086
:10C5D0007DFF014610B1064844F0DAFAB422201D6E
:10C5E00054F0DEFE034B2360204610BD480C0120B2
:10C5F000634509005C64090038B51C4608461146CD
:10C600004FF0021223F0A2FC20684FF49C6160F00E
:10C61000CFFE09490446082056F080FB63790546A1
:10C620000BB95DF008F8207933F080FB20790DF02C
:10C6300085F86C60284638BD10CC090008B5406804
:10C640004DF089F9BDE808409FED010A2AF0AEBB24
:10C650003333534070B5064640683C4D4DF07BF98E
:10C660003B4A002303212B80C2F8F0150121C2F8B8
:10C67000F435C2F8001519461A0102F1804202F59C
:10C68000E0420133082BC2F81415C2F81015F3D19B
:10C690002F4C4FF49053C4F81835736801265B791A
:10C6A000C4F814354FF48071C4F810352046C4F82E
:10C6B0002C56C4F830665CF03FF84FF48271204687
:10C6C0005CF03AF84FF4847120465CF035F84FF492
:10C6D000867120465CF030F84FF48A7120465CF099
:10C6E0002BF82660D4F80031002BFBD018484FF40B
:10C6F00080715CF021F801236360154CD4F804319B
:10C70000002BFBD012484FF482715CF015F8012326
:10C71000A360D4F81431002BFBD00D484FF48A717C
:10C720005CF00AF80023C4F80035C4F81435C4F8E6
:10C7300010352B881BB223EAE373181340EA8300F9
:10C7400080B2400040F0010070BD00BFCC68012005
:10C75000007000401C4608B5084611464FF0021212
:10C7600023F0F4FB4FF49C61206860F021FE044943
:10C77000042056F0D3FA0348F02144F0E7F900BF53
:10C78000F4CB09004A5209002DE9F04F2DED088B3A
:10C790008FB009AB01936D4B0093052323F00EFC82
:10C7A0000021099830F040FF002180460A9830F0BF
:10C7B0003BFF044600210B9830F036FFE379012B54
:10C7C00005460AD1C379012B07D1A268012A04D9F1
:10C7D0008368012B01D99A4202D05D4844F00AFADD
:10C7E0006621D8F808005BF08AFEE6692779059093
:10C7F000394630465BF012FEA368A069013B00FB9E
:10C8000003603946B0EE40AA5BF008FE0C98EE6972
:10C810000E28F0EE40AA28D1297930465BF0FEFDC3
:10C820000D980E28F0EE408A22D1A868AB692979CC
:10C83000013803FB00605BF0F1FDEB690493D8F86D
:10C840001C300293059BD4F81CB0DB690393B0EE57
:10C85000409A4FF00009D8F808304B450BD805989E
:10C860000FB0BDEC088BBDE8F08F29F0F1F9D7E7E8
:10C8700029F0EEF9E1E7029898F804105BF0CEFD9C
:10C88000029AD8F81830B4EEC0AA1A44F1EE10FAA1
:10C89000B0EE408A029252DCF4EEC0AAF1EE10FA39
:10C8A00050D4A668D4F818A02179013E0027F31BC4
:10C8B000012B32D80AFB07B006915BF0AFFD069959
:10C8C00006FB0AB0F0EE40BA5BF0A8FDAB69049A33
:10C8D0002979079103FB0720F0EE409A06935BF05D
:10C8E0009DFD049A069B079906FB0320B0EE40BA13
:10C8F0005BF094FD38EE6B8A30EE4B0A79EEEB9AE2
:10C9000028EE008A88EE290A30EE0B0A039BA3EC7E
:10C91000010A039309F101099DE707EB530303FBA8
:10C920000AB0079106935BF079FD069B0799B4EE78
:10C93000C80AF1EE10FAB4BF1F461E46B7E7B0EEC4
:10C94000680AE3E7B0EE490AE0E700BF386B0A0087
:10C950005D3B09002DE9F04F2DED048B87B003AB53
:10C960000193504B0093032323F028FB03980021ED
:10C9700030F05AFE8368012B044640F28C80C67961
:10C98000012E02D0484844F035F9007930F0D0FE4D
:10C9900081460498E5690E2857D0002130F044FE06
:10C9A000C779012F834603D1A26883689A4201D0D8
:10C9B0003E48E8E700799FED3E8A30F0B9FE8246B6
:10C9C0002846DBF81C80C847A3694046EE18F0EE05
:10C9D000408AD047DBF81830B0EE409A9844A568FA
:10C9E000BD4211D86B1E00EE103AF6EE007A28EE2A
:10C9F000278AB8EE400A20EE080A07B0BDEC048B87
:10CA0000BDE8F04F2AF0D2B93046C847A369404686
:10CA1000F0EE409A1E44D04778EEA98A30EE499A4B
:10CA2000F0EE486AD9EE286ADBF8183007EE907A03
:10CA3000B8EE677A9844C6EE877A0137B0EE409A2E
:10CA400038EE278AF0EE698AC9E705989FED188AC3
:10CA500029F0FEF82846B0EE409AC847A568F0EEE7
:10CA6000408AB54202D828EE098ABBE732462179CE
:10CA7000E0695BF09AFC07EE906A78EE808AB8EE87
:10CA8000677A78EEC88A0136C8EE877AF0EE408A77
:10CA900038EE278AE5E7074807B0BDEC048BBDE810
:10CAA000F08F00BF206B0A00B3340900BD340900C9
:10CAB00000000000020080801E280CD03E280AD012
:10CAC00010F0010307D1820707D10068044BC31A95
:10CAD000584258417047012070471846704700BFC0
:10CAE000C0320900F0B51B288DB006460C4615462D
:10CAF00072D03CD80E2800F09C8004D8042840F264
:10CB0000B580002430E01028FBD115F0010206D1D9
:10CB100015F00303F5D12968704A9142F1D12846F6
:10CB200055F029FD0122054609A9204600F024F907
:10CB3000102E0A9F3DD121790022402023F082FB54
:10CB4000A3686B4300FB03F1E06854F01AFBA36891
:10CB5000E0606B43A360636803F0FF0363601DB193
:10CB6000013DC319002F34D120460DB0F0BD1D2862
:10CB7000CBD02428C5D1012203A9284626F0A2FF44
:10CB8000002860D0A10712D12268554B9A420ED1DD
:10CB9000012209A9204600F0EFF801230093DDE906
:10CBA0000901DDE9032353F0F4F800285CD11E24C9
:10CBB000DAE7A1689DF82C00694300F035F9C368F5
:10CBC0000446CFE7184609993A4654F0A8FB013DC0
:10CBD000C319002DF6D1C7E70A68424B9A4290D09C
:10CBE00009A90122204600F0C7F806A90522284617
:10CBF00026F068FF9DF82C100022402023F022FB35
:10CC0000A168079DB5FBF0F5064629449DF82C0068
:10CC100000F00AF90446DDE90912C06854F07FFB10
:10CC2000E0680A9B069905FB06F2184454F077FB6E
:10CC30009AE70A682B4B9A423FF463AF2946204695
:10CC40004BF072FB90E7EA0702D5002043F076FF35
:10CC5000AB0703D12A68214B9A42F6D0284655F0FB
:10CC60009DFF0028A3D0F0E73E247DE7012209A91B
:10CC7000204600F081F8012206A9284626F022FF6E
:10CC8000002894D00B9A012A21D05A2A21DC203284
:10CC90000146089B012B1ED05A2B01DC2033014694
:10CCA0009342D2D123F00203642BCED0022E01D0C6
:10CCB0000029CAD0079B0093DDE90912069B304684
:10CCC00056F000FB002814BF3E241E244CE74222ED
:10CCD000DDE70021DDE74223E0E700BFC0320900C5
:10CCE000385E0900585D0900F0B5012885B0074697
:10CCF0000E4608D08B0727D10B681C4A934202D0FE
:10CD00001B4A934220D1012201A9304626F0DAFEC7
:10CD1000D0B139460022402023F094FA029BB3FBA5
:10CD2000F0F100FB01F5AB4202D0124843F062FF84
:10CD3000384600F079F8019904462A46C06854F054
:10CD4000EEFA204605B0F0BD304629F0D5FE58B1C8
:10CD500045102946384600F067F82B463A463146DA
:10CD600004464BF027FBECE70546F2E704620900B6
:10CD7000385E09001941090070B50D460179044675
:10CD800001F07F0116464020002223F05BFAE368A1
:10CD90002B60A26842436A60227902F07F02AA6097
:10CDA0002168094A91420BD194F90420002A01DB41
:10CDB000B20707D46268C2F3172200FB02332B606C
:10CDC000002070BD0120FCE7585D0900074BC1E958
:10CDD00000300023C1E90233054B02689A4202BFCA
:10CDE0004368C3F317238B60084670476C660900DD
:10CDF000585D090038B50D461C4611462846094ABB
:10CE000023F0A4F820682BF0ADF8012D007804D1B0
:10CE1000BDE83840002100F007B86168BDE838403F
:10CE2000FFF762BF040002007828F8B505460E46F9
:10CE300002D10F4843F0DEFE00220146402023F0DD
:10CE400001FA0C4B0C490746012D18BF194610205A
:10CE500055F064FF0571436803F0FF030446C0E921
:10CE6000013606FB07F054F089F9E0602046F8BD72
:10CE700085410900FC650900385E090070B50A7932
:10CE8000012A05460C460DD1184956F050F9D4E94F
:10CE9000022128462CF034FE28461549BDE8704092
:10CEA00056F045B9134956F051F9A368002BF3D059
:10CEB0001149284656F03BF90026A368B34204D82E
:10CEC0000E49284656F033F9E6E71EB10C492846CC
:10CED00056F02DF93246E168207923F08BFA0122D1
:10CEE000014628462AF0BEF90136E6E7BCE1080013
:10CEF00035220900C8E10800D3E10800322009000A
:10CF00006C2309002DE9F04F044687B00D46164604
:10CF10000AB90025D0E011F003078068DFF82CA2E1
:10CF200040F0DF800B68814A934240F0DA806A4625
:10CF300056F056FA10B97E4843F000FE2179042ECF
:10CF400001F07F013A464FF0400000F0968023F058
:10CF500079F916F00302054655D131688B7B002B19
:10CF600042D001EB83031869724B98423CD131796E
:10CF7000402001F07F0123F065F9A84202D06E48FD
:10CF800043F038FE33685345D6E9028B38D17368D5
:10CF9000C3F3172905FB09F9DDE900062368E768F3
:10CFA000361A5345A8EB06062FD194F90430002B0E
:10CFB000AFDA002EE3D16368C3F3172305FB0377D1
:10CFC00005FB08F20BEB090105FB007054F0D2F9E8
:10CFD0000199A268009B521A08EB03006A4305FB03
:10CFE000017105FB007039E0544B99420BD1012DC2
:10CFF000C5D1052203A9304626F064FDDDE903B85A
:10D000004FF00009C8E74E4896E7002ED8DD636868
:10D01000B6EB132F2FD9A16831446943384654F039
:10D02000B0F86368E06066F31F2382466360BB4527
:10D0300008BF83460098A268019940443244121AFE
:10D040006A4301FB05A105FB00A054F093F9009889
:10D0500005FB08F20BEB090100FB05A054F08AF96F
:10D060006368C6EB132262F31F236360A368334433
:10D07000A3600E2520E0BA46DCE723F0E3F8216840
:10D08000009B514506461BD1B3F1807F03DB2D4940
:10D090002D485FF0B2FF102055F040FE054694E8A1
:10D0A0000F0085E80F00009A02EB112363F31F21A4
:10D0B0006960019B9B1AAB60284607B0BDE8F08F02
:10D0C00001992079C91AFFF7AFFEDDE90032E16866
:10D0D000D21A0546724306FB0311C06854F01FF9CB
:10D0E000EAE700232A460146206826F009FD236866
:10D0F0005345024620790ED16368042E02EB1322B9
:10D100000BD003067FF505AFE168334600F07F00E2
:10D1100023F068FCADE7042EF6D1E16800F07F0053
:10D1200007B0BDE8F04F23F065B900BF885C090087
:10D13000E937090005CF0200743A090004620900CA
:10D140000B420900C83909005C580900585D090004
:10D1500010EE102A08B522F00043B3F17E5FB0EE66
:10D16000406A12D319BF76EE467A9FED1F7ADFED43
:10D170001F7A9FED1F7A12BF87EE276AE0EE077ACB
:10D18000B0EE676AB0EE460A08BDB3F17C5F0BD221
:10D19000A3F50003B3F1645FF4D320EE000AFBF7BC
:10D1A00041FAA0EE066AEDE7B0EEC06AB7EE000AFB
:10D1B00030EE460AF6EE007A20EE270AB1EEC06A9B
:10D1C000FBF730FA002ADFED0B7AA0EE066AB0EE2C
:10D1D000007AE6EE077A9FED066A36EE676AB8BF18
:10D1E000B1EE466ACEE700BF0000000000008003F9
:10D1F000DA0FC93F6821A2B31FB58DED010A019B6B
:10D2000023F00042B2F18B4F00EE102A4FEAD370A8
:10D210000AD320F0A3FDDFED1E7A30EE270A08B115
:10D22000B1EE400A05B000BD5B0014D5B7EE007A40
:10D23000F0EE476AE0EE006AF1EEE67A77EE807A89
:10D24000C7EE276AF0EE007AE0EE276AB0EE660AD3
:10D2500020F084FDE3E7B2F1665F10D320EE007AA0
:10D26000F7EE006A37EE266AF1EEC67A77EEA67A16
:10D27000C7EE276A36EE800A20F0C4FCCFE7DFED68
:10D28000057A70EE277ACDED037A039BC7E700BFDE
:10D290001872313F0000807B08B5044B1A68044BBC
:10D2A0009A4202D00D2039F097F908BD009C032066
:10D2B000EF2978011FB5044690B10E2810D00079EF
:10D2C0004DF03EFA60B94FF4F773039301A920467D
:10D2D00003AB02AA1BF0B0F90399024843F092FC99
:10D2E00004B010BD0C520900F4EE400AF1EE10FA41
:10D2F00010B5F0EE407A04D770EE207AB0EE670AEF
:10D3000010BD10EE902AB2F17E5F03D1BDE810404F
:10D3100000F082B810EE103A940F04F0020444EAD0
:10D32000D37433F0004308D1022C59D09FED317AE9
:10D33000032C08BFF0EE477AE0E732F0004209D153
:10D34000DFED2D7A9FED2D7A14F0010F08BFF0EE7E
:10D35000477AD3E7B2F1FF4F10D1B3F1FF4F04F199
:10D36000FF3407D1022C3ED8254B03EB8403D3EDC9
:10D37000007AC3E7022C39D8224BF6E702F150615C
:10D380009942DDD3B3F1FF4FDAD0A10703D503F102
:10D39000506393420CD387EEA00AB0EEC00A00F0AF
:10D3A0003BF8012CF0EE407A04D1F1EE407AA5E78B
:10D3B000DFED157A022C0AD0002C9FD09FED137A56
:10D3C00077EE877A9FED127A77EEC77A96E79FED30
:10D3D0000F7A77EE877A9FED0E7A77EE677A8DE790
:10D3E000DFED0B7A8AE7DFED0B7A87E7DFED067A70
:10D3F00084E700BFDB0F49C0DB0FC9BFDB0FC93FAC
:10D40000D8650A00CC650A00000000002EBDBB33C1
:10D41000DB0F4940DB0F493F10EE102A22F000439A
:10D42000B3F1994F82B04FEAD2700ED3B4EE400AF6
:10D43000F1EE10FA07D69FED410ADFED417A0028A0
:10D4400018BFB0EE670A02B070473E498B420BD856
:10D45000B3F1665F5AD212F0FF4FF4D160EE007A5A
:10D46000CDED017A019BEEE7374A9342F0EEC07AA8
:10D4700037D8A2F5D002934229D8F0EE006ABFEE69
:10D48000007AA7EEA67A002377EEA67A87EE270A1F
:10D490005A1C60EE006A9FED2D6ADFED2D7ADFEDFC
:10D4A0002D5A26EEA67AE7EE067A9FED2B6AA7EEB6
:10D4B000876ADFED2A7AE7EE257A67EE877AE6EE6D
:10D4C000267A67EE807A24D130EE670ABBE7B7EEA2
:10D4D000007A77EEC76A77EE877A012386EEA70A8D
:10D4E000D6E71F4A93420BD8F7EE086AB7EE007AE8
:10D4F000A7EEA67A022337EEE66A86EE070AC7E7AA
:10D50000BFEE007A87EE270A0323C1E74FF0FF330F
:10D51000BEE7144A144902EB830201EB830393ED47
:10D52000007A77EEC77A37EEC00AD2ED007A37EE8E
:10D53000C00A002887D0B1EE400A84E7DA0FC93F5D
:10D54000DA0FC9BFFFFFDF3EFFFF973F25AC7C3DF1
:10D550000DF5113E4712DABDA9AAAA3E98CA4CBEE3
:10D56000FFFF1B40F4650A00E4650A002DE9F84F4F
:10D57000D1F800800128064640468CBF01F1040B1B
:10D580004FF0000B0F46914629F0E6F930B94046BE
:10D5900028F0E8FBC188274843F020FB06F1FF3A5A
:10D5A000B9F1000F2DD0D9F80050C5F3DC051AEB06
:10D5B000050404D02C44A00053F0C2FD0446002210
:10D5C000924520D804EB86000022954221D11A4EC4
:10D5D000DFF868903168D9F800000131090153F093
:10D5E000D0FD3368C9F800005A1C32601A0100EB04
:10D5F000031340F802A0C3E90158DC603868BDE8B5
:10D60000F88F4D46D3E75BF8223044F822300132E0
:10D61000D6E7D9F80830083053F8323040F80C3CDF
:10D62000D9F8083003EBC20301325B6840F8083CCC
:10D63000CBE700BFD650090000510120F85001206F
:10D64000F0B50023DFF838E00C4E19460E27DEF85F
:10D650000020934201D30E20F0BD346804EB031286
:10D660004FEA031C9568854208BF44F80C1003F18B
:10D67000010304BFC2E90117D160E8E7F8500120B7
:10D680000051012038B590F82330FF2B044629D0F3
:10D69000154B01225A600022C3F8002590F826306D
:10D6A0009B0707D590F8210032F040FB94F8220048
:10D6B00032F03CFBFF2594F8210038F0A3FF94F8EA
:10D6C000220084F8215038F09DFF94F8230084F85C
:10D6D000225038F097FF054B84F8235000221A603F
:10D6E0003EF090FD0E2038BD00500240185F012032
:10D6F0002DE9F04788B0084611461A4602AB01935F
:10D70000434B0093062353F0A4FF9DF81C7002982E
:10D7100040F2C5210FB345F001FC40F26D610546B2
:10D72000039845F0FBFB40F23A31044604985FF061
:10D730003FFE40F25F41824605985FF041FE354969
:10D740008046282055F0F1FA0646B8F1000F0DD0BA
:10D75000314840F25F4143F0F9F95FF029FE40F2B1
:10D760006D61054603985FF023FEDCE72B4BD3F891
:10D770000080B8F1000F02D0294843F009FA186080
:10D7800028799DF818900BF0D9FF20790BF0D6FF7F
:10D790009AF804000BF0D2FF96F8263067F34103A5
:10D7A00086F826301F4B2A7986F82120C3F8642595
:10D7B000227986F82220C3F868259AF8042086F892
:10D7C0002320C3F8702507B32879414632F0BEFA0A
:10D7D0002079414632F0BAFA0122124B0121C3F8F6
:10D7E00004254F400022C3F80825C3F80C15C3F8E0
:10D7F0001075C3F81C15C3F82025C3F824953EF016
:10D800001BFD304608B0BDE8F0873A46E5E700BFAB
:10D8100030260A00C4CB09004A520900185F0120D3
:10D82000C04C09000050024010B5044690F8230097
:10D830004CF08BF80A4AD2F8083143B194F82630FC
:10D8400023F0040384F826300023C2F8083194F84A
:10D85000263013F0040F0CBF1E203E2010BD00BF69
:10D860000050024010B5044690F823004CF06DF8CB
:10D870000C4AD2F8083143B194F8263023F004035F
:10D8800084F826300023C2F8083194F826305A076D
:10D8900001D400F009F843F0200384F826300E206C
:10D8A00010BD00BF0050024008B5014843F070F9B8
:10D8B000CB4809002DE9F04F0D4685B055F8044BD3
:10D8C000064694F8230017464CF03FF802AB01934C
:10D8D0006D4B00933A4602232946701E22F06EFBE0
:10D8E0006A4A029DD2F808319DF80C6043B194F861
:10D8F000263023F0040384F826300023C2F80831D0
:10D9000094F8263059070BD5604A0123536094F8E8
:10D91000263043F0080384F826302023C2F8083369
:10D92000294640F2FD402BF047FC94F82630656014
:10D9300066F3861384F826302A7B6968534FD20831
:10D9400084F82520AB7BE87B6D7B84F82450003B7A
:10D9500018BF0123DB0143EA0023E08C013A03F402
:10D96000C07320F4C07018BF01220343E384C7F8DA
:10D970001C2594F824305A1E53425341C7F82835C9
:10D9800094F8263013F002033DD00B4694F825009E
:10D99000638394F824304843584300014FF47A736A
:10D9A000B0FBF3F0033020F0030080B2208353F08B
:10D9B000E5FBA060208B53F0E1FBE06060684AF07B
:10D9C000EDFF0023C4E9043384F8203094F82630B6
:10D9D00023F03C0343F00403204684F826301CF077
:10D9E000B3FB228B294B9208C3F850252022C3F8A1
:10D9F00004230122C3F800251A601CF087FB0E20C7
:10DA000005B0BDE8F08F2248DFF88C90B7EE007AC1
:10DA10009E4698461E46D7F81C25012A01D18279D8
:10DA20003AB307EE901A1B4AD0F800B0B0F904C020
:10DA300099FBFCFCF8EE676A02F1580A55689CFBFA
:10DA4000F5F507EE905AF8EEE77A76EEE77AF0EE23
:10DA5000E77A87EEA66AB4EEC76AF1EE10FA05D54A
:10DA6000D2F800E0B0EE467A2B46D846083292450E
:10DA7000E4D10136092E00F10800CCD1034AC2F8E6
:10DA80001885C2F814E581E720260A0000500240FC
:10DA9000D8250A0080250A000048E80110B5044690
:10DAA00090F823004BF051FF064A0123536094F88D
:10DAB000263043F0080384F826302023C2F80833C8
:10DAC0000E2010BD0050024038B5084B1B680022E4
:10DAD0000446C3F80025FF25007938F093FD6079EE
:10DAE000257138F08FFD65710E2038BD440201208C
:10DAF0002DE9F0432DED028B8BB0084611461A46F6
:10DB000003AB01933E4B0093072353F0A2FD40F279
:10DB1000063103985FF04CFC40F23D310746049813
:10DB20005FF046FC9DF818506A07064604D040F2A4
:10DB3000C621344843F066F89DF820305B0702D0D8
:10DB400040F2C941F5E70998DDF814809DF81C9072
:10DB500010B328F07DF8B0EE408A40F2D252012195
:10DB60000020B0EE480A53F089FD2749082055F0FF
:10DB7000DCF8044638790BF0E1FD30790BF0DEFD7E
:10DB800084F806903A79227133796371B8F57A5F37
:10DB900005D01E4843F02EF89FED1D8ADDE7102DBD
:10DBA00001D01C48F6E71C4BDFED1C7A1B681C49B2
:10DBB000C3F840256279C3F8442528EE278A4FF040
:10DBC0000462C3F804250022C3F82025FCEEC87ABD
:10DBD0002822C3F81825C3F81C250122C3F8002504
:10DBE00017EE900AC3F86015C3F864251A6026F092
:10DBF00025F820460BB0BDEC028BBDE8F08300BFDA
:10DC000060260A0079510900A8CB0900FE370900F7
:10DC1000AE47E13D153809004402012000007A4476
:10DC2000C85601202DE9FF411446074600790D46EC
:10DC30004BF085FE4FF48961204622F0D3FA4FF471
:10DC400089620021044653F043FDAB0706D12A68E0
:10DC50002D4B9A4202D12D4842F070FF062201A9B5
:10DC6000284625F02FFF9DF80C10029D0022402031
:10DC700022F0E8FAB5FBF0F5A54202D2244842F0C2
:10DC8000B9FF039B482B01D02248F8E7DFF89080CA
:10DC9000019DD8F800300122C3F80825C3F860556B
:10DCA000C3F864451C4B4FF4485043F001039847B8
:10DCB000D8F800300022C3F80821184AC3F86025BC
:10DCC00001222E46C3F86425D8F80030D3F8083175
:10DCD0006BB105EB4405B5420CD1BB7983B124F09F
:10DCE0000104640044F0010004B0BDE8F08102F0DA
:10DCF00097FFE9E73388A3F5004326F8023BEAE7FC
:10DD000024F00304EDE700BF2C180A00094E0900B7
:10DD1000D64C0900973E0900C0260A00C8560120CB
:10DD20004402012070B58AB0084611461A4606AB77
:10DD30000193264B0093042353F08BFC0698052295
:10DD400003A925F0BFFE059C622C0ED0682C0FD0D5
:10DD5000482C1FD0422C01D1002507E0012C1BD0FC
:10DD60001B4840F2E52142F04DFF0125012401E06E
:10DD7000012502249DF8243083B9079B049A63434C
:10DD80005B00B2FBF3F103FB11223AB1114840F200
:10DD9000E521E8E70025ECE70025EBE70E49182030
:10DDA00054F0BCFFE4009DF824309DF81C10089A44
:10DDB000039E0473049CC37300230661857384600F
:10DDC0004173426003750AB070BD00BF98260A0017
:10DDD000915109003E4A090088CB09002DE9F04124
:10DDE0001C460D4692B011462846824A22F0AEF8F3
:10DDF0002668814B3340062B05D0B10710D132681D
:10DE00007E4B9A4208D145F2761231467C4853F057
:10DE10005FFD8207064603D132687A4B9A4202D0F0
:10DE2000794842F0D3FE012D14D9062208A9606872
:10DE300025F048FE40F2E5230998089F4FF48062E0
:10DE4000082122F07FF94307054605D06F480821D5
:10DE500042F0D8FE00252F466D49402054F05EFF69
:10DE6000044606630022002306F1080050F07BFC04
:10DE7000206B10226B460DEB0201083050F0A4FF1E
:10DE800010B1052042F06EFE009B102B0BD16149B2
:10DE9000042204A853F02FFA28B95F49082206A8E3
:10DEA00053F029FA18B140F2AF3022F079F8206B24
:10DEB00004226B460DEB0201083050F085FF00286C
:10DEC000DFD1009B042B02D1019A282A02D95348A2
:10DED00042F090FE206B6B4608A9083050F074FFAA
:10DEE0000028CED1019A282A03D0BDF82030012B7A
:10DEF0000CD1BDF82210022908D8BDF82E30102B05
:10DF000004D8122A04D1BDF830208AB14448DFE792
:10DF1000282A0DD1BDF820004FF6FE729042F5D1AF
:10DF2000BDF83820012AF1D1BDF832209A42EDD156
:10DF3000082B099A237394BF00230123A3734FF482
:10DF40000073A360002362606173E373206B6B4610
:10DF5000042202A9083050F037FF002891D1009E1A
:10DF6000042E8ED12F49324602A853F0C4F98046C0
:10DF7000206B6B46324603A9083050F025FF00287D
:10DF80007FF47FAF009B042B7FF47BAF206B039A61
:10DF9000B8F1000F0AD0D0E91013521843F1000372
:10DFA000083050F0E0FB0028D0D06AE72262036C12
:10DFB000A38465B94FF48070E06253F0DFF8034644
:10DFC0002061E06A63B9A561657342F07DFD6D086B
:10DFD00027612F44E562A761204612B0BDE8F081B9
:10DFE00053F0CCF8A0610028F6D1E06A2561657392
:10DFF000EBE700BF040002000F0080FF343109008E
:10E000000C5B09002C180A00BF3D0900E04E090016
:10E0100068CB0900372209003C2209009C4A09000C
:10E02000794B09002EFF08002DE9F04F2DED028BF2
:10E0300095B004460C920993426A002943D00C9B88
:10E04000012B00D1826A209BA1691960216A237F7C
:10E05000914240F04284D4E90421002B18BF1146BC
:10E06000099B07911960237F83F001032377A3693C
:10E070009B080B9304F130030E9300230D9306933A
:10E0800094F82C300D9A93421FDC069B3BB9079AFB
:10E090000B99069B02EB8101914240F0FD83A37B2B
:10E0A000002B00F0FD83236A013323620C9B002BBD
:10E0B00040F01B84636A01336362012015B0BDEC3C
:10E0C000028BBDE8F08F0C91BDE70E9B53F8045F07
:10E0D0000E93AB680A93002B40F0D0830D9B013365
:10E0E0000D93CDE7AB60069B002B00F0CE830123A0
:10E0F0000693F3E76B699B086B61431E58425841D6
:10E1000068730A98637B407BD5F810B06A699842BF
:10E110004FEA032140F0B180914228BF1146089A8E
:10E12000D4ED017A8A4294BF05920591F8EE677AA0
:10E13000F7EE000A80EEA77A059AB2FBF3F3A74A3E
:10E1400005F1180007EE903AF8EEE77AA44B9FED40
:10E15000A50A67EE877A27EE287AC3ED007AA24BEC
:10E1600083ED007A1378013313705DF0F4FCDFED7A
:10E170009F0AB0EE408A05F11C009FED9D0A5DF0FC
:10E1800006FDDFED9C7A627B28EE278A022ABCEE30
:10E19000C88A18EE103A9BB2029374D110F4004F63
:10E1A00047F6FF73029909BF1B1AC0189BB24FF4C0
:10E1B00000401CBF80B24FF400434B434843C1139F
:10E1C000DB13039102932B6A11936B6A12930698E7
:10E1D0000A9B217B5B7B00261396002840F08D81F3
:10E1E000102940F00981A17B002900F084809A4227
:10E1F0007FD0DDF810A0DDF81880059B434565D978
:10E200005BF81890039B01931FFA89F0029B00931F
:10E2100040EA094012AB11AA13A94AF011F9119E64
:10E22000360436FB00F6129F3F0437FB10F726F347
:10E23000CF3627F3CF37C6EA07464AF8086B4FEACE
:10E240001940039E01960004029E009640EA194080
:10E250004AF0F6F8119B1B0433FB00F3129A1204E8
:10E2600032FB10F223F3CF3322F3CF32C3EA02435F
:10E270004AF8043C08F10208BFE752008A4228BF6E
:10E280000A4608994CE7029B03939CE7039B5BF8C3
:10E2900026000193029B009311AA12AB13A94AF026
:10E2A000CFF8119B1B0433FB00F3129A120432FBCC
:10E2B00010F223F3CF3322F3CF32C3EA0243049A9E
:10E2C00042F826300136059BB342DFD1059A089B00
:10E2D000607B9B1A0893049B03EB820304930A9BC5
:10E2E0005B7B9842D5E9041200F09B82059B5B089A
:10E2F00098E2069EE7E79A426BD0DDE904A35B084B
:10E300000BEB8303D9460F934FF0802B0F9B4B45AC
:10E31000DCD059F8043B93FA4BF8039B01931FFAA6
:10E3200088F0029B009340EA084012AB11AA13A99F
:10E330004AF086F8119E360436FB00F6129F3F0421
:10E3400037FB10F726F3CF3627F3CF37C6EA074659
:10E350004AF8086B4FEA1840039E01960004029E9B
:10E36000009640EA18404AF06BF8119B1B0433FBFF
:10E3700000F3129A120432FB10F223F3CF3322F38C
:10E38000CF32C3EA02434AF8043CBFE75BF82600F9
:10E3900090FA47F0039B0193029B009311AA12ABE2
:10E3A00013A94AF04DF8119B1B0433FB00F3129A9A
:10E3B000120432FB10F223F3CF3322F3CF32C3EA3D
:10E3C0000243049A42F826300136059BB342DDD160
:10E3D0007CE7069E4FF08027F7E700BF126F012011
:10E3E00084680120000000008068012000FE7F3F5B
:10E3F00000FE7FBF000000479A42059B4FEA430999
:10E400002BD1069E4FF080274E45BFF45FAF3BF8FF
:10E4100016005EF013FEA37B0BB990FA47F0039B46
:10E420000193029B009311AA12AB13A94AF008F8BA
:10E43000119B1B0433FB00F3129A120432FB10F2FF
:10E4400023F3CF3322F3CF32C3EA02405AF006FB64
:10E45000049B23F816000136D6E7069F4FF080286C
:10E460007B1C4B45BFF432AF3BF807005EF0E6FD86
:10E47000A37B06460BB990FA48F6039B0193B0B212
:10E48000029B009340EA064012AB11AA13A949F07F
:10E49000D7FF119B1B0433FB00FC129B1B0433FBB7
:10E4A00010F32CF3CF3C23F3CF33CCEA03405AF0E4
:10E4B000D5FA049B23F81700039B0193300C029BB1
:10E4C0000093000412AB40EA164049F0B9FF119BDB
:10E4D0001B0433FB00F3129A120432FB10F223F3F5
:10E4E000CF3322F3CF32C3EA02405AF0B7FA049B8B
:10E4F000023323F817000237B2E7102940F0F88002
:10E50000A17B002975D09A424CD0DDE90483D9461D
:10E510004FEA530B09EB8B0BD9453FF4D7AE59F8B3
:10E5200004AB039B01931FFA8AF0029B009340EA1D
:10E530000A4012AB11AA13A949F082FF119E3604BA
:10E5400036FB00F6129F3F0437FB10F726F3CF3659
:10E5500027F3CF37C6EA074658F8080B96FA10F6A5
:10E5600048F8086C4FEA1A40039E01960004029E88
:10E57000009640EA1A4049F063FF119B1B0433FBED
:10E5800000F3129A120432FB10F223F3CF3322F37A
:10E59000CF32C3EA024358F8042C93FA12F348F836
:10E5A000043CB9E7049B1F1F059B0BEB8308D84570
:10E5B0003FF48CAE039B5BF8040B0193029B00932A
:10E5C00011AA12AB13A949F03BFF119B1B0433FBAB
:10E5D00000F3129A120432FB10F223F3CF3322F32A
:10E5E000CF32C3EA024357F8042F93FA12F33B6089
:10E5F000DDE79A4251D0DDE904935B080BEB83031E
:10E60000DA460F934FF0802B0F9B9A453FF45EAE96
:10E610005AF8043B93FA4BF8039B01931FFA88F0D6
:10E62000029B009340EA084012AB11AA13A949F0DB
:10E6300007FF119E360436FB00F6129F3F0437FB9E
:10E6400010F726F3CF3627F3CF37C6EA074659F837
:10E65000080B96FA10F649F8086C4FEA1840039E2A
:10E6600001960004029E009640EA184049F0E8FE38
:10E67000119B1B0433FB00F3129A120432FB10F2BD
:10E6800023F3CF3322F3CF32C3EA024359F8042CE9
:10E6900093FA12F349F8043CB6E7049B1F1F059B4D
:10E6A0004FF080290BEB8308C3453FF40FAE5BF8B6
:10E6B000040B90FA49F0039B0193029B009311AA6B
:10E6C00012AB13A949F0BCFE119B1B0433FB00F3F2
:10E6D000129A120432FB10F223F3CF3322F3CF321B
:10E6E000C3EA024357F8042F93FA12F33B60DBE7C7
:10E6F00005999A424FEA410A40F08E80049B4FF000
:10E7000080289F1E5645BFF4E1AD3BF816005EF031
:10E7100095FCA37B0BB990FA48F0039B0193029BF5
:10E72000009311AA12AB13A949F08AFE119B1B0496
:10E7300033FB00F3129A120432FB10F223F3CF33AF
:10E7400022F3CF32C3EA024237F8020F5EF076FCC2
:10E7500092FA10F05AF082F901363880D2E73BF88D
:10E7600006005EF06BFCA37B07460BB990FA49F7F5
:10E77000039B0193B8B2029B009340EA074012AB9F
:10E7800011AA13A949F05CFE119B1B0433FB00FE88
:10E79000129B4FEA034C3CFB10FC2EF3CF332CF3BF
:10E7A000CF3CC3EA0C430F93049B33F816005EF092
:10E7B00045FC0F9B93FA10F05AF050F9049B23F894
:10E7C0001600039B0193380C029B0093000412ABCC
:10E7D00040EA174049F034FE119B1B0433FB00F361
:10E7E000129A120432FB10F223F3CF3322F3CF320A
:10E7F000C3EA0242049B33F818005EF01FFC92FA51
:10E8000010F05AF02BF9049B023623F8180008F197
:10E810000208C245A3D859E54FF001084FF08029FE
:10E82000F7E7059B01EB8301D21AC5E90412029BAD
:10E830002B62039B6B62089B002B3FF458AC6B6907
:10E84000002B7FF45EAC6B7B33B92B7B002B3FF44A
:10E8500049ACA8684AF0A2F8A86800283FF451AC77
:10E8600005F1140205F110014AF04DF802287FF479
:10E8700041AC0023AB606B616B7334E40B9B08937A
:10E88000079BDFED228A0493D5E7089B069904983D
:10E890009A0052F085FD2AE442F8043BFFF7FCBBE6
:10E8A000237B0B9A102B079B03EB82020AD04FF0BD
:10E8B00080309A423FF4F7AB196881FA40F143F88F
:10E8C000041BF6E74FF080209A423FF4ECAB196846
:10E8D00091FA40F143F8041BF6E723B92369099A3A
:10E8E0001360FFF7E3BB6369F9E70C9B012B7FF42F
:10E8F000E4ABA36A227B0133A362099B1B6803EB91
:10E90000D203099A1360FFF7D8BB00BFDB0FC940E1
:10E910002DE9F04788B0084611461A4602AB01932C
:10E92000364B0093062352F094FE40F25D63FF22C3
:10E930000121029852F0C0FE40F2FB23064602225B
:10E940000498012152F0B8FE079D002D804604DC9A
:10E9500040F27151012021F0C3FBDDF814A0BAF19F
:10E96000080F05D0BAF1100F02D0254842F042F945
:10E9700006F10D002349800054F0D0F9039F9DF863
:10E9800018900446F8088000A06152F0F7FB034697
:10E990002061A0691BB96373636142F095F852F07E
:10E9A000EDFB606118B960732061A069F5E76560EF
:10E9B0000025A76084F80CA084F80E9084F80D80E0
:10E9C000E57384F82C6004F13007B5420ADB94F853
:10E9D0002C0004F1340128F075FB2063204608B0B8
:10E9E000BDE8F087002308481A46194600F068F889
:10E9F000013547F8040F4460E7E700BFFC270A0031
:10EA00006841090048CB0900E0270A00F0B50C4630
:10EA100087B054F8045B0646687B174649F06EFFE2
:10EA200003AB0193114B00933A4603232146701E1A
:10EA300021F0C4FA95F82C209DF810309A4203D8A2
:10EA400040F25C6021F0ACFA05EB8303039E5C6B43
:10EA50009DF814706068314602F026F82046A660E2
:10EA600027734BF031FA284607B0F0BDC8270A00DB
:10EA7000F0B50D4685B055F8044B0646607B174649
:10EA800049F03CFF03AB01930C4B00933A46012342
:10EA90002946701E21F092FA94F82C209DF80C3033
:10EAA0009A4203D840F25C6021F07AFA04EB8304C6
:10EAB0000022636B0E209A6005B0F0BDC0270A00EB
:10EAC00010B508461146002221F040FA0B492820D3
:10EAD00054F024F900230446836000F1180140F249
:10EAE000494207483EF03AFB064840F2D24204F160
:10EAF0001C013EF033FB204610BD00BFE0270A009A
:10EB0000020000C0020080807FB502AB51F8044BC8
:10EB100001930A4B00930138022321F04FFA029D22
:10EB200060689DF80C60294601F0BEFF2046A56094
:10EB300026734BF0C9F90E2004B070BDB0270A004F
:10EB40001FB503AB0193064B51F8044B00930138FA
:10EB5000012321F033FA00230E20A36004B010BD7E
:10EB6000A8270A002DE9F04FAFB0446A04901CB901
:10EB7000389B1C60022021E00029049989681491C7
:10EB80003899149C0C60049991F9541008BF002224
:10EB90008A42049915D1049891F9551000EB81012E
:10EBA000496B01EB42021A60FF2380F85430389B16
:10EBB0001A68836D03EB5203836501202FB0BDE813
:10EBC000F08F91F84410049CB1FA81F1490984F85E
:10EBD000441084F85510C2F1010204EB810184F85D
:10EBE00054204A6B1A60069252F06FFC0498002180
:10EBF00052F046FC049B044670B99A680146069898
:10EC000052F0CEFB389B1C60049B93F8450080F0CB
:10EC100001004000C0B2D1E7049ADB6A126BD21A3D
:10EC20000992049A12690392002A01F01685049A47
:10EC30000398576A1F44394647F0F6F8421C0646C7
:10EC400001F00F85039BD3F80090B9F1000F00F09D
:10EC50003D81D3F80480B8F1000F00F0378199F8B6
:10EC600000B099F81C303C18BBF1000F3ED1032BCB
:10EC70004FF0090114BF4FF0200A4FF0110A2AA8E3
:10EC8000CDE92A4BCDE92CBA5FF025F9C8F8000090
:10EC900099F81C30032B14BF032105212AA85FF02B
:10ECA0001AF9454645F8040F039BD3F8BC379B453A
:10ECB0000DDB4FF0000B039BD3F8C4379B4580F26C
:10ECC000C880902303FB0B850023059392E005F198
:10ECD000100301212AA805935FF0FDF8059B45F874
:10ECE000040F9D42F5D10BF1010BDDE7032B4FF033
:10ECF000080114BF4FF0110A4FF0090A00232AA897
:10ED0000CDE92B332A94CDF8B4A05FF0E4F8C8F82D
:10ED1000000099F81C30032B14BF022101212AA8FE
:10ED20005FF0D9F8C8F80400C3E70C212AA85FF007
:10ED3000D2F80921A8622AA85FF0CDF80821E8627C
:10ED40002AA85FF0C8F8286399F80030002B14BF98
:10ED5000092104212AA85FF0BEF8012168632AA8CE
:10ED60005FF0B9F8A863002856D002212AA85FF006
:10ED7000B2F80121E8632AA85FF0ADF80521286404
:10ED80002AA85FF0A8F8052168642AA85FF0A3F814
:10ED90000023EB64A86403212AA85FF09CF80321F8
:10EDA00028652AA85FF097F8032168652AA85FF014
:10EDB00092F8EB6BA86533BBC5E90A336B63E86D6A
:10EDC000C0F11400286699F80030002B3FD10121D2
:10EDD0002AA85FF080F8686601212AA85FF07BF816
:10EDE0000121A8662AA85FF076F8059BE866013342
:10EDF00005934835039B059AD3F8BC379A4294DBB8
:10EE00000BF1010B57E7022B04D12B6C13B908232C
:10EE1000EB65D4E70723FBE7C5E90F0005212AA826
:10EE20005FF059F8052168642AA85FF054F80521BD
:10EE3000A8642AA85FF04FF80421E8642AA85FF0CC
:10EE40004AF80321E8652AA85FF045F8BAE70020F0
:10EE5000C1E7039A0999D8F80080C2F8D88706EB71
:10EE60000A028A1A03990992D1F8B817039A04EB97
:10EE70000A05D2F8B02700295AD0002A40F0A48011
:10EE8000039BD3F8CC27099B934280F2AE8006996E
:10EE9000039847F02CFF4FF0FF34149A0698002196
:10EEA00052F07EFA049B93F845300BB903341BD81B
:10EEB000049B06989A68002152F072FA389A00234F
:10EEC0001360049A012382F8453053E606990398AB
:10EED00047F00DFF6FF00604049B099A1B6B9B1A09
:10EEE000049AD362002CD8D1049B149A9B6D03EB37
:10EEF0005203049A9365104652F0E7FA04980021F1
:10EF000052F0BEFA049B049A1B6BD26A9A1A049BB5
:10EF10009B6A9B1AB3F5007F044607DD049AAE4B4B
:10EF200002F11400C2E9053201F03EFE204645E63A
:10EF3000002A49D10399DDF824B00122C1F8B02795
:10EF4000A94659464846059347F0E5FE431C059BF4
:10EF500018D019F800C039788C4509EB00021DD192
:10EF600092F801C079788C4518D197F802C0917851
:10EF70008CEA0101032911D81CF0020F18BF02F11D
:10EF8000FF32501B039A0028C2F8B4070CDA069926
:10EF9000104647F0ACFE6FF002049DE7033002F12B
:10EFA0000309ABEB000BCCE7039A0644D2F8C02769
:10EFB00056445643039AD2F8C8275343039AF6009F
:10EFC00096FBF3F3C2F8B837039BD3F8B4271B685A
:10EFD00043B15B69003B18BF01231344039AC2F895
:10EFE000CC374DE74FF0FF33F7E7039B0399D3F896
:10EFF000DC37434501F11C003DDBA3EB0801424631
:10F0000041180A9052F0B6F9039BD3F8D807D3F809
:10F01000CC270A9B2946184452F081F9039B039997
:10F02000D3F8CC27D3F8D8371344C1F8DC37DB004A
:10F030001093039B099903F2DC738A1A1A93002335
:10F0400009920C930593039B059AD3F8C4379A420F
:10F0500081F21E837C2353431193902353431993CE
:10F06000119B013B1F93119B08931A9B189300233C
:10F070000D939B46FEE32946184452F050F9039B3A
:10F080000399D3F8CC27D3F8DC3703981344C1F89D
:10F09000DC37099B06999B1A09936FF0010447F02E
:10F0A00026FE19E7039B1E68002E00F0D4805B68E3
:10F0B0000793002B00F0CF80039B9D68002D00F08C
:10F0C000CA800A9B22930023CDE923330C9A109B1C
:10F0D0009A18D31D48BF02F10E03DB1025930C9B39
:10F0E0001BB1194622A85EF0F6FE059B31789022EE
:10F0F0005A43482303FB0B22079B1A44536BD2F855
:10F100003CC0002940F04E81344810F8136000EBF9
:10F110004300BCF1020F477862D1D2F84090B9F1B8
:10F12000000F10D0089B884605EB0309314622A842
:10F130005EF0D1FE08F10108B8F1080F09F8010BE3
:10F14000F4D14FF00309119B05EB03080D9B984484
:10F1500009EB49039844314622A85EF0BCFE3146D3
:10F1600088F8170022A85EF0B6FE314688F818002D
:10F1700022A85EF0B0FE09F10109B9F1060F88F886
:10F18000190008F10308E6D1089BEE18394622A8B9
:10F190005EF0A1FE394686F8290022A85EF09BFEAB
:10F1A000394686F82A0022A85EF095FE09F1010989
:10F1B000B9F10C0F86F82B0006F10306E6D1059A8B
:10F1C0007C2353433E2202FB0B332B44002283F863
:10F1D0003B209A8724E000BFE9FE040058640A003F
:10F1E000059B002B3ED10D9BDDF8148005EB030938
:10F1F000314622A85EF06FFE08F10108B8F10B0F4E
:10F2000009F8010BF4D10D9B1D44394622A85EF08C
:10F2100062FE05F8080008F10108B8F1150FF4D1F5
:10F22000059B189A90265E434820079B00FB0B66BF
:10F2300033449B6A5360229B0A9A9B1A249AC2EB1E
:10F24000C302D71007D4189B53F804CF1893109B10
:10F25000634580F2ED810699039847F048FD6FF011
:10F26000070439E64FEA0B13079A083302EB030948
:10F2700052F80380B8F1000F1FD00D9B8846EB18A1
:10F280001F9913F8012B5A5408F10108B8F1060F21
:10F29000F6D1D9F80430FBB9089B4FF0060805EB0E
:10F2A000030A314622A85EF016FE0AF8080008F1AB
:10F2B0000108B8F10B0FF4D121E0089B05EB030A1C
:10F2C000314622A85EF007FE08F10108B8F1060FEA
:10F2D0000AF8010BF4D1DCE7059C3E2303FB0BF39A
:10F2E0007C20EA1800FB04332B4491799971D17981
:10F2F000D971117A1972517A5972927A9A72D9F82F
:10F3000008306BB9089B0B2605EB0308394622A889
:10F310005EF0E1FD08F806000136102EF6D112E08D
:10F32000059C3E2303FB0BF37C20EA1800FB04330F
:10F330002B44D17AD972117B1973517B5973917B0C
:10F340009973D27BDA73D9F80C306BB9089B10260D
:10F3500005EB0308394622A85EF0BDFD08F806005B
:10F360000136152EF6D112E0059C3E2303FB0BF36C
:10F370007C20EA1800FB04332B44117C1974517C67
:10F380005974917C9974D17CD974127D1A75059A3F
:10F390007C2353433E2202FB0B332B4400225A753D
:10F3A0009A753DE7366A16F0010603D0BBF1010FEE
:10F3B00000F0B280B3F5C87F7BDA1911052291FB0A
:10F3C000F2F2269202EB8202891AC3F3810228929A
:10F3D00003F0030300222791299311461346BCF141
:10F3E000020F40F0CE80059C902060434827079C88
:10F3F00007FB0B002044006C002808BF4FF0010CF5
:10F4000001EB41018948614410F821702A9700EB13
:10F41000810148782B908878C9782C902D910EB373
:10F42000BBF1010F1ED10DF1980C05F1FC070DF198
:10F43000A80E664603CE764538607960B44607F17B
:10F440000807F6D10DF1A80C05F58677664603CEC0
:10F4500079602EA98E423860B44607F10807F5D1CD
:10F46000C5F8F820059990224A43482101FB0B2258
:10F4700007990A445366D36B022B40F0C580176C82
:10F48000002F00F0A880089B0026EF18269922A8DC
:10F490005EF021FD0136062E07F8010BF6D14FF084
:10F4A00001080327119B05EB030A0D9B0AEB0304DC
:10F4B0008BE0B3F5FA7F12DAA3F5C8739910052231
:10F4C000B1FBF2F2269202EB8202891A03F00303E7
:10F4D0000022279128932992134601217FE7A3F563
:10F4E000FA730321B3FBF1F101EB41020598269178
:10F4F0009B1A0022CDE9282290224243482000FB9B
:10F500000B22079827930244126C0AB1CDE9271306
:10F5100000220123022162E7B3F5B47F03F0010268
:10F520004FEA630110DA242091FBF0F3269300FBED
:10F530001313062093FBF0F100FB113328930023F3
:10F540002791299303214AE7F3290CDCB4390B11E5
:10F550002693C1F38103279301F00301002328912F
:10F56000299304213BE7F4390323B1FBF3F32693FA
:10F5700003EB4303C91A00232791CDE92833052162
:10F580002DE74FF0000C3BE726AB22A853F828A04C
:10F5900051465EF0A0FC5146F07522A85EF09BFC3F
:10F5A0005146307622A85EF096FC033609F1010937
:10F5B000B0752AAB53F828209145E5DB08F1010826
:10F5C000B8F1040F3FF4FBAD4F4407EB4706264468
:10F5D0004FF00009EDE7B84664E753F8261022A87B
:10F5E0005EF079FC09F8010B013726AB5AF82620AA
:10F5F0009742F2DB0136042E0DD0B84404EB080923
:10F6000000270DF1A80AF1E7089B4FF00008EC185D
:10F61000464626ABF2E7059A7C2353433E2202FB83
:10F620000B331D440023AB756B75F9E578640A0054
:10F63000039B1D68002D00F0C2815B680B93002BBB
:10F6400000F0BD81039B9B68002B00F0B881039BF9
:10F65000D968002900F0B38102F0070313930C9BD3
:10F66000139AC3EBC70313441C93BCEB0303079328
:10F6700000F1A5810A9B6A6B3B441D930B9B1E44C2
:10F68000B36B002B00F02381F36B022B40F01F8142
:10F69000336C002B40F00381059C9023634300FBF7
:10F6A0000B330B9803440320DB6D013393FBF0F322
:10F6B00002EB4303B3F92E0000EB40004FF410724D
:10F6C000059C9023634348250B9C05FB0B33234487
:10F6D000DB6A5B00B3F5107FA8BF4FF41073934251
:10F6E000D4BF2C932C920A932D938342D4BF2B9397
:10F6F0002B9001EB8B03209303F580530A9AC3F8F8
:10F7000000224FF4106303FB0B131593139B0F930D
:10F710001D9B0C93002316930E93199B4033E31803
:10F7200021930E9B169F01332AAA0E9352F8233081
:10F730001693A3EB070EBEF1000F23DD159B0E9A67
:10F740000C9903EB8707219B53F82250B14B03EB35
:10F75000C5031E790F9B5A4202F0070213462AB1D5
:10F7600011F8010BC2F1200200FA02F2002E40F063
:10F77000C08033463A1D47F8263042F8263002361C
:10F78000B645F8DC00230F9A0C991A4401EBE2010C
:10F7900002F007020F92079A0C91D31A07930E9B5F
:10F7A000032BBED1109B1C9A9B1A0E93079B002B18
:10F7B00000F09F82159B0A9A0C9803EB8205059A2C
:10F7C00090235343482202FB0B330B9AD318924ADF
:10F7D000DB6E52F823200B92904A52F823100F9BB5
:10F7E0005B4203F007031A462BB110F8016BC3F11B
:10F7F000200306FA03F3079CA61A0A9C4FF000099F
:10F80000C4F50F7AC1F120014F460AF1010A0A91AD
:10F81000BA4500F3F081209B03F58052D2F8003204
:10F820003B44C2F800320022B3F5107FC0F263827D
:10F83000079A0F9B13440C9A02EBE30203F00703B1
:10F840000C93089B0A923E3308930D9B3E330D9315
:10F85000199B4833199313461D9A9B1A00F1AF80E8
:10F86000139AC2EBC3030C9A13440E9AD31A109343
:10F870000BF1010B039BD3F8BC379B45FFF612AC91
:10F880000599039844F0E4FE013040F0578506994D
:10F89000039847F02CFA6FF00904FFF71DBB2B7893
:10F8A0005BB9059C9023634300FB0B330B98034427
:10F8B000DB6D013332F9130000E7B2F93600B2F91B
:10F8C0003430C31AB2F90C0000EB4300F6E6059B96
:10F8D00090255D43482303FB0B550B9B1D44EB6DAB
:10F8E0002D6E013332F913002B44013332F913200A
:10F8F000E6E64B4850F825C04A4800EB4C0017900C
:10F900000798012EA0EB030040F08E80454C34F8A0
:10F910001C6006F00F064FF000094FF0004AC6F1D8
:10F9200020060F2853DD8C46C3F118081CF8025B33
:10F93000497805FA08F5C3F1100801FA08F10D43FA
:10F940002A431033103861460A2BEADD22FA06F505
:10F95000179C013534F815504FEA153C15F0F00F9F
:10F9600002FA0CF218BF02F0004CA3EB1533C5F3FA
:10F9700003181EBF520003F1FF334CEA080815F4C8
:10F98000706FC5F3032C1FBF03F1FF3302F0004576
:10F9900045EA0C0C52004B4511DB47F8088BAEF1E1
:10F9A000020EBEF1000F47F804CCCDDCA3EB090337
:10F9B000079A0344D31A079A93427FF6E4AE069956
:10F9C000039847F094F96FF00804FFF785BA1D1803
:10F9D000002DF4DD002812DD082891F800C0C8BF12
:10F9E0004878C3F118080CFA08FCC8BFC3F110032B
:10F9F00042EA0C02C9BF98400131024302316B1E3A
:10FA00004AFA03F31A404FF00B0905F10B030020EB
:10FA10009AE700BF54410A0050640A0048640A0093
:10FA200078630A0054420A00A6F1020CBCF1010FEF
:10FA3000C5D8DFF8F0C25CF83580DDF85CC0002482
:10FA4000129408F101041B94C8F120041E940F289D
:10FA500027DD8946C3F1180A19F8025B497805FACF
:10FA60000AF5C3F1100A01FA0AF10D432A431033D3
:10FA7000103849460A2BEADDBCF8009009F00F095E
:10FA8000C9F1200522FA05F501353CF815505FEA69
:10FA9000153A2AD1A3EB090302FA09F20CEB450C43
:10FAA000E8E7C518002D8ADD002812DD082891F846
:10FAB0000090C8BF4878C3F1180A09FA0AF9C8BF0C
:10FAC000C3F1100342EA0902C9BF98400131024361
:10FAD00002314FF000406B1E40FA03F30B201A4036
:10FAE000129005F10B030020C4E7C5F30319B9F127
:10FAF0000F0FA3EB0A0302FA0AF2C5F3032523D181
:10FB0000032E24D11B9C03EB000C002D0CBFA2463E
:10FB100004F1010AE2453FF752AF9C46E24552DC50
:10FB20000344B3EB0C0006D5581E9C464FF000432F
:10FB300003411A4000201E9B22FA03F909F10F0924
:10FB4000ACEB080302FA08F2B9F1000F05D002F09D
:10FB5000004C49EA0C095200013B0F2D1DD1032E28
:10FB60001CD11B9C1D18AC423FF729AF9C461B9C27
:10FB7000644533DC0344B3EB0C0006D5581E9C46A9
:10FB80004FF0004303411A4000201E9B22FA03F568
:10FB90000F35ACEB080302FA08F22DB102F0004C6D
:10FBA00045EA0C055200013B129CA342FFF607AF49
:10FBB000AEF1020EBEF1000FC7E9009518DDDDF8C9
:10FBC0005CC0083756E711F8019BCCF1180409FA1C
:10FBD00004F942EA09020CF1080C9FE711F8015BF5
:10FBE000CCF1180A05FA0AF52A430CF1080CBEE715
:10FBF000129A9B1ADCE60F2E56DD8446C2F1180ECF
:10FC00001CF8021B407801FA0EF1C2F1100E00FA46
:10FC10000EF001430B431032103E60465745BFF6CD
:10FC2000F7AD092A7FF7F4AD0A990B9C23FA01F18D
:10FC300021443B4C615C4FEA111C03FA0CF311F0B8
:10FC40000808A2EB11121FBF03F0004802F1FF32B7
:10FC50005B0048F0010811F0040E1FBF03F0004ED6
:10FC600002F1FF325B004EF0010E11F0020C1FBFDB
:10FC700003F0004C02F1FF325B004CF0010C11F07C
:10FC800001011FBF03F0004102F1FF3241F0010109
:10FC90005B004A45FFF6BFAD45F8108B043745E9D8
:10FCA00003EC45F8041CB9E7B11800297FF7B3ADA0
:10FCB000002E12DD082E90F800C0C8BF4678C2F1B1
:10FCC000180E0CFA0EFCC8BFC2F1100243EA0C0376
:10FCD000C9BF96400130334302304A1E4FF0004402
:10FCE00044FA02F213404FF00A0901F10A02002619
:10FCF00094E7079F8FE5159941F82320013393E599
:10FD0000059903982A4645F063FC01300CD1069909
:10FD1000039846F0ECFF6FF00A04FFF7DDB800BF70
:10FD2000F8630A0054410A000135039BD3F8BC373D
:10FD30009D42E5DB039AD268002A00F08684039A8C
:10FD400052690B92002A00F08084039A926907920C
:10FD5000002A00F07A84039AD2F8C867059A5643BD
:10FD6000069A5E43022B02EB460640F0E9820B9BAB
:10FD70001193331D089300230E93079B03F5005343
:10FD80000D930E9B0D9A0799119803F001030F93A1
:10FD90000B9B03F580554FF00077D5F8183B009387
:10FDA000D2F800220F9B45F0F3F8D5F81C3B0D9AD2
:10FDB000079911980093D2F800220F9B803100F52B
:10FDC000106045F0E5F80F9B0D9A5B42D2F80022D7
:10FDD00003F488631344079A02EB830B4FF0000C83
:10FDE00052F82320DBF85C306046C2FB007C6FF0E9
:10FDF0007301C3FB017C4FF00076DBF88020DBF859
:10FE0000DC300546C2FB0065C3FB01654FF4557944
:10FE1000DBF80430DBF85820C3FB097C834BC2FBC2
:10FE2000037CDBF88410DBF8D820C1FB0965C2FB3A
:10FE3000036541F6D478DBF80830DBF85420C3FBC7
:10FE4000087C7B4BC2FB037CDBF88810DBF8D420FA
:10FE5000C1FB0865C2FB036546F2B86EDBF80C30E7
:10FE6000DBF85020C3FB0E7C724BC2FB037CDBF83B
:10FE70008C10DBF8D020C1FB0E65C2FB03656E4A17
:10FE8000DBF81030DBF84C10C3FB027C6B4BC1FB82
:10FE9000037CDBF89000DBF8CC10C0FB0265C1FBF3
:10FEA0000365DBF81420DBF84830C2FB0E7C45F21A
:10FEB0008401C3FB017CDBF89420DBF8C830C2FB73
:10FEC0000E65C3FB0165DBF81820DBF84430C2FB8C
:10FED000087C40F22C71C3FB017CDBF89820DBF836
:10FEE000C430C2FB0865C3FB0165DBF81C20DBF8EE
:10FEF0004030C2FB097C7421C3FB017CDBF89C20F1
:10FF0000DBF8C030C2FB0965C3FB01650C24384631
:10FF10004FF014080CFA04F34CFA08FC20FA08F02D
:10FF200040EA030046F0D6FB089B23F8040C304659
:10FF300005FA04F345FA08F520FA08F040EA030050
:10FF400046F0C8FB089B0BF5805723F8020C3B6872
:10FF50004FF4D0704FF000724FF0000CC3FB002C38
:10FF60004FF00073D7F880100026C1FB003641F631
:10FF70007C007968C1FB002CD7F88410C1FB0036E7
:10FF800049F2FC70B968C1FB002CD7F88810C1FB9E
:10FF900000362B49F868C0FB012CD7F88C00C0FB59
:10FFA000013628493D69C5FB012CD7F89050C5FBA7
:10FFB00001366FF0B3057969C1FB052CD7F89410B1
:10FFC000C1FB05364FF41275B969C1FB052CD7F892
:10FFD0009810C1FB05366FF0130EF969C1FB0E2CAA
:10FFE000D7F89C101D46C1FB0E5610460CFA04F3C0
:10FFF0004CFA08FC20FA08F040EA030046F06AFBDD
:020000023000CC
:10000000089B9887284606FA04F346FA08F620FA71
:1000100008F040EA030046F05DFB089B0A49D887D8
:1000200004331293089B043B13930FE0D4F8FFFFB3
:100030007CAFFFFF3CB6FDFF78940400C44902008A
:100040004CE803002464FFFF343D0A00D1F840E08F
:10005000DBF80051DBF85C014FF000730022C5FBB8
:100060000E324FF000764C6C4FF00009C5FB04696E
:10007000C4F1000CC0FB0C32C0FB0E69DBF8DC01E4
:10008000DBF8804115904FF000774FF0000AC4FB79
:100090000E7A4FF00075486C4FF00008C4FB005812
:1000A0001598C0FB0C7AC0FB0E58D1F848E0DBF87D
:1000B00004C1DBF85801CCFB0E32CC6CCCFB0469DC
:1000C000C4F1000CC0FB0C32C0FB0E69DBF8D80198
:1000D000DBF884411590C4FB0E7AC86CC4FB005851
:1000E0001598C0FB0C7AC0FB0E58D1F850E0DBF835
:1000F00008C1DBF85401CCFB0E324C6DCCFB04691B
:10010000C4F1000CC0FB0C32C0FB0E69DBF8D4015B
:10011000DBF888411590C4FB0E7A486DC4FB00588B
:100120001598C0FB0C7AC0FB0E58D1F858E0DBF8EC
:100130000CC1DBF85001CCFB0E32CC6DCCFB04695A
:10014000C4F1000CC0FB0C32C0FB0E69DBF8D0011F
:10015000DBF88C411590C4FB0E7AC86DC4FB0058C7
:100160001598C0FB0C7AC0FB0E58D1F860E0DBF8A4
:1001700010C1DBF84C01CCFB0E324C6ECCFB046999
:10018000C4F1000CC0FB0C32C0FB0E69DBF8CC01E3
:10019000DBF890411590C4FB0E7A486EC4FB005802
:1001A0001598C0FB0C7AC0FB0E58D1F868E0DBF85C
:1001B00014C1DBF84801CCFB0E32CC6ECCFB0469D9
:1001C000C4F1000CC0FB0C32C0FB0E69DBF8C801A7
:1001D000DBF894411590C4FB0E7AC86EC4FB00583E
:1001E0001598C0FB0C7AC0FB0E58D1F870E0DBF814
:1001F00018C1DBF84401CCFB0E324C6FCCFB046918
:10020000C4F1000CC0FB0C32C0FB0E69DBF8C4016A
:10021000DBF898411590C4FB0E7A486FC4FB005878
:100220001598C0FB0C7AC0FB0E58D1F878E0DBF8CB
:100230001CC1DBF84001CCFB0E32CC6FCCFB046957
:10024000C4F1000CC0FB0C32C0FB0E69DBF8C0012E
:10025000DBF89C411590C4FB0E7AC86F1691C4FB65
:1002600000581599C1FB0C7AC1FB0E580C24184696
:10027000142102FA04F342FA01F220FA01F040EAF2
:10028000030046F027FA129B23F8040C3846142783
:100290000AFA04F34AFA07FA20FA07F040EA0300E0
:1002A00046F018FA129B23F8020C304609FA04F3C0
:1002B00049FA07F920FA07F040EA030046F00AFA83
:1002C000139BA3F87C00284608FA04F348FA07F8C1
:1002D00020FA07F040EA030046F0FCF9139B169958
:1002E000A3F87E00129B04331293139B043B1393D9
:1002F000DE4B40318B420BF5807B7FF4A7AE0D9B2C
:100300000F9AD3F800329B1A0D9A03F00703C2F834
:1003100000320E9B01330E93119B80331193089B87
:10032000803308930E9B122B7FF42BAD059B01337A
:1003300005931A9B08331A93FEF785BE0025F4E453
:10034000079B4036002703F5005807F001030E9382
:100350000B9B0B98079903F5805300EBC710D3F85C
:10036000183B0093D8F8002207F0010344F010FE78
:1003700007F00103D8F800225B4203F488631344BA
:10038000079A02EB8309002052F82310D9F85C2069
:100390004FF000730446C1FB04306FF07301C2FBE1
:1003A00001304FF4557ED9F80420D9F85810C2FB1B
:1003B0000E30AF4AC1FB023041F6D47CD9F8082098
:1003C000D9F85410C2FB0C30AA4AC1FB023046F2E5
:1003D000B865D9F80C20D9F85010C2FB0530A64AF0
:1003E000C1FB0230A54AD9F81010C1FB0230A44A63
:1003F000D9F84C10C1FB0230D9F81410D9F84820B4
:10040000C1FB053045F28401C2FB0130D9F8181058
:10041000D9F84420C1FB0C3040F22C71C2FB0130F2
:10042000D9F81C10D9F84020C1FB0E307421C2FB52
:1004300001300C2402464FF0140A184602FA04F365
:1004400042FA0AF220FA0AF040EA030046F042F9C2
:1004500009F5805126F8400C0A684FF0007000231F
:100460004FF4D075C2FB050341F67C054A68C2FB18
:10047000050349F2FC758A68C2FB0503814DCA6811
:10048000C2FB0503804A0D69C5FB02036FF0B3058B
:100490004A69C2FB05034FF412758A69C2FB050362
:1004A000CA696FF01301C2FB010303FA04F243FAB5
:1004B0000AF320FA0AF040EA020046F00BF9DFF8EE
:1004C000CCA126F8200CA6F140030D930896DAE99A
:1004D00010ECD9F80021D9F85C114FF0007000231E
:1004E000C2FB0E034FF000754FF0000BC2FB0C5B1C
:1004F000CCF10002C1FB0203C1FB0E5BDAE912EC96
:10050000D9F80411D9F85821C1FB0E03C1FB0C5BCB
:10051000CCF10001C2FB0103C2FB0E5BDAE914EC73
:10052000D9F80811D9F85421C1FB0E03C1FB0C5BAB
:10053000CCF10001C2FB0103C2FB0E5BDAE916EC51
:10054000D9F80C11D9F85021C1FB0E03C1FB0C5B8B
:10055000CCF10001C2FB0103C2FB0E5BDAE918EC2F
:10056000D9F81011D9F84C21C1FB0E03C1FB0C5B6B
:10057000CCF10001C2FB0103C2FB0E5BDAE91AEC0D
:10058000D9F81411D9F84821C1FB0E03C1FB0C5B4B
:10059000CCF10001C2FB0103C2FB0E5BDAE91CECEB
:1005A000D9F81811D9F84421C1FB0E03C1FB0C5B2B
:1005B000CCF10001C2FB0103C2FB0E5BDAE91EECC9
:1005C000D9F81C11D9F84021C1FB0E03C1FB0C5B0B
:1005D000CCF10001C2FB0103C2FB0E5B0C24142111
:1005E00003FA04F243FA01F320FA01F040EA0200B0
:1005F00046F070F80D9B23F8020F14210D93284646
:100600000BFA04F34BFA01FB20FA01F040EA030075
:1006100046F060F8089B23F8020D0893134B0AF18B
:10062000400A9A4509F580797FF451AFD8F8003235
:100630000E9A01379B1A03F00703122FC8F80032F5
:1006400006F140067FF481AE70E60699039846F005
:100650004EFB6FF00B04FEF73FBC6FF00404FEF797
:100660003BBC6FF00504FEF737BC00BFF4400A0046
:10067000D4F8FFFF7CAFFFFF3CB6FDFF7894040089
:10068000C44902004CE803002464FFFF343D0A0023
:100690000024FEF721BC00BF2DE9FF411C460D469A
:1006A00028461146424A1FF051FC2768414B3B4007
:1006B000062B05D0BA070AD13A683F4B9A4206D1B9
:1006C00039463E4845F2761251F002F907460121BB
:1006D000384623F049FA067C16F0010602D0384865
:1006E00040F074FA012D2BD96068062201A923F08D
:1006F000E9F9DDE9015633495C2052F016FBEB07BE
:1007000004461FD50135013EB6F5305F1CD905F50D
:1007100090536563A6F5105605F51055A363656201
:10072000A6620023C4E90B335DF063FB206100285F
:1007300035D1204649F0DDFB234924485CF05DFCBF
:100740003546D8E7002DDFD14FF40068C4F8288083
:10075000404650F013FD606228B9204649F0C9FBBD
:10076000404640F0B1F9B6F5105F04D3656305F576
:100770009055A563D5E74FF4905050F0FFFC6063AF
:1007800028B9204649F0B5FB4FF49050E9E74FF403
:10079000905050F0F3FCA0630028C2D1F1E720464E
:1007A000394609F021FB204604B0BDE8F08100BFC6
:1007B000040002000F0080FF343109000C5B0900C7
:1007C000BF3D090028CB0900364D0900B8300900AB
:1007D00010B50446407B48F091F8A3689FED107A6D
:1007E0005A0800EE102A94F8442004EB820423F007
:1007F0000103626B13449A4209D1F1EEC77ABDE856
:100800001040B8EEC00A87EE800A26F0CFBA32F95F
:10081000021B07EE901AF8EEE77AA7EEA77AEAE74E
:100820000000000038B504460D46407B48F066F8ED
:1008300045F276122946044851F04AF8014620460E
:1008400009F0D2FA0E2038BD0C5B090038B50D4610
:100850000446407B48F052F80121284623F084F9F1
:10086000037CDB0702D5044840F0B0F92046294656
:1008700009F0BAFA0E2038BDBF3D0900F0B587B0C7
:10088000084611461A4603AB0193274B00930323F6
:1008900050F0DFFE40F2454103985CF089FD4FF4D3
:1008A000AA61074604985CF08BFD20490646242087
:1008B00052F03BFABDF814501D49044600220B6863
:1008C000D3F80005C0070AD50132042A01F104015A
:1008D000F5D10023A36033B9164840F059F9164901
:1008E0008A5C2277F6E70022C3F80C25A368012270
:1008F000C3F81025A2683B792376C2F860353879B1
:1009000008F01CFF3EB1A26833796376C2F86835FF
:10091000307908F013FFA3682D0A01222046A58232
:10092000C3F8002507B0F0BD44290A000CCB09002C
:100930000C210A00AF4F090006210A00F0B50D4650
:1009400085B055F8044B0646A068174648F0F2FFFC
:1009500002AB0193524B0093701E294602233A4684
:100960001FF02CFB2046029E9DF80C5049F0D2FA55
:1009700010B1204649F0D9FA314640F2FD4028F046
:100980001BFC666084F82050337B7568DB08E376D7
:10099000F37B84F82230B37B003B18BF012384F83B
:1009A0002130B768737BA376384640F2E5224FF6D4
:1009B000FF71BF001FF0B2FB384650F0DFFB94F828
:1009C0002230E0601BB9384650F0D8FB206105F5B5
:1009D00074432333B3FBF5F36B43590801F57401FA
:1009E00001F51051B1FBF3F14B08A26803F5740354
:1009F00003F51053B3FBF1F303EB5503B3FBF5F32E
:100A0000013BC2F84835A268C2F828354B1EE38284
:100A1000A368C3F80815A3680122C3F81425606809
:100A200047F0BCFF1F4A00231146106890BB41F8F5
:100A300023403BF001FCA36800250422A577204653
:100A4000C3F8002229464FF049F8A368D3F82025BF
:100A5000C3F84025A368D3F82425C3F84425A36828
:100A6000C3F80851A368C3F80C51A368C3F8105128
:100A7000A368C3F81451A368C3F80451A3680C22F7
:100A8000C3F80423A26801230E2093606377E577FF
:100A900005B0F0BD0133042B02F10402C5D1CAE751
:100AA00034290A00CC50012070B50D46044640F2AE
:100AB000FD4028F081FB6E7B304647F01FFF6A68DF
:100AC00063689A4204D040F271510D4840F09AF8A0
:100AD000637B022B04D0B34202D040F2FB21F4E747
:100AE0002A7B237B9A4202D040F2CE21EDE7AA7BFB
:100AF000A37B9A4202D040F2A651E6E770BD00BF48
:100B00002046090010B50C4C206890B10B4B1B68B7
:100B100083B95AF048FF236898422368A0EB03008A
:100B200038BF00F1FF3040F2EE23984294BF00201E
:100B3000012010BD0020FCE71C5F0120EC500120CB
:100B4000024A136823EA000313607047EC50012047
:100B5000024A136803431360704700BFEC50012042
:100B600038B50C4B1B78A3B10B4B1B688BB90B4CE6
:100B700025685AF018FF2060236813B923680133F1
:100B8000236035B9064B01221A70064B03F1780237
:100B90009A6238BD2F6E0120EC5001201C5F0120AD
:100BA000646D0120F462012010B504460BF092FA46
:100BB000E3681BB90A4A1168A14203D1BDE810409D
:100BC0000BF09ABAA360074B1968E160196809B184
:100BD00019688C60116801B914601C60EEE700BFF1
:100BE000FC5001200451012008B50BF073FA044AAF
:100BF0001368013B1360BDE808400BF07DBA00BFED
:100C0000F050012008B50BF065FA044A136801336F
:100C10001360BDE808400BF06FBA00BFF050012030
:100C20002DE9F041134E33680BB3134D0BF052FA1C
:100C30002C681CB1BDE8F0410BF05EBA0F4A0123ED
:100C40002B603368346014601BB92B68013B2B6048
:100C5000F0E7D3E900689F68C3E902440BF04CFA5F
:100C60000EB14046B0470BF035FA3B46ECE7BDE825
:100C7000F08100BFFC500120F05001200451012000
:100C800008B525F06FF8C1880348972914BF97224B
:100C900042223FF0A3FF00BF9F40090010B5064A63
:100CA000002352F83340844202EBC30101D90133DF
:100CB000F7E7486810BD00BFC8210A00F0B595B03D
:100CC000054601A80E4617461C4657F009FD10B10F
:100CD000002015B0F0BD3A46314628461FF014FCFE
:100CE0002EF0F6FF830703D10268034B9A42EFD040
:100CF00020600120EDE700BF0C310900014A042308
:100D000033F092BDE4380A00F0B587B008461146CA
:100D10001A4602AB0193254B0093042350F099FC33
:100D20002349182052F001F8DDE904230361214B27
:100D30009A428CBF0123B3FBF2F3C3601E4BD3F87E
:100D4000A831DDE9027604465BB317F0AFF880F016
:100D50000105EDB204F11503009300222B4640F289
:100D60007A51384610F06CFC04F1160360600022E2
:100D7000009340F27D512B46304610F061FC012279
:100D80001146A060606810F0DFFC0122A0681146E7
:100D900010F0DAFC20465AF0ADF820B905203FF0FB
:100DA000E1FE0125D6E7204607B0F0BD14290A0070
:100DB000F0CA090020A10700F4620120F0B50C463A
:100DC00087B054F8045B06462846174648F0CDFD28
:100DD000284648F0D7FD02AB0193094B00933A46F1
:100DE0002146701E04231FF0E9F8059B0093284656
:100DF000DDE90323029958F0E7FD0E2007B0F0BDAE
:100E0000F4280A00F0B50C4687B054F8045B064697
:100E10002846174648F0A9FD284648F0B3FD02AB26
:100E200001930A4B00933A462146701E04231FF09B
:100E3000C5F801230193059B00932846DDE90323B0
:100E400002995CF067FF0E2007B0F0BDD4280A00BD
:100E5000F0B50C468BB054F8045B0646284617469E
:100E600048F083FD284648F08DFD03AB01930E4BFF
:100E700000933A462146701E07231FF09FF8002377
:100E80000193079B0093DDE90312069B28465CF063
:100E900041FF099B00932846089B059A039958F047
:100EA00093FD0E200BB0F0BD9C280A00F0B50D4656
:100EB00087B055F8044B06462046174648F055FDC6
:100EC000204648F065FD02AB0193204B00933A4663
:100ED0002946701E04231FF071F840F2EC430122F2
:100EE0000021039850F0E8FB40F2DC43012200218E
:100EF0000646C5B2049850F0DFFB4FF43373092265
:100F000008210746059850F0D7FB0299104AB2FB1A
:100F1000F1F301FB132202B101332361237DC3F3FB
:100F20008002AA420AD066F3820323756B1E5942DF
:100F300060684FF00002594110F006FC237D0E203E
:100F400067F3C303237507B0F0BD00BF64280A0030
:100F500020A107002DE9F04186B0084611461A4647
:100F600003AB01932D4B0093032350F072FB2C49EC
:100F7000182051F0D3FE2B4B059ED3F8A831DDE9A4
:100F800003870446002B47D016F090FF80F0010540
:100F9000EDB204F11503009300222B4640F2053117
:100FA000404610F04DFB217D60600022C1F38001BE
:100FB00010F0CAFB04F11603009301222B4640F205
:100FC0009441384610F03CFB227DA060B0F10E0346
:100FD00018BF012363F341029307227503D5002252
:100FE000114610F0B1FB04F11703009301222B46C8
:100FF00040F28541304610F023FB05232361237D19
:10100000E06023F00D030E2818BF43F001032046D3
:10101000237506B0BDE8F0810125BAE784280A00EF
:10102000D4CA0900F46201202DE9F04F0D468DB0BD
:1010300055F8044B06462046174648F096FC2046D5
:1010400048F0A6FC08AB01934A4B009329460423C1
:10105000701E3A461EF0B2FF062205A9089822F03B
:1010600031FD9DF81C10002240201FF0EBF8099B79
:1010700004930546069B0A99B3FBF0F303AA04A860
:10108000039357F045FB049E039B6E435D43049618
:101090000395002D4BD0237DDF0704D4364840F262
:1010A00085413FF0AFFD9807DDF814A0DDF82C90E6
:1010B000276940D4554406EB0A0835445FFA89F69F
:1010C0004FF0080B4FF0000A237D990703D5A06865
:1010D000F1094BF009FE217D0A0735D438462EF080
:1010E00093FF217D606881F00401C1F380014BF022
:1010F000FBFD0DF10B01E0684BF0DDFD9DF80B30C1
:10110000217D43EA4A0A0B072BD438462EF07CFF98
:10111000217D6068C1F380014BF0E6FD7600BBF1F4
:10112000010BF6B2D0D108F801AB4545C6D10E206F
:101130000DB0BDE8F08FA06800214BF0D5FD002870
:10114000B8D105203FF00EFDC1F3800181F001010F
:10115000606801F001014BF0C7FD38462EF054FFE6
:10116000C7E76068C1F380014BF0BEFD38462EF042
:101170004BFFD3E72C280A00964909002DE9F04FD0
:101180000D468BB055F8044B06462046174648F0EE
:10119000ECFB204648F0FCFB07AB0193444B00936B
:1011A000294603233A46701E1EF008FF052204A9B3
:1011B000079822F087FC9DF81810002240201FF0AD
:1011C00041F8089B03930546059B0999B3FBF0F38F
:1011D00002AA03A8029357F09BFA039B029A6B435F
:1011E000554303930295002D5AD0227D920704D4D3
:1011F000304840F294413FF005FD049AD4F8109035
:1012000002EB0308002798F800604FBBA068F109C3
:101210004BF06AFD002847D0BA46217D0B0708F144
:10122000010B24D448462EF0EFFE217D606881F04A
:101230000401C1F380014BF057FD48462EF0E4FE57
:10124000217D6068C1F380014BF04EFD0AF1010A77
:10125000BAF1080F21D07600F6B203E0D846D2E703
:101260004FF0000AA068F1094BF03EFDD5E7C1F34D
:10127000800181F0010101F0010160684BF034FD53
:1012800048462EF0C1FE217D6068C1F380014BF01D
:101290002BFD48462EF0B8FED8E70137BD42DDD120
:1012A0000E200BB0BDE8F08F05203FF05BFC00BFC7
:1012B0004C280A00964909002DE9F04F0D4697B0D9
:1012C00055F8044B06462046174648F04EFB20468C
:1012D00048F05EFB10AB0193614B00932946062357
:1012E000701E3A461EF06AFE05220DA9109822F0E3
:1012F000E9FB9DF83C10002240201EF0A3FF129B4A
:101300001399099305460E9BB3FBF0F308AA09A8AD
:10131000089357F0FDF906220AA9119822F0D2FB92
:101320009DF83010002240201EF08CFF149B159970
:10133000079306460B9BB3FBF0F306AA07A8069398
:1013400057F0E6F9089A099B06996B435543079AAB
:10135000099372434E43B54208950792069602D010
:1013600040483FF047FC002D76D00D99C8180390F7
:10137000207D860706D4CE1826B140F294413A4823
:101380003FF040FC0A9EC00706EB020A05D4BAF102
:10139000000F02D040F28541F1E7CE5CA068D4F89E
:1013A00010B0F1094BF0A0FC00283BD105203FF024
:1013B000D9FB7600F6B2A068F1094BF095FC217DCF
:1013C0000A0733D458462EF01FFE217D606881F055
:1013D0000401C1F380014BF087FC0DF11701E068B7
:1013E0004BF069FC9DF81730217D43EA49090B0752
:1013F00029D458462EF008FE217D6068C1F3800193
:101400004BF072FC08F10108B8F1080FD1D10AF8CD
:1014100007900137BD421FD0039B4FF00008DE5DEF
:10142000C146C8E70027B846B946C8E7C1F38001FE
:1014300081F00101606801F001014BF055FC584654
:101440002EF0E2FDC9E76068C1F380014BF04CFC6F
:1014500058462EF0D9FDD5E70E2017B0BDE8F08F25
:101460009C290A0034410900964909000E2AF7B563
:1014700006460D46174602D133483FF03BFB8068D5
:1014800048F058FAAA0706D12A68304B9A4202D18E
:101490002F483FF053FBEB071FD5B288F388534327
:1014A000B3EB650F4FEA650405D8013B00225C21D0
:1014B00028483FF037FB94FBF2F502FB1544042F5C
:1014C00024B22DB22AD12A462146304648F0BEFE2B
:1014D000400040F0010003B0F0BD01AA02212846FF
:1014E00024F078FB019B186851F045F8041EB3887E
:1014F00001DB9C4204DB013B002240F27B61D7E729
:10150000019B586851F037F8051EF38801DB9D42B6
:10151000D5DB013B002240F28161C9E7384651F03A
:101520002AF8B27B4FF0FF31C2F1200221FA02F219
:10153000A223002150F0C0F82A4603462146304637
:1015400048F0BAFE0E20C6E7454E0900885C090047
:10155000D4460900C25109002DE9F04F93B00DABFC
:101560000193684B009305231EF028FD0D9D6649ED
:1015700040F2553228461EF007FEDDF838806249F9
:1015800040F2CC5240461EF0FFFDDDF83C905E4933
:1015900040F2CD5248461EF0F7FD109C204625F043
:1015A000DBF920B12146594850F086F90446012163
:1015B00020464EF0B6FE824660B9204624F0D2FBAB
:1015C000C3880093524840F20E23432240F25A410E
:1015D0003FF004FB119F0E2F13D04B4940F26542A0
:1015E00038461EF0D1FD4146284607F0DBFE49464D
:1015F000284607F0D7FEAB7B102B04D045483FF0C0
:10160000F9FA0027EFE7EB8804930026049BB34226
:1016100003DC0D9813B0BDE8F08FAB89AA68734363
:1016200002EB83030593AB880693B8F80C30D8F827
:101630000820734302EB83030393B9F80C30D9F805
:101640000820734302EB8303089333B24FF0000B7F
:101650000B93069B5B4501DC0136D7E7039B33F810
:10166000024B03933FB10B9A0FFA8BF1384648F0C7
:10167000EDFD00283FD163BAADF82430089B33F864
:101680001B305ABAADF82820C3F3C402C4F30421B6
:101690000792C4F3002242EA4102C3F3042EC3F3CB
:1016A000002141EA4E014FF0400012FB0012079961
:1016B0001AF80220C4F3C40CC3F3C003C4F3C0047B
:1016C00043EA410344EA4C04402114FB0134099BE2
:1016D0001AF804406408E40244EA52040A9AC3F384
:1016E0004513C2F3451213FB01231AF8033044EAF1
:1016F000431464BAA4B2059B23F81B400BF1010B01
:10170000A7E700BFDC290A007CC6090028C9090038
:101710006C5109001234090070B586B003AB019317
:10172000164B009303231EF049FC039E144940F21C
:10173000C92230461EF028FD049D12494FF49A62DA
:1017400028461EF021FDA8684FF49A624FF480717C
:101750001EF0D8FC059C0E2C0DD0094940F26542C4
:1017600020461EF011FD30466A68214637F010FC15
:10177000039806B070BD0024F5E700BF142A0A00E4
:101780007CC60900D8C509002DE9F04FA7B003AB0E
:1017900001934B4B009303231EF010FC039D49491A
:1017A00040F2C92228461EF0EFFC049C204624F09B
:1017B000D9FAC37B002B40D000EB8300424B026977
:1017C0009A423AD1606840F25A4203211EF09AFCD4
:1017D000D4E90378A4680DF11809002632462146A1
:1017E0001F2058F001FC444509F8010B04D0324693
:1017F00041461F2058F0F8FB0136202E89F85F0083
:10180000ECD10DF137060024224639463F2058F02E
:10181000EBFB0134402C06F8010FF5D1059F0E2F8C
:101820000ED0284940F2654238461EF0ADFCAB7B35
:10183000102B07D025483FF0DDF9A0462746CAE720
:101840000027F4E7B5F806900026B14503DC0398BD
:1018500027B0BDE8F08FAB89AC68B5F804A073433E
:1018600004EB83044FF000080FFA86FBC24501DC4D
:101870000136EAE737B15A460FFA88F1384648F0A0
:10188000E5FCC8B9228853BAC3F3451398336B44B7
:1018900013F8601CC2F30423C2F3C40298339832D5
:1018A0006B446A4413F8203C12F8802C43EAC223AC
:1018B00043EA41135BBA238008F101080234D5E7FB
:1018C0002C2A0A007CC609001D8305001234090079
:1018D0002DE9F04FABB00FAB0193924B0093032374
:1018E0001EF06CFB0F9C904940F2C92220461EF06E
:1018F0004BFC3022002112A84FF052FD109E16F032
:10190000030566D13368894A934224D112AF294630
:1019100030464EF04CFB01353B46032D07F11407D2
:1019200083ED000AF3D1119F0E2F63D07E4940F260
:10193000654238461EF028FC12AD0DF178080026ED
:10194000731E0B2B71D8DFE803F06D70686A706A44
:1019500057706D706873764A934217D10DF148083D
:101960004746294630464EF022FB4346691C83ED2C
:10197000000A30464EF01BFB0235062D87ED030AA8
:1019800008F1140807F11007EBD1CCE7694A93423C
:1019900011D14FF00308294630464EF008FBB5FB45
:1019A000F8F72AAB2F44013503EB8707092D07ED24
:1019B000180AF0D1B7E7604A93420AD112AF29461C
:1019C00030464EF0F4FA01350C2DA7EC010AF6D1A1
:1019D000A9E7304624F0C6F9C38801934FF4877312
:1019E0000093564840F20D1340F2272240F2262180
:1019F0003FF008F900279FE7514BB5EC010A07EECD
:101A0000903AF8EEE77A013627EE800A35F024FDA9
:101A1000BDEEC00AA8EC010A92E74A4BEDE74FF48D
:101A20000033EAE74FF40043E7E74FF48033E4E79D
:101A3000A37B102B02D044483FF0DCF81E9B02939E
:101A40001F9B0393209B0493219B0593229B079349
:101A5000239B0893249B0993259B0A93269B0B9316
:101A6000279B0C93B4F80690289BDDF8A4A00D9357
:101A70000026B14503DC0F982BB0BDE8F08FA38999
:101A8000A568B4F804B0734305EB83054FF0000874
:101A900032B2C34501DC0136EBE747B10FFA88F1FA
:101AA0003846069248F0D2FB069A002835D1B5F8A0
:101AB00000C0039B9CFA9CF1C1F3451103FB01F0AC
:101AC000029BCCF3C40E03FB0E00049BCCF3042C4E
:101AD00003FB0C00059BC3180693089B07984B4318
:101AE00000FB0E33099800FB0C330A9803440C9852
:101AF00041430B9800FB0E110D9800FB0C1106984A
:101B0000A3F306435144A0F305405B0143EAC0231D
:101B1000A1F305410B435BBA2B8008F101080235A4
:101B2000B7E700BF5C2A0A007CC6090054CA090056
:101B300004CA0900A8C9090040C909007B3309008B
:101B4000C1FF3E00E1FF1E00123409002DE9F04FF5
:101B50002DED028BA7B002AF07F1700301938F4BFD
:101B6000009308231EF02AFAD7F870B08C4940F28F
:101B7000C92258461EF008FBD7F88C303B660E2B66
:101B80001CD0874940F2654218461EF0FDFAF86FF6
:101B900024F05EF8D7F874804046F0EE408A24F0D6
:101BA0009BFFC4070DD4404624F0DCF84FF40B72C1
:101BB000C3887C4840F269613FF024F800233B660B
:101BC000E5E7441007EE904AB8EE677AF1EEC77A7F
:101BD000FDEEE77A17EE905AE90703D505FB05F30A
:101BE0009C4202D070483FF005F8A300073323F071
:101BF0000703ADEB030D02AB4FF000097B654E46CA
:101C0000A1451AD1B86F0E2828D024F021F8B0EEE3
:101C1000408A6B08FB6697F880307B6397F88430C6
:101C20003B6397F88830FB62FB6E0133BB669BF821
:101C30000E30102B1FD05D48D5E74FEA4901042232
:101C400041F00101404626F0B1FA50F094FC7B6D62
:101C5000064443F8290009F10109D1E7B7EE007AFB
:101C600036B107EE906AF8EEE77A87EE278AD0E77A
:101C7000B0EE478ACDE7BBF804304D4D4D4CD5F85A
:101C800000A001335B10BB65BA6DBB6E02FB03F6AF
:101C9000B60040D1BAF1000F02D0504632F084F9BC
:101CA000002323602B609A469FED430A28EE000A2A
:101CB00035F0D2FBFDEEC07A9FED400AC7ED127AF7
:101CC00028EE800A35F0C8FBFDEEC07ABBF806307E
:101CD0003B6217EE903A5B007B61FB6EC7ED117AB9
:101CE0005B42FB65FB6E5B003B614FF000093B6AAA
:101CF0004B4500F3D181BBF80650FB6EEC1A24EA89
:101D0000E474A54200F33383386F9437BD46BDECCD
:101D1000028BBDE8F08FBAF1000F00F0B3812368A9
:101D20009E42C1D9264B1C6820465AF0E0FC8642F0
:101D300080F09F8155460C2E55F8043DB04623F0A7
:101D4000030938BF4FF00C08C14580F09B8005EBBC
:101D500009004168CA0706D521F0030109F104030F
:101D60000B4443452ED2314620465AF0C7FC054667
:101D7000002800F07E81B1454A46514628BF3246D0
:101D80004FF0CDFA514620463DF0F4FAAA46084BF2
:101D9000C3F800A0074B1E6086E700BF5C290A005D
:101DA0007CC6090051510900903309001234090022
:101DB0002C670120306701200000804700007C4A2A
:101DC0004C5C0120638AC3F3C7139942AAF1080946
:101DD00080F007812269C2F38532B3FBF2F300225F
:101DE000B1FBF3F37B66D0E902C1CCF80C10C1F86B
:101DF00008C021697B6ED4F820E0C1F3853102FB75
:101E000001315EF8213098421AD1A4454EF821C024
:101E100016D1D4F81CE07B6E5EF822104FF0010C56
:101E20000CFA03F321EA03014EF82210E36953F898
:101E300022302BB9A3690CFA02FC23EA0C03A3613C
:101E40005AF8043C4268043322F0030213444AF86F
:101E5000043C23F0030343F80590BA4B1BB1012265
:101E60001021AFF300805AF8043C23F003032B4405
:101E70005A6822F002025A605AF8043C23F0010327
:101E80004AF8043C23F0030308F110029342FFF4E4
:101E90007EAF4544A3EB08036A68043B02F00302EB
:101EA00013436B605AF8043C03F0030343EA08034E
:101EB0004AF8043C6B6805F1080E23F003037344F1
:101EC00043F8045C53F8042942F002025A6068683F
:101ED00020F0020320F0030043F0010370446B6024
:101EE00050F80419CB074DD5638A21F00301C3F3E1
:101EF000C7138B4240F28E8022694FF0000CC2F370
:101F00008532B3FBF2F3B1FBF3F37B66D0E9021247
:101F1000CA60916022697B6ED4F82090C2F385324A
:101F20000CFB023259F82230984219D1A14249F8EB
:101F3000221015D1D4F81C807B6E58F82C2001217A
:101F400001FA03F322EA030248F82C20E36953F86C
:101F50002C302BB9A36901FA0CF123EA0103A36128
:101F60006B684268043322F0030213446B6023F071
:101F700003039E44734B4EF8045C1BB101221021F5
:101F8000AFF300806968638A206921F00301C3F31D
:101F9000C7139942C0F3853053D2B3FBF0F3B1FBC2
:101FA000F3F30022216A02FB003051F82010C5E94A
:101FB0000214CD602169206AC1F3853102FB013131
:101FC00040F821500125A16905FA02F00143E069BA
:101FD000A16150F8221005FA03F3194340F82210CA
:101FE000D5E6A9B1B1FA81F2C2F1200294F812C08B
:101FF000531ECCF3021CA3EB0C0321FA03F30121C3
:1020000001FA0CF14B40217C7B66A2EB5112EAE60F
:102010000A46EBE799B1B1FA81FCCCF1200CA27C25
:102020000CF1FF33C2F302129B1A21FA03F30121D0
:102030009140227C4B407B66ACEB521C66E78C46A1
:10204000EDE7A1B1B1FA81F2C2F1200294F812C019
:10205000531ECCF3021CA3EB0C0321FA03F3012162
:1020600001FA0CF14B40217CA2EB51129AE70A468F
:10207000ECE7504631F098FF334B00221A603046AF
:102080003EF022FD304632F03FF82660824628605E
:1020900000287FF409AEF2E7BBF80C30DBF808202B
:1020A00009FB03F302EB8303BA6EFB63BB6EB9FB60
:1020B000F3F302FB1393BA6D53430AEB8303FB6103
:1020C000BBF80430BB613B690133BB63FB6EA9EB1A
:1020D0000303BB600FFA89F34FF000087B60BB6914
:1020E00043451DDCFB6E4B4517DCBBF80C00BD6E99
:1020F000BC6EBBF80420A9EB03014843B1FBF4F428
:1021000005FB1411BC6DDBF80830614352000AEB8B
:10211000810103EB80004FF002F909F10109E6E5C6
:102120003B6E9BB17A680FFA88F1184648F08EF83A
:1021300060B1FB6B33F81830FA6922F8183008F1F7
:102140000108CCE7000000002C670120DBF8081034
:102150003964BBF80C103965F96EBBF80430BBF874
:102160000620414500F3BC80591A884580F2B880AA
:10217000F96E494500F3B480511A894580F2B08068
:10218000BB683A6DD7F85CC002FB03F4A300FB64A4
:102190003B6C002003EB4803BB62024678660146B5
:1021A0007B6DFC6CFE6D03EB80033B64BB6A2344D8
:1021B0007B627B6A33F816503B6C53F804EB3B644C
:1021C0006CBAC5F3C4030EFB0311C4F345137C6E54
:1021D0000EFB03437B66FB6E0136C5F30425B34259
:1021E0000EFB0522E5DABB6B1844D7E9134304EB79
:1021F0008303FB64FB6E0CF1010C6345D0DAD7E975
:1022000011307C6E01FB00317B6904FB0033D7E9A0
:102210001104A3F3064302FB0402A1F305415B0191
:10222000A2F3054243EAC12313437A6B002A54D038
:102230001D1205F0F8027A66DA1002F0FC01DB00EC
:102240003965D9B2F964F96B31F8180041BAC1F3B4
:10225000CC0606F0FC043C64FC6CC3F3421323433D
:102260007C6EC5F3421525433C6DC2F381122243B7
:1022700002EB8202C2EB0212262415FB04254FF06A
:102280000F0413FB04533C6C3A6BC6F381163443C2
:1022900000F0F80CC900C0F3421004EB840401F014
:1022A000F80E4CEA0000C1F34211C4EB04144FF0E5
:1022B0002605C2EBE3134EEA01010F2210FB054095
:1022C00011FB0201B3EBE11FF96AB4BF0122002246
:1022D0004FF6FF738A4208BF00235BBA9BB22BE71D
:1022E0000024013A013BFE6DBA627B6222467C66A5
:1022F0002146BB6AD7F85CC009EB060020EAE07013
:102300009842A8BF18463B6D4343FB607B6D03EBCF
:102310008403FB647B6A08EB0C0525EAE5759D42A6
:10232000A8BF1D463B6C03EB4505FB6835F8235001
:10233000FB6C53F804EBFB6468BAC5F3C4030EFBF3
:102340000311C0F34513786E0EFB03037B66FB6E2F
:102350000CF1010CC5F3042563450EFB0522D9DA07
:10236000BB6B1C44FB6E0136B342C2DA47E7BE6E5C
:10237000BBF80C00B96EB4FBF1F106FB1141BE6D68
:10238000DBF80830BBF804206043714352000AEBCD
:10239000810103EB80004EF0C2FF0134B1E400BFC5
:1023A0002DE9F04F2DED028B89B005AB01935E4B0B
:1023B000009303231DF002FE0698C8B123F048FCE9
:1023C000B0EE408A059C594940F2C92220461DF0D2
:1023D000DBFE079F0E2F0ED0544940F2654238466F
:1023E0001DF0D2FEA37B102B07D051483EF002FC1B
:1023F000B6EE008AE6E70027F4E79FED4E0A28EEE6
:10240000000A35F029F8B4F806A0BDEEC08A00260F
:102410004FF0260B4FF04009B24505DC059809B096
:10242000BDEC028BBDE8F08FA3880393A389A56858
:10243000734305EB83054FF00008039B434501DC24
:102440000136E9E73FB132B20FFA88F1384647F07A
:10245000FDFE002864D129884BBA01F0F802C1F3CF
:1024600042111143C3F3CC0202F0FC0CC2F38112FF
:1024700042EA0C00DB0000EB800203F0F80EC2EB36
:102480000212C3F3421343EA0E034FF00F0C18EE8F
:1024900010EA11FB0B2213FB0C22BEEBE21F4FEAEA
:1024A000E21C3DDACCEB4E024FF6D57C10FB0CFC67
:1024B0004FF6EB7E11FB0ECC4FF6CA7E10FB0EF0F2
:1024C00011FB09014FF6F67013FB09CC13FB001347
:1024D000DB114BF2D2614FEAEC1C594345F61A006E
:1024E00000FB0C11144882F30802A2EB2141434384
:1024F00002EB2343114881F30801C90083F3080369
:1025000001F4FC6100EA03230B430D4901FB0CFCC1
:1025100002EB2C4282F3080243EAD2035BBA2B801F
:1025200008F10108023588E7442A0A007CC6090040
:102530001234090000008043E966010000F8FFFF43
:10254000A2C501002DE9F04F2DED028B9FB014AB19
:102550000193A94B00930A231DF030FDA74914985D
:1025600040F256321DF010FEA44940F2BE5207461A
:1025700015981DF009FEA149834640F2BF521698F6
:102580001DF002FE049018980E2836D023F060FB50
:10259000F0EE408A19980E2832D1B7EE008A38EE54
:1025A000688A179E964940F2123230461DF0ECFDC3
:1025B0001A9D944940F2D72228461DF0E5FDBB88BC
:1025C000BBF80410994215D1FA88BBF80630934243
:1025D00010D1B87B9BF80E2082420BD104988088E2
:1025E000884207D10499C988994203D1049B9B7BF7
:1025F00093420AD084483EF0FDFAF6EE008AC9E71D
:1026000023F026FBB0EE408ACBE73479092C0EDCB0
:102610000121A14011F0AA0F05D1092C07D1082BE7
:1026200007D07A48E7E7102B03D07948E3E77948E9
:10263000E1E71B98B5F904500E281FD04FF09BFF1F
:102640000023089009931C980E281CD04FF093FF8C
:1026500000230A9005931D980E281ED040F2654273
:1026600066491DF091FDBB8882889A42804603D15D
:10267000C288FB889A420BD06748BCE7002301213F
:10268000CDE90831DFE70123059300230A93E2E750
:10269000837B082B03D06148ADE74FF00008EBB215
:1026A0000B93BB88ADF848300025FB88119511A924
:1026B0003846ADF84A3013950FF078FFF0EE687A9F
:1026C000FEEECC7A092CCDED027AF0EE487AFEEEE1
:1026D000CC7ACDED067A40F0BD809DF8203007938E
:1026E0009DF828300699089378E0BA89BB68DBF832
:1026F00008406A4303EB820ABBF80C306B4304EBDF
:1027000083030393049B9A899B686A4303EB8202C9
:10271000B8F1000F00F09C80B8F80C00D8F8083031
:10272000684303EB8000D64652E0099B002B5ED144
:10273000039B079E1B789B1B18BF0123059E002E41
:1027400057D11678089C361B18BF012670B190F837
:1027500000C00699BCF1000F0CBF002606F0010670
:1027600001FB0CF17F31FF2491FBF4F1002B63D0CE
:10277000039C14F8013B0394029C6343002E57D042
:102780000B9C12F8016B012C01FB06F648D106FBED
:1027900003FC0CF57F4909F1FF093CEA2C0C28BF2A
:1027A000CC461E44A6EB2C46029B4B439C4648BF9E
:1027B00003F1FF0C029B0B44A3EB2C23002B45DD04
:1027C00096FBF3F383F308030EF8013B00B10130ED
:1027D000BE88AEEB0A039E42A7DC0135FB889D4212
:1027E00083DB0E201FB0BDEC028BBDE8F08F012310
:1027F000A4E7059EAAE700BFF42A0A007CC60900E8
:1028000044C609007CC80900144F09009C4B09000C
:10281000804B0900F5430900184A09002B4A0900BA
:10282000C1F58074634348BFFF3306EB2326BBE743
:10283000002B06DAFF3304E02EB112F8013B4B43C4
:10284000F8D41B12BEE79EF80030BBE70023B9E7BF
:10285000404668E704F0FB03069E0D93FB889D420B
:10286000BFDABA89BB686A4303EB8203BBF80C206A
:102870000C93DBF808306A4303EB82030E93049B4E
:102880009A899B686A4303EB82030F93B8F1000FA8
:1028900000F00481B8F80C20D8F808306A4303EB44
:1028A000820307930023A7E00E9B039A039933F852
:1028B00012200F9B33F811100D9B032B099B01BFB6
:1028C00052BA49BA92B289B2002B40F09D80089B5F
:1028D000B3EB020C18BF4FF0010C059B002B40F02E
:1028E00096800A9B5B1A18BF0123079880B10446A3
:1028F000069814F801EB079400FB0EF6BEF1000FEA
:102900000CBF002303F001037F36FF2096FBF0F697
:10291000BCF1000F00F0A880002B00F08E80029B1D
:102920000298734348BFFF3300EB0609A9EB232944
:10293000B9F1000F5EDD1312D410D20003F0F803DA
:1029400004F0FC04D2B24343444342430B984FEAA1
:10295000212E4FEAE10CC9000EF0F80E0CF0FC0C31
:10296000C9B2012806FB0EFE06FB0CFC06FB01F1BA
:102970004FD10EFB03FA0AF57F40FF303AEA2A0AEC
:1029800028BF824673440CFB04FEA3EB2A430EF5DA
:102990007F4A0AF1FF0A3EEA2E0E28BFD64664445B
:1029A00001FB02FCA4EB2E440CF57F4E0EF1FF0E52
:1029B0003CEA2C0C28BFF44602EB010AAAEB2C4A95
:1029C0000D9A93FBF9F394FBF9F41B02E40003F472
:1029D000784304F4FC6423439AFBF9FA032ACAF30C
:1029E000C40A43EA0A0301D15BBA9BB20C9A039969
:1029F00022F81130039B01330393039ABB889A4258
:102A0000FFF652AF013529E74FF0010C65E7059B52
:102A10006BE7C6F5807A5046434348BFFF334443D3
:102A200048BFFF345043024648BFFF320EEB23231A
:102A30000CEB242401EB222AC2E7029B029802F449
:102A40007841594302F4FC6343434FEA212148BFD4
:102A5000FF3341EA2323029902F01F024A4348BF91
:102A6000FF3243EA2223C0E79BB101F4784201F42C
:102A7000FC63734306FB02F201F01F0148BFFF3302
:102A80001212714342EA232348BFFF3143EA212354
:102A9000ABE70C9B039A33F81230A7E7CDF81C8004
:102AA00000E700BF2DE9F04F99B011AB01933F4B08
:102AB000009307231DF082FA3D49119840F2C92284
:102AC0001DF062FB054605220BA9129820F0FAFFC3
:102AD000EB88AA8813A909A801F0DEFABDF928300D
:102AE000BDF92690BDF924A0BDF92AB00493A3EB4B
:102AF0000A049DF83410ABEB0903002240205C432C
:102B00001DF0A0FB0C9BB3FBF0F6179B05900E2B62
:102B10004F46039308D018464FF02DFD0690B4425F
:102B200005D924483DF0F6FF00230693F7E7AB7B79
:102B30000B9C01269E40013EBB4534DC049BADF856
:102B40003C30284600230EA9ADF838A0ADF83A90E5
:102B5000ADF83EB010930FF029FD0E2019B0BDE87E
:102B6000F08F059B022B18D0042B19D014F8013BD1
:102B700003990E2902D00699994207D033400FFAE3
:102B800088F1284607920FF035FD079A08F10108F1
:102B9000049B4345E5DC0137CEE734F8023BE7E729
:102BA00054F8043BE4E7D0463AB2F1E7042C0A00BB
:102BB0007CC60900263C09002DE9F04F97B002AF12
:102BC00007F140030193B54B009304231DF0F6F980
:102BD000B349786C40F2BD521DF0D6FAB0490646B2
:102BE00040F25632386C1DF0CFFAFC6CAD4981468C
:102BF00040F2912220461DF0C7FABD6CAA4940F26E
:102C0000C25228461DF0C0FAB9F804A0B388534553
:102C100009D1D9F80430BB60B9F80630BB61BA6994
:102C2000F388934202D0A1483DF0D0FF99F80E30CE
:102C3000102B03D0012B01D09D48F5E72A79092AF2
:102C400006DC0121914011F0AA0F03D1092A06D018
:102C50009848E9E7B37B102B06D09748E4E7B37BAD
:102C6000082B01D09548DFE7032AB4F9043053D08C
:102C7000072A4FD0052A52D1002242F0020B904A77
:102C8000DBB252F8235069780AEB410303EB4303AC
:102C90005B0007336A46DB08A2EBC3039D460A23A9
:102CA00001EB41084B4302AC03EB8A03D04404EB35
:102CB000410204EB48081C440AF11F0368465B0903
:102CC000A0EB43139D46BA62C7F82C803C6343F8DF
:102CD000081B30467B62594600234CF0A0FF6B78FE
:102CE000009342460123594630464CF098FF6B78DA
:102CF000009322460223594630464CF090FF4FF095
:102D000000084446BB69434540F3DC80BB6A3B6234
:102D1000002227E00122B0E74FF0010BAFE74FF0B0
:102D2000000BACE73B6A786A33F9123023447F2BFF
:102D3000D4BF00210121802B8154B4BF0021FF2189
:102D40005B1AFB61E81C4FF0000C29788C4544DBD2
:102D5000AC78FB6914FB03F4002CB8BFFF3444F3D8
:102D60000F2401329245DDDC7A6A414648465AF02A
:102D700042FFFB6AFB61BB623B6B7B61FB623B6AB0
:102D80003B6308F101037B60BB6908F101029342D8
:102D900000F098806B7800933A6A08F10303594673
:102DA00030464CF03CFF5246002A35D17A6A7968A9
:102DB00048465AF020FF7B69BB623B6AFB62FB69B5
:102DC0003B636B780093FA6908F104035946304677
:102DD0004CF025FF08F1020894E790F9011090F9F2
:102DE000004007F1500303EB8101FB6951F8281CF7
:102DF000796190F90210144411FB03F17B690029F9
:102E000033F814E0B8BFFF310EEB212E033023F866
:102E100014E00CF1010C98E7013AFB6933F8123029
:102E2000234419B27F29D4BF0020012080297C6A65
:102E3000B4BF0021FF215B1AA0543B61E81C4FF096
:102E4000000C29788C4509DBAC783B6914FB03F452
:102E5000002CB8BFFF3444F30F24A5E790F901100C
:102E600090F9004007F1500303EB81013B6951F8F1
:102E7000281CF96090F90210141B11FB03F1FB6888
:102E8000002933F814E0B8BFFF310EEB212E0330D8
:102E900023F814E00CF1010CD3E700BFE42C0A0086
:102EA0007CC6090060C8090044C6090070410900D9
:102EB000C835090002340900BA350900B1350900E6
:102EC000DC2C0A00BA68002307F134014846C7E940
:102ED0000E237B630FF06AFB0E205437BD46BDE81E
:102EE000F08F00BF2DE9F04395B00AAB0193304B52
:102EF00000930A231DF062F82E490A9840F25632D8
:102F00001DF042F940F27B638288044600210C9850
:102F10004EF0D2FBE28840F28163002107460D9813
:102F20004EF0CAFB234940F2BD5280460B981DF07B
:102F30002BF90546C38882880EA908A801F0ACF8D1
:102F4000A27BAB7B9A4202D21B483DF053FE129803
:102F50000E2825D04FF00FFB4FF0000906461398BE
:102F60000E2821D04FF007FB0023CDE90603BDF961
:102F700026300393BDF924300293BDF9223001932A
:102F8000BDF9203000932046CDE904690FFA88F39B
:102F90003AB2294606F0C4FF0E2015B0BDE8F08312
:102FA0004FF001090026DAE701230020DDE700BF2A
:102FB000642C0A007CC60900D83509002DE9F04FC1
:102FC00091B00BAB0193974B009305231CF0F6FFD8
:102FD00040F2563294490B981DF0D6F80E9B827B36
:102FE000029301239340029A9A42064602D38F48E5
:102FF0003DF000FE0F9F6FF00042974203D0BB42AE
:1030000001D88B48F4E7BDF93090B9F1000F02DB2D
:10301000B388994501DB8748EAE7BDF93480B8F108
:10302000000FF8DBF3889845F5DA029BBB4200F00D
:10303000F58000201AF0E6FB054648464FF0B6FE44
:10304000069040464FF0B2FE06A90790022024F0F9
:1030500041F8014628464FF0D4FD6FF000439F42EF
:103060000CD106984FF087FA044607984FF083FA80
:1030700021B202B2304647F0E9F80746002304AA1D
:1030800005A928460593CA464FF0F1FDCDF80C80FE
:10309000059A8AB9039BADF820900AF1010A013321
:1030A00008A93046ADF82280ADF824A0ADF826304E
:1030B0000A920FF07BFAB1E004AA05A928464FF066
:1030C000D6FD0021284623F051FD044680684FF0CC
:1030D00052FA8346E0684FF04EFA0FFA8BF102B2D3
:1030E000304647F0B3F8B84205D004AA05A92846EF
:1030F0004FF0BDFDCCE7A0684FF0DEFB8346E068F3
:103100004FF0DAFBCB45039BB8BF0FFA8BF9D345E1
:10311000C8BF0FFA8BFA4045B8BF0FFA80F8984243
:10312000C8BF03B2A068C8BF03934FF024FA834618
:10313000E0684FF020FA029B02B20FFA8BF13046A2
:103140000FF058FAE0684FF0B7FB002811DDA368D4
:103150000893E0684FF0B0FB0138400040F00100F8
:10316000099008A9022023F0B5FF014628464FF038
:1031700048FDA0684FF0A0FB002811DDA0684FF0CB
:103180009BFB0138400040F001000890E368099380
:1031900008A9022023F09EFF014628464FF031FD8A
:1031A000A0684FF089FBB3880130984211DAA0681B
:1031B0004FF082FB0130400040F001000890E368CE
:1031C000099308A9022023F085FF014628464FF005
:1031D00018FDE0684FF070FBF3880130984211DA77
:1031E000A3680893E0684FF067FB0130400040F0AF
:1031F0000100099008A9022023F06CFF014628462F
:103200004FF0FFFC04AA05A928464FF030FDFDF75A
:1032100007FD094B9B6A002B3FF43AAF0E2011B01B
:10322000BDE8F08F742B0A007CC60900B03309009A
:103230009F4109002E370900F46201202DE9F04F6B
:1032400093B00DAB0193714B009305231CF0B6FEB8
:1032500040F256326E490D981CF096FF827BDDF8E5
:103260004480012393409845044602D369483DF0C9
:10327000C1FCBDF938A08288BDF9406040F27B6393
:10328000002150464EF018FABDF93C90E28840F219
:103290008163002148464EF00FFA40F20E520021A1
:1032A00030464EF001FA0EAA8CCA0025D11BCDE99A
:1032B00009553A44ADF81C10D91B3B44ADF8202009
:1032C000ADF82230A388ADF81E1007AA1046ADF85D
:1032D0002C300AA9E388ADF82E300C9549F0A7FEF2
:1032E00007A920460FF062F94B4940F27B6347F68D
:1032F000FF7250464EF0E0F940F2816347F6FF72EC
:10330000454948464EF0D8F9A088E28850454FEA32
:103310004703A8BF5046C3F103034A451BB200B29E
:10332000A8BF4A4612B2039320EAE073049322EA4C
:10333000E277B54203DD0E2013B0BDE8F08F049BA9
:1033400006EB070B05EB03090FFA8BF20FFA89F175
:10335000434620460FF04EF9049BA7EB060A591B83
:1033600009B20FFA8AF24346204605910FF042F95E
:103370000FFA8BF20599434620460FF03BF90FFAFE
:103380008AF20FFA89F1434620460FF033F9049B85
:1033900005EB070B03EB06090FFA8BF243460FFA16
:1033A00089F120460FF026F9049BA3EB060A0FFAD9
:1033B0008BF24346A7EB050B0FFA8AF120460FF07C
:1033C00019F943460FFA8BF20FFA8AF120460FF0F3
:1033D00011F90FFA8BF243460FFA89F120460FF0EC
:1033E00009F9039B002BC5BF039BAA1B06330A33B5
:1033F000D2BF03EB850303EB820306F1FF361BB25A
:10340000C8BF36B20393013593E700BFB42C0A005E
:103410007CC609002E3709000080FFFF2DE9F0432C
:103420008FB008AB01932A4B009306231CF0C6FD16
:1034300040F25632274908981CF0A6FE827BDDF840
:103440003490012393409945044602D322483DF02D
:10345000D1FB0B98099A0C990A9B15B207B21EB2C0
:103460000FFA81F8BD42B5BF421C384628460132EA
:103470004645B4BF4B1C0133ADF80E304FF000038E
:10348000CDE90433ADF80C20A288ADF81820E2880D
:10349000ADF81A20B4BF3146414602AAADF8080083
:1034A000ADF80A10104605A9079349F0C0FD02A91E
:1034B00020460FF07BF82046CDE900893B46324696
:1034C00029464AF0E3FE0E200FB0BDE8F08300BFAE
:1034D000442B0A007CC609002E3709002DE9F04F65
:1034E0009FB019AB01935B4B009305231CF066FD65
:1034F0005949199840F256321CF046FE052210A98F
:1035000006461A9820F0DEFA05220DA91B9820F035
:10351000D9FA9DF84810002240201CF093FE9DF837
:103520003C100546002240201CF08CFE854202D053
:103530004A483DF05FFB119BB3FBF5F30993099AF1
:103540000E9BB3FBF5F39A4201D04548F1E71C9B73
:103550000293B37B029A012404FA03F39A4201D343
:103560004048E6E79DF874300A93109B07932A467B
:103570000D9B0798089300214DF056FA2A4607B292
:10358000002108984DF050FA0FFA80F8CDE9037841
:10359000C246CDF81880BB460597099BA3422BD89D
:1035A0000A9B43B1029BDDE90312CDE9008330465B
:1035B0003B464AF06BFE059BADF84C30069BADF8E0
:1035C0004E300023CDE91533ADF852A0ADF850B020
:1035D000B288ADF85C20F288ADF85E2013AA16A977
:1035E0001046189349F023FD304613A90EF0DEFF74
:1035F0000E201FB0BDE8F08F214607982A464DF0F7
:1036000013FA214603B22A4608980B934DF00CFAA0
:10361000029B0FFA80F9CDE90093DDE903120B9BC1
:1036200030464AF033FE0B9B059A9A42D4BF05926E
:1036300005939B45069AB8BF9B464A45D4BF069260
:10364000CDF81890CA45CDE90339B8BFCA46013450
:10365000A3E700BF3C2C0A007CC609004A4D0900C4
:103660005F4D09002E370900F0B591B00AAB019308
:10367000274B009306231CF0A1FC40F2563225494B
:103680000A981CF081FD827B0F9F012393409F428B
:10369000044602D320483DF0ADFA8288C3880BA9C6
:1036A00002A800F0F9FC029B04930025039B0593FC
:1036B00004A8069549F0AAFCA388ADF8203004AA16
:1036C000E388079507A91046ADF82230099549F01F
:1036D000AEFC04A920460EF069FFBDF91050BDF9FB
:1036E0001430AB4202DC0E2011B0F0BDBDF9126007
:1036F000BDF91630B34202DC01352DB2EFE7324698
:103700003B462946204601360EF074FF36B2EFE7FD
:103710009C2B0A007CC609002E3709002DE9F047D2
:1037200086B003AB01931F4B009303231CF046FCB0
:1037300040F2C9221C4903981CF026FD827BDDF86B
:103740001090012393409945044603D2DDF814A05C
:103750009A4524D3154840F20D313DF053FA3A46CC
:103760002946204646F072FD814505D153463A462A
:10377000294620460EF03EFF08F10108E3880FFAC3
:1037800088F79F42EBDB0136A38835B29D4203DB0D
:103790000E2006B0BDE8F0874FF00008EEE70026E7
:1037A000F2E700BFDC2A0A007CC60900325109009A
:1037B0002DE9F04F2DED0C8B99B00BAB01930D4B18
:1037C00000930D231CF0FAFB0B490B9840F2563284
:1037D0001CF0DAFC40F2BD52804607490C981CF000
:1037E000D3FC98F80E20837B9A42074608D2034800
:1037F0003DF000FA742A0A007CC60900D835090099
:10380000B8F804100D98490859F008FEB8F80610E9
:103810000DEE100A49080E9859F000FEB9880CEE1A
:10382000100A4908119859F0F9FDF9880BEE900A31
:103830004908129859F0F2FD0023109C009307AA42
:103840000DF11E010BEE100A0F9811F011F9B8F9E5
:103850000620B8F904300092204606AA0DF11A019C
:1038600011F006F9BDF91E20BDF91A00824206DDED
:103870001346ADF81E00ADF81A2002461846BDF9F1
:103880001C30BDF918108B4206DD1C46ADF81C102B
:10389000ADF818300B462146002ABCBF0022ADF817
:1038A0001E20B8F80440002BBCBF0023ADF81C302C
:1038B000A242B8F80620C8BFADF81E409342C8BF68
:1038C000ADF81C2000284FF0000380F21B829942C3
:1038D000ADF81A3002DAADF8183019468A424FF0C6
:1038E0000003B8BFADF81820149C1398009305AAE4
:1038F0000DF1160111F0BCF8B7F90620B7F9043044
:103900000092204604AA0DF1120111F0B1F8BDF9A0
:103910001620BDF91200824206DD1346ADF81600EE
:10392000ADF8122002461846BDF91430BDF910104A
:103930008B4206DD1C46ADF81410ADF810300B4676
:103940002146002ABCBF0022ADF81620BC88002BFF
:10395000BCBF0023ADF81430A242FA88C8BFADF84E
:1039600016409342C8BFADF8142000284FF0000362
:1039700080F2D2819942ADF8123002DAADF81030FF
:10398000194615988A42B8BFADF810200E2800F0ED
:10399000CD8122F05DF9F0EE40CA16980E2840F075
:1039A000C881B7EE00AA17980E2800F0CD814EF01E
:1039B000E2FD002383460293BDF91630BDF91C20B9
:1039C000039208EE103ABDF91430BDF91A60BDF942
:1039D0001E90BDF918A008EE903ABDF9123009EE1C
:1039E000103ABDF91030B0EE6C0A09EE903A35F09D
:1039F000FDFDF0EE40AAB0EE6C0A0CF063FBF8EEB1
:103A0000EB4AB8EECB4A20EE647A2AEE843A27EEEF
:103A10000A7A23EE0A3AF8EECD3A77EE035A6AEEC6
:103A2000E47A60EE046A02EE906A75EEA35A67EEDD
:103A30008A7A66EE8A6AF8EEE22AB8EECC5A37EE57
:103A4000E66AF4EEE25AF1EE10FA36EE056A039AEF
:103A500040F17F81FDEEE52A12EE903A0FFA83FCE9
:103A600002EE909AF8EEE22AF4EEE25AF1EE10FA43
:103A700040F37181FDEEE55A15EE903A1DB205EE68
:103A800090AAF8EEE55AB4EEE56AF1EE10FA40F1CC
:103A90006481FDEEC65A15EE903A19B205EE902AF1
:103AA000F8EEE55AB4EEE56AF1EE10FA40F357810C
:103AB000BDEEC66A16EE103A1CB2BB881BEE900A29
:103AC0001B1A06EE103AB8EEC66A02EE90CA60EE15
:103AD000065A2AEE866A65EE8A5A26EE0A6A33EE9E
:103AE000253AF8EEE22A33EE233A76EE666AB4EE31
:103AF000E23AF1EE10FA76EE856A05D5FDEEC32ABC
:103B000012EE903A0FFA83FC02EE905AF8EEE22A97
:103B1000B4EEE23AF1EE10FA04DDBDEEC33A13EE74
:103B2000103A1DB203EE101AB8EEC33AF4EEC36AAF
:103B3000F1EE10FA04D5BDEEE63A13EE103A19B2E2
:103B400003EE104AB8EEC33AF4EEC36AF1EE10FA8F
:103B500004DDFDEEE66A16EE903A1CB2FB881BEE21
:103B6000100A1B1A06EE903AF8EEE66A02EE90CAC8
:103B70002AEEA63A60EE266A23EE0A3A66EE8A6AD2
:103B800075EEC35AF8EEE22A75EEA35A36EE266AAF
:103B9000F4EEE25AF1EE10FA36EE056A05D5FDEEC6
:103BA000E52A12EE903A0FFA83FC02EE905AF8EEF4
:103BB000E22AF4EEE25AF1EE10FA04DDFDEEE55AE7
:103BC00015EE903A1DB205EE901AF8EEE55AB4EEF5
:103BD000E56AF1EE10FA04D5FDEEC65A15EE903AFC
:103BE00019B205EE904AF8EEE55AB4EEE56AF1EE48
:103BF00010FA04DDBDEEC66A16EE103A1CB277EE7E
:103C0000A67A37EE437A06EE90CA37EE237AF8EEBC
:103C1000E66A77EE857AB4EEE67AF1EE10FA05D52B
:103C2000FDEEC76A16EE903A0FFA83FC06EE905A44
:103C3000F8EEE66AB4EEE67AF1EE10FA04DDBDEED7
:103C4000C77A17EE103A1DB207EE101AB8EEC77A0F
:103C5000F4EEC77AF1EE10FA04D5BDEEE77A17EE6E
:103C6000103A19B207EE104AB8EEC77AF4EEC77AE6
:103C7000F1EE10FA04DDFDEEE77A17EE903A1CB291
:103C8000CAEE8ABA731EE1451BB2B8BFE146AE4226
:103C9000D8BF1D468A42B8BF0A460AF1FF331BB29D
:103CA000A245D8BF1C466B1CADF82430631C80EEC7
:103CB0000ABAADF8263008A9002340461646ADF8EA
:103CC0002090ADF822200A9365EE2B7A25EE0B5A50
:103CD000E3EE8B7AABEEE35A74EEE7AA07EE902A96
:103CE00034EE45AAF8EEE77AEBEEA7AAABEE27AAE8
:103CF0000EF05CFCB44234DA0E2019B0BDEC0C8B33
:103D0000BDE8F08F0029BCBFADF8183019468442D9
:103D1000B8BFADF81A40E1E50029BCBFADF81030DE
:103D200019468442B8BFADF812402AE6DFED37CA23
:103D300033E621F08DFFB5EEC00AF1EE10FAB0EED9
:103D400040AA7FF530AE2CE6012302934FF0000B22
:103D500032E6B44684E64D4691E651469EE6144668
:103D6000ABE607EE909AF8EEE77AB0EE6ACAF0EEAC
:103D70004ACAABEE27CACA46EBEEE7CA554506DA91
:103D800001367AEEABAA3AEE0BAA36B2B2E7F8EEFB
:103D9000C87AF4EECC7AF1EE10FA2DD8F8EEC97AA2
:103DA000B4EEE7CAF1EE10FA26D5F8EEE87AF4EEB2
:103DB000EC7AF1EE10FA1FD8F8EEE97AF4EEE7CAE1
:103DC000F1EE10FA18D5FDEEEC7A3846CDED037A17
:103DD000FDEECC7ABDF90C20CDED037ABDF90C10C7
:103DE00046F034FA029A03460AB9834504D03246B3
:103DF000514640460EF0FEFB0AF1010A3CEE0BCAAA
:103E00007CEEEBCA0FFA8AFAB8E700BF00000000A8
:103E10002DE9F04F9DB002AF07F14C030193974B92
:103E2000009307231CF0CAF89549F86C40F2C922A8
:103E30001CF0AAF9BE6D731E012B824605D9042E13
:103E400003D0904831463CF0DDFED7F85480B8F1FD
:103E5000020F05DCB8F1000F14DC8B484146F2E795
:103E6000A8F104031C2BF8D8884A012199400A4084
:103E700042B9142BF1D1012E04D0854818223146C5
:103E80003CF0C0FE3B6DBB6297F85C30FB6297F87C
:103E900060303B6297F86430FB619AF80E30B86A84
:103EA000012101FA03F3013B7B611FF05DFEBAF8CB
:103EB000043078600024A7F8443007F14001BAF8D4
:103EC0000630A7F8463050463C64BC640EF06EFBEA
:103ED000BAF804307C6308FB03F303EBC603F2007B
:103EE000013BB3FBF2F373433B63033323F0030360
:103EF0007B623B6B013323F00103BB617B6A0733B9
:103F000023F00703BB60BAF806907B6B994504DC8D
:103F10000E206C37BD46BDE8F08FBB68C7F810D0E7
:103F2000ADEB030DFB6902AD9BB17B6B09F1FF3972
:103F3000A9EB03090023FB637B683A6B5C68B86AF2
:103F4000294607F13C03A047F96B29B108463CF02C
:103F500009FED7F83490EDE73B6B834202D04D4821
:103F600059F04BF83B6A93B1022E0BD0042E0ED1C0
:103F70007A6A2B46A918994209D01A6812BA43F8EE
:103F8000042BF8E7BA692B465119994210D108F170
:103F9000FF33AB460024FB600FFA89F9BAF804300E
:103FA0009C420ADB7B6BD7F810D001337B63AAE716
:103FB0001A8852BA23F8022BE7E7B8F1080F08DC99
:103FC000FA68072A0ED8DFE802F00F270D360D0D2C
:103FD0000D45B8F1180F42D0B8F1200F4AD0B8F112
:103FE000100F39D0002309E0FA6AE3108AB1E243E6
:103FF00002F00702EB5C134103F001037A6921B27E
:10400000134050464A460EF0F5FA01340BF1030B0B
:10401000C4E704F00702EDE7FA6AA31042B1E243F5
:1040200002F00302EB5C5200134103F00303E5E7E7
:1040300004F00302F6E7FA6A631042B1E24302F0C9
:104040000102EB5C9200134103F00F03D6E704F08A
:104050000102F6E72B5DD1E735F81430CEE79BF887
:1040600001309BF800201B0243EA02439BF8022028
:104070001343C3E755F82430C0E700BFCC2B0A0038
:104080007CC60900153B0900363B090011100010E1
:10409000283B0900305A090073B504460D461E46F8
:1040A0006846084B44F02EFE291D0DF10200064B18
:1040B000324644F027FE6B4603CB20602046616009
:1040C00002B070BDD4290A00CC290A002DE9F04FB6
:1040D0000D4687B00021924629F0A6FA0446002139
:1040E000284629F0A1FA2379662B02D00379662BA2
:1040F00002D1C8483CF07EFD0023039008208DF8D3
:1041000017304DF01DF8074608204DF019F8064607
:1041100008204DF015F80399CDE9006005463B46AF
:104120000DF11702204654F035F8039950B938467E
:1041300013F004FD304613F001FD284613F0FEFC99
:10414000B548D7E70AF1FF3A9DF81700D4F81C905C
:10415000D1F81C802279BAF1030F05D8DFE81AF0F4
:10416000E901BD0398053B08AA46B3462379D4F874
:104170001C90D1F81C80422B40F0C1800A79422A61
:104180003DD1394654F0B3F9C269044600201346C4
:1041900098F800C099F8001001EA0C0103F8011B1F
:1041A000DAF80410D4F810C0DBF804E00391884476
:1041B000991A8C45F144EBD8DBF80010DAF80020AE
:1041C0000CFB1E11894403990CFB11229044E268F8
:1041D0000130904211D3384613F0B0FC304613F052
:1041E000ADFC284613F0AAFC204607B0BDE8F08FCE
:1041F0005A461C46D3469246B8E71A46C7E7622A93
:1042000028D13946682254F072F9C1690446002366
:10421000002298F900C099F8000000EA0C0021F88B
:10422000020B2069DBF804E0DAF804C001328242B4
:10423000F144E044EDD3DBF8002000FB1E22914462
:10424000DAF8002000FB1C229044E268013393421C
:10425000DED3C0E7482A27D1394654F048F9C1696E
:10426000044600230022B8F800C099F8000000EAD4
:104270000C0021F8020B2069DBF804E0DAF804C036
:1042800001328242F144E044EDD3DBF8002000FB30
:104290001E229144DAF8002000FB1C229044E268C0
:1042A00001339342DED396E7682A41F037823946DC
:1042B00054F01DF9C169044600230022B8F800C07B
:1042C00099F8000000EA0C0021F8020B2069DBF8E5
:1042D00004E0DAF804C001328242F144E044EDD354
:1042E000DBF8002000FB1E229144DAF8002000FBDE
:1042F0001C229044E26801339342DED36BE7622BC9
:1043000040F08C800A79622A2CD1394654F0EFF8BB
:10431000C26904460020134698F800C099F80010BE
:1043200001EA0C0103F8011BDAF80410D4F810C0FC
:10433000DBF804E003918844991A6145F144EBD31A
:10434000DBF80010DAF800200CFB1E1189440399F9
:104350000CFB11229044E26801309042BFF43BAF65
:104360001A46D8E7482A27D1394654F0C0F8C1691F
:10437000044600230022B8F800C099F9000000EAC2
:104380000C0021F8020B2069DBF804E0DAF804C025
:1043900001328242F144E044EDD3DBF8002000FB1F
:1043A0001E229144DAF8002000FB1C229044E268AF
:1043B00001339342DED30EE7682A0B4621467FF491
:1043C00017AF394654F093F8C16904460023002220
:1043D000B8F800C099F9000000EA0C0021F8020BBF
:1043E0002069DBF804E0DAF804C001328242F144CB
:1043F000E044EDD3DBF8002000FB1E229144DAF804
:10440000002000FB1C229044E26801339342DED37B
:10441000E1E600BF8B380900CF370900482B57D1A0
:104420000A79482A27D1394654F061F8C16904460F
:1044300000230022B8F800C0B9F8000000EA0C0020
:1044400021F8020B2069DBF804E0DAF804C001323D
:104450008242F144E044EDD3DBF8002000FB1E2251
:104460009144DAF8002000FB1C229044E2680133FA
:104470009342DED3AFE6682A0B4621467FF4B8AEFE
:10448000394654F034F8C169044600230022B8F8D4
:1044900000C0B9F8000000EA0C0021F8020B206906
:1044A000DBF804E0DAF804C001328242F144E0446F
:1044B000EDD3DBF8002000FB1E229144DAF8002047
:1044C00000FB1C229044E26801339342DED382E673
:1044D000682B41F023810A79682A0B4621467FF434
:1044E00087AE394654F003F8C16904460023002220
:1044F000B8F800C0B9F8000000EA0C0021F8020B7F
:104500002069DBF804E0DAF804C001328242F144A9
:10451000E044EDD3DBF8002000FB1E229144DAF8E2
:10452000002000FB1C229044E26801339342DED35A
:1045300051E6AA46B3462379D4F81C90D1F81C80E2
:10454000422B40F0B5800A79422A31D1394653F0E6
:10455000CEFFC26904460020134698F800C099F8BF
:10456000001041EA0C0103F8011BDAF80410D4F83A
:1045700010C0DBF804E003918844991A6145F144C6
:10458000EBD3DBF80010DAF800200CFB1E11894495
:1045900003990CFB11229044E26801309042BFF471
:1045A0001AAE1A46D8E75A461C46D3469246C2E788
:1045B000622A28D13946682253F099FFC16904461E
:1045C0000023002298F900C099F8000040EA0C008E
:1045D00021F8020B2069DBF804E0DAF804C00132AC
:1045E0008242F144E044EDD3DBF8002000FB1E22C0
:1045F0009144DAF8002000FB1C229044E268013369
:104600009342DED3E7E5482A27D1394653F06FFFBE
:10461000C169044600230022B8F800C099F80000E0
:1046200040EA0C0021F8020B2069DBF804E0DAF81C
:1046300004C001328242F144E044EDD3DBF80020B3
:1046400000FB1E229144DAF8002000FB1C2290445B
:10465000E26801339342DED3BDE5682A41F05E8013
:10466000394653F044FFC169044600230022B8F8DC
:1046700000C099F8000040EA0C0021F8020B206904
:10468000DBF804E0DAF804C001328242F144E0448D
:10469000EDD3DBF8002000FB1E229144DAF8002065
:1046A00000FB1C229044E26801339342DED392E582
:1046B000622B40F087800A79622A2CD1394653F068
:1046C00016FFC26904460020134698F800C099F806
:1046D000001041EA0C0103F8011BDAF80410D4F8C9
:1046E00010C0DBF804E003918844991A6145F14455
:1046F000EBD3DBF80010DAF800200CFB1E11894424
:1047000003990CFB11229044E26801309042BFF4FF
:1047100062AD1A46D8E7482A27D1394653F0E7FE5A
:10472000C169044600230022B8F800C099F90000CE
:1047300040EA0C0021F8020B2069DBF804E0DAF80B
:1047400004C001328242F144E044EDD3DBF80020A2
:1047500000FB1E229144DAF8002000FB1C2290444A
:10476000E26801339342DED335E5682A0B462146E1
:104770007FF419AF394653F0BAFEC16904460023ED
:104780000022B8F800C099F9000040EA0C0021F8B6
:10479000020B2069DBF804E0DAF804C0013282423F
:1047A000F144E044EDD3DBF8002000FB1E229144ED
:1047B000DAF8002000FB1C229044E26801339342A7
:1047C000DED308E5482B57D10A79482A27D1394644
:1047D00053F08DFEC169044600230022B8F800C0E2
:1047E000B9F8000040EA0C0021F8020B2069DBF860
:1047F00004E0DAF804C001328242F144E044EDD32F
:10480000DBF8002000FB1E229144DAF8002000FBB8
:104810001C229044E26801339342DED3DBE4682A31
:104820000B4621467FF4BFAE394653F060FEC169A6
:10483000044600230022B8F800C0B9F8000040EA9E
:104840000C0021F8020B2069DBF804E0DAF804C060
:1048500001328242F144E044EDD3DBF8002000FB5A
:104860001E229144DAF8002000FB1C229044E268EA
:1048700001339342DED3AEE4682B40F04F870A79D0
:10488000682A0B4621467FF48EAE394653F02FFE40
:10489000C169044600230022B8F800C0B9F800003E
:1048A00040EA0C0021F8020B2069DBF804E0DAF89A
:1048B00004C001328242F144E044EDD3DBF8002031
:1048C00000FB1E229144DAF8002000FB1C229044D9
:1048D000E26801339342DED37DE4AA46B3462379EE
:1048E000D4F81C90D1F81C80422B40F0B7800A7994
:1048F000422A31D1394653F0FAFDC26904460020FC
:10490000134698F800C099F8001081EA0C0103F8EA
:10491000011BDAF80410D4F810C0DBF804E00391AE
:104920008844991A6145F144EBD3DBF80010DAF8BA
:1049300000200CFB1E11894403990CFB11229044AA
:10494000E26801309042BFF446AC1A46D8E75A46B6
:104950001C46D3469246C2E7622A28D139466822CD
:1049600053F0C5FDC16904460023002298F900C038
:1049700099F8000080EA0C0021F8020B2069DBF8AE
:1049800004E0DAF804C001328242F144E044EDD39D
:10499000DBF8002000FB1E229144DAF8002000FB27
:1049A0001C229044E26801339342DED313E4482A88
:1049B00028D1394653F09BFDC169044600230022EB
:1049C000B8F800C099F8000080EA0C0021F8020B4A
:1049D0002069DBF804E0DAF804C001328242F144D5
:1049E000E044EDD3DBF8002000FB1E229144DAF80E
:1049F000002000FB1C229044E26801339342DED386
:104A0000FFF7E9BB682A40F08986394653F06FFD0D
:104A1000C169044600230022B8F800C099F80000DC
:104A200080EA0C0021F8020B2069DBF804E0DAF8D8
:104A300004C001328242F144E044EDD3DBF80020AF
:104A400000FB1E229144DAF8002000FB1C22904457
:104A5000E26801339342DED3FFF7BDBB622B40F027
:104A600089800A79622A2CD1394653F040FDC26907
:104A700004460020134698F800C099F8001081EA17
:104A80000C0103F8011BDAF80410D4F810C0DBF8AD
:104A900004E003918844991A6145F144EBD3DBF8B3
:104AA0000010DAF800200CFB1E11894403990CFB5E
:104AB00011229044E26801309042BFF48CAB1A4658
:104AC000D8E7482A28D1394653F011FDC169044678
:104AD00000230022B8F800C099F9000080EA0C0019
:104AE00021F8020B2069DBF804E0DAF804C0013297
:104AF0008242F144E044EDD3DBF8002000FB1E22AB
:104B00009144DAF8002000FB1C229044E268013353
:104B10009342DED3FFF75FBB682A0B4621467FF442
:104B200016AF394653F0E3FCC16904460023002266
:104B3000B8F800C099F9000080EA0C0021F8020BD7
:104B40002069DBF804E0DAF804C001328242F14463
:104B5000E044EDD3DBF8002000FB1E229144DAF89C
:104B6000002000FB1C229044E26801339342DED314
:104B7000FFF731BB482B59D10A79482A28D1394649
:104B800053F0B5FCC169044600230022B8F800C008
:104B9000B9F8000080EA0C0021F8020B2069DBF86C
:104BA00004E0DAF804C001328242F144E044EDD37B
:104BB000DBF8002000FB1E229144DAF8002000FB05
:104BC0001C229044E26801339342DED3FFF703BB1B
:104BD000682A0B4621467FF4BAAE394653F087FC6B
:104BE000C169044600230022B8F800C0B9F80000EB
:104BF00080EA0C0021F8020B2069DBF804E0DAF807
:104C000004C001328242F144E044EDD3DBF80020DD
:104C100000FB1E229144DAF8002000FB1C22904485
:104C2000E26801339342DED3FFF7D5BA682B40F038
:104C300075850A79682A0B4621467FF488AE394685
:104C400053F055FCC169044600230022B8F800C0A7
:104C5000B9F8000080EA0C0021F8020B2069DBF8AB
:104C600004E0DAF804C001328242F144E044EDD3BA
:104C7000DBF8002000FB1E229144DAF8002000FB44
:104C80001C229044E26801339342DED3FFF7A3BABB
:104C9000422A40F0A8800B79422B28D1394653F0A4
:104CA00026FCC26904460020134698F800C099F813
:104CB000001001FA0CF103F8011BD4F810C0D6F86B
:104CC00004A0D5F804E0991A6145D144F044ECD32E
:104CD0002A6831680CFB1E229044E26801300CFB0C
:104CE0001A1190428944BFF476AA1A46DCE7622B77
:104CF00027D16822394653F0FAFB0446C0690023E5
:104D0000002298F900C099F8001001FA0CF120F87F
:104D1000021B2169D6F804E0D5F804C001328A42AA
:104D2000F144E044EDD3326801FB1E2291442A682D
:104D300001FB1C229044E26801339342E0D3FFF769
:104D40004ABA482B27D11A46394653F0D0FB0446BD
:104D5000C06900230022B8F800C099F8001001FAD9
:104D60000CF120F8021B2169D6F804E0D5F804C044
:104D700001328A42F144E044EDD3326801FB1E2245
:104D800091442A6801FB1C229044E268013393425B
:104D9000E0D3FFF720BA6822394653F0A8FB044657
:104DA000C06900230022B8F900C099F8001001FA88
:104DB0000CF120F8021B2169D6F804E0D5F804C0F4
:104DC00001328A42F144E044EDD3326801FB1E22F5
:104DD00091442A6801FB1C229044E268013393420B
:104DE000E0D3FFF7F8B9622A40F0A8800B79422B94
:104DF00027D16822394653F07AFB0446C069002364
:104E0000002298F800C099F9001001FA0CF120F87E
:104E1000021B2169D6F804E0D5F804C001328A42A9
:104E2000F144E044EDD3326801FB1E2291442A682C
:104E300001FB1C229044E26801339342E0D3FFF768
:104E4000CAB9622B28D1394653F051FBC2690446D6
:104E50000020134698F900C099F9001001FA0CF1EE
:104E600003F8011BD4F810C0D6F804A0D5F804E06C
:104E7000991A6145D144F044ECD32A6831680CFB9F
:104E80001E229044E26801300CFB1A1190428944C2
:104E9000BFF4A1A91A46DCE7482B27D11A463946A8
:104EA00053F025FB0446C06900230022B8F800C077
:104EB00099F9001001FA0CF120F8021B2169D6F8CB
:104EC00004E0D5F804C001328A42F144E044EDD355
:104ED000326801FB1E2291442A6801FB1C22904487
:104EE000E26801339342E0D3FFF775B9682239468F
:104EF00053F0FDFA0446C06900230022B8F900C04F
:104F000099F9001001FA0CF120F8021B2169D6F87A
:104F100004E0D5F804C001328A42F144E044EDD304
:104F2000326801FB1E2291442A6801FB1C22904436
:104F3000E26801339342E0D3FFF74DB9482A40F0CD
:104F4000A7800B79422B26D1394653F0D0FA04467C
:104F5000C0690023002298F800C0B9F8001001FAD7
:104F60000CF120F8021B2169D6F804E0D5F804C042
:104F700001328A42F144E044EDD3326801FB1E2243
:104F800091442A6801FB1C229044E2680133934259
:104F9000E0D3FFF720B9622B29D11A46394653F0E6
:104FA000A6FAC26904460020134698F900C099F990
:104FB000001001FA0CF103F8011BD4F810C0D6F868
:104FC00004A0D5F804E0991A6145D144F044ECD32B
:104FD0002A6831680CFB1E229044E26801300CFB09
:104FE0001A1190428944BFF4F6A81A46DCE7482B10
:104FF00026D1394653F07BFA0446C06900230022CB
:10500000B8F800C0B9F8001001FA0CF120F8021B42
:105010002169D6F804E0D5F804C001328A42F1448F
:10502000E044EDD3326801FB1E2291442A6801FB63
:105030001C229044E26801339342E0D3FFF7CBB8DF
:105040006822394653F053FA0446C069002300220F
:10505000B8F900C0B9F8001001FA0CF120F8021BF1
:105060002169D6F804E0D5F804C001328A42F1443F
:10507000E044EDD3326801FB1E2291442A6801FB13
:105080001C229044E26801339342E0D3FFF7A3B8B7
:10509000682A40F043830B79422B394625D153F0DF
:1050A00026FA0446C0690023002298F800C0B9F926
:1050B000001001FA0CF120F8021B2169D6F804E077
:1050C000D5F804C001328A42F144E044EDD332689D
:1050D00001FB1E2291442A6801FB1C229044E268D5
:1050E00001339342E0D3FFF776B8622B25D153F01A
:1050F000FEF90446C0690023002298F900C0B9F9FE
:10510000001001FA0CF120F8021B2169D6F804E026
:10511000D5F804C001328A42F144E044EDD332684C
:1051200001FB1E2291442A6801FB1C229044E26884
:1051300001339342E0D3FFF74EB8482B25D153F00B
:10514000D6F90446C06900230022B8F900C0B9F8B6
:10515000001001FA0CF120F8021B2169D6F804E0D6
:10516000D5F804C001328A42F144E044EDD33268FC
:1051700001FB1E2291442A6801FB1C229044E26834
:1051800001339342E0D3FFF726B853F0B0F9044659
:10519000C06900230022B8F900C0B9F9001001FA73
:1051A0000CF120F8021B2169D6F804E0D5F804C000
:1051B00001328A42F144E044EDD3326801FB1E2201
:1051C00091442A6801FB1C229044E2680133934217
:1051D000E0D3FFF700B8422A40F0A8800B79422BB9
:1051E00028D1394653F083F9C2690446002013469A
:1051F00098F800C099F8001041FA0CF103F8011B6F
:10520000D4F810C0D6F804A0D5F804E0991A8C455B
:10521000D144F044ECD82A6831680CFB1E2290443B
:10522000E26801300CFB1A1190428944BEF4D3AFFE
:105230001A46DCE7622B27D16822394653F057F92A
:105240000446C0690023002298F900C099F80010B4
:1052500041FA0CF120F8021B2169D6F804E0D5F8D8
:1052600004C001328A42F144E044EDD3326801FBCC
:105270001E2291442A6801FB1C229044E2680133FB
:105280009342E0D3FEF7A7BF482B27D11A463946F1
:1052900053F02DF90446C06900230022B8F800C07D
:1052A00099F8001041FA0CF120F8021B2169D6F898
:1052B00004E0D5F804C001328A42F144E044EDD361
:1052C000326801FB1E2291442A6801FB1C22904493
:1052D000E26801339342E0D3FEF77DBF682239468E
:1052E00053F005F90446C06900230022B8F900C054
:1052F00099F8001041FA0CF120F8021B2169D6F848
:1053000004E0D5F804C001328A42F144E044EDD310
:10531000326801FB1E2291442A6801FB1C22904442
:10532000E26801339342E0D3FEF755BF622A40F0B2
:10533000A8800B79422B27D16822394653F0D7F841
:105340000446C0690023002298F800C099F90010B3
:1053500041FA0CF120F8021B2169D6F804E0D5F8D7
:1053600004C001328A42F144E044EDD3326801FBCB
:105370001E2291442A6801FB1C229044E2680133FA
:105380009342E0D3FEF727BF622B28D1394653F072
:10539000AEF8C26904460020134698F900C099F996
:1053A000001041FA0CF103F8011BD4F810C0D6F834
:1053B00004A0D5F804E0991A8C45D144F044ECD807
:1053C0002A6831680CFB1E229044E26801300CFB15
:1053D0001A1190428944BEF4FEAE1A46DCE7482B0F
:1053E00027D11A46394653F082F80446C069002393
:1053F0000022B8F800C099F9001041FA0CF120F829
:10540000021B2169D6F804E0D5F804C001328A42B3
:10541000F144E044EDD3326801FB1E2291442A6836
:1054200001FB1C229044E26801339342E0D3FEF773
:10543000D2BE6822394653F05AF80446C0690023A8
:105440000022B8F900C099F9001041FA0CF120F8D7
:10545000021B2169D6F804E0D5F804C001328A4263
:10546000F144E044EDD3326801FB1E2291442A68E6
:1054700001FB1C229044E26801339342E0D3FEF723
:10548000AABE482A40F0A7800B79422B26D1394684
:1054900053F02DF80446C0690023002298F800C09C
:1054A000B9F8001041FA0CF120F8021B2169D6F876
:1054B00004E0D5F804C001328A42F144E044EDD35F
:1054C000326801FB1E2291442A6801FB1C22904491
:1054D000E26801339342E0D3FEF77DBE622B29D10F
:1054E0001A46394653F003F8C269044600201346B1
:1054F00098F900C099F9001041FA0CF103F8011B6A
:10550000D4F810C0D6F804A0D5F804E0991A8C4558
:10551000D144F044ECD82A6831680CFB1E22904438
:10552000E26801300CFB1A1190428944BEF453AE7C
:105530001A46DCE7482B26D1394652F0D8FF0446FC
:10554000C06900230022B8F800C0B9F8001041FA81
:105550000CF120F8021B2169D6F804E0D5F804C04C
:1055600001328A42F144E044EDD3326801FB1E224D
:1055700091442A6801FB1C229044E2680133934263
:10558000E0D3FEF728BE6822394652F0B0FF044649
:10559000C06900230022B8F900C0B9F8001041FA30
:1055A0000CF120F8021B2169D6F804E0D5F804C0FC
:1055B00001328A42F144E044EDD3326801FB1E22FD
:1055C00091442A6801FB1C229044E2680133934213
:1055D000E0D3FEF700BE682A40F0A0800B79422B92
:1055E000394625D152F083FF0446C06900230022CA
:1055F00098F800C0B9F9001041FA0CF120F8021B2C
:105600002169D6F804E0D5F804C001328A42F14499
:10561000E044EDD3326801FB1E2291442A6801FB6D
:105620001C229044E26801339342E0D3FEF7D3BDDD
:10563000622B25D152F05BFF0446C0690023002293
:1056400098F900C0B9F9001041FA0CF120F8021BDA
:105650002169D6F804E0D5F804C001328A42F14449
:10566000E044EDD3326801FB1E2291442A6801FB1D
:105670001C229044E26801339342E0D3FEF7ABBDB5
:10568000482B25D152F033FF0446C0690023002285
:10569000B8F900C0B9F8001041FA0CF120F8021B6B
:1056A0002169D6F804E0D5F804C001328A42F144F9
:1056B000E044EDD3326801FB1E2291442A6801FBCD
:1056C0001C229044E26801339342E0D3FEF783BD8D
:1056D00052F00DFF0446C06900230022B8F900C053
:1056E000B9F9001041FA0CF120F8021B2169D6F833
:1056F00004E0D5F804C001328A42F144E044EDD31D
:10570000326801FB1E2291442A6801FB1C2290444E
:10571000E26801339342E0D3FEF75DBD0024FEF75B
:105720005ABD00BF38B50C4BD3F8B43004460D4613
:1057300043B90C204BF004FD2A462146BDE8384011
:1057400000F00CB89A68A24202D15A68AA4201D06D
:105750001B68EDE738BD00BFF462012070B5094C4D
:10576000D4F8B4502B462BB9C0E900528160C4F87C
:10577000B40070BD9E688E4202D15E689642F8D039
:105780001B68F0E7F462012030B5094A52F8B43FD3
:105790004BB19C6884421C6806D15D688D4203D180
:1057A000146000221A6030BD1A462346F0E700BF9D
:1057B000F4620120044B1B7823B1044843680BB109
:1057C00044F0F6BB184670475D6D0120F04F012094
:1057D00008B50348012104F07DFC0E2008BD00BF80
:1057E0008851012070B52DED028B8EB006AB019370
:1057F000574B00930431022301381AF0DFFB4FF4BA
:105800002272544906981AF0BFFC40F20A6104461D
:105810009FED510A07981AF0A5FC204604A9B0EEA6
:10582000408A42F055F80E2200210AA84BF0B8FD3C
:10583000DFED4A7A9FED4A7A4A4B4B4A0A9328EEAB
:10584000278AA023C8EE077AADF82C30106851687B
:10585000B6EE007A77EE877AFCEEE77A17EE903AAA
:10586000ADF82E3008AB03C3404803A9FFF75AFF39
:1058700000238DF80E3008AA01230AA904A854F0C9
:10588000B7FC044630B1394803A9FFF77DFF204635
:1058900044F08BF89DF80E3063B1344803A9FFF74C
:1058A00073FFBDF80C604FF6FF739E4205D1304880
:1058B00023F0BEFCFBF7B4F9ECE700202AF0BEF9B8
:1058C0000446B8B16378012B36D12378DB0733D592
:1058D00006220DF1110104F151004BF00CFD58BBF3
:1058E00004F1240204F13601304654F08FFCB0FA82
:1058F00080F46409002502A93046ADF8085054F040
:1059000089FC4FF40071304654F09AFC44F04DF895
:1059100029462A46304654F06FFC44F046F8154BB1
:10592000882101FB05F2D0189A5AB24206D00135FF
:10593000052DF6D11048BBE72046BFE70123837051
:1059400080F85A4000F066FD0EB0BDEC028B70BDD1
:1059500044230A00B4B40900000000000024744984
:1059600000401C460001A00070E008002BC50700A5
:10597000DE4B0900A0090120E64B09002DE9F041AA
:105980000746806986B0F0B9104D044606464FF6CA
:10599000FF782B8843450CD0E86D0E2803D12846AC
:1059A00000F038FDE86506AB03EB8403013443F8EF
:1059B000140C0136052E05F18805EAD101A920460F
:1059C00021F080FBB86106B0BDE8F081A00901209C
:1059D00008B501483BF0B2F84C4E090007B50A790A
:1059E0009DF8003062F347038DF80030D1F80530A0
:1059F000CDF801306846B1F80930ADF8053054F003
:105A0000E7FB10B1024823F013FC0E2003B000BDE9
:105A1000414D09002DE9F04F2DED028B95B00CABF7
:105A200051F8044B01935F4B0093013808231AF09F
:105A3000C5FA0C98052209A91EF044F80D98002318
:105A40000E28CDE90633089303D0052206A91EF0DF
:105A500039F8119808B95448119040F223411AF0CE
:105A6000A9FBDFED527AB4EEE70AF1EE10FAB0EEE0
:105A7000408A06D4DFED4E7AB4EEE70AF1EE10FA72
:105A800004DD4C4A4C494D483BF0BCF8DDF840A0E1
:105A9000BAF1000F04DA40F20A6100201AF020FB8C
:105AA0000A9B9DF838601F2B05D926B1079B13B1BF
:105AB000434823F0BDFB13980E280DD00EB9414882
:105AC000F7E7414940F265321AF05EFB074694F869
:105AD00044301BB13D48ECE70027F8E7E3689DF848
:105AE0003C80DDF8489013B1204604F061FC0A9D2B
:105AF0003146284603F0ACFBDDF81CB03146584671
:105B000003F0A6FB1F2D04D9BBF1000F02D03048D3
:105B1000CFE715B10FB12F48CBE7B8F1000F09D18E
:105B20002D4B2E4A03FB0AF3934205D92C48B4218E
:105B300023F07EFB4FF0B40A616819B9FF2011F021
:105B400033FC6060A16819B9FF2011F02DFCA06042
:105B5000DDE9091260684BF0E2FBDDE90612A0689E
:105B60004BF0DDFBCDE90497BDF81C300393A3682F
:105B70000293BDF82830019363680093B0EE480AA1
:105B80005346424631462046F4F732FD43F00DFFBE
:105B900040F201130E20A4F8443015B0BDEC028B86
:105BA000BDE8F08F44220A00CECC4CBE0AD7A33CFD
:105BB0000AD72341072109000D210900513B0900A3
:105BC000124E09005C480900B4B40900A64F090050
:105BD0001A4C0900074D090040420F000FBCBA0AD9
:105BE000804509002DE9F04F2DED068B93B00AABEF
:105BF00051F8044B0193834B0093013808231AF0AA
:105C0000DDF90D980E2828D09FED7F0A40F20A6139
:105C10001AF0A8FAF0EE408A0E9808B97B480E9068
:105C20000F9B0BB9794B0F9340F223411AF0C2FA44
:105C3000DFED777AB4EEE70AF1EE10FAB0EE408AC3
:105C400006D4DFED747AB4EEE70AF1EE10FA07DD60
:105C5000714A724972483AF0D5FFDFED6B8ADBE793
:105C6000F5EE408AF1EE10FA07D0F4EEC08AF1EEBC
:105C700010FA02D56B483AF0BDFF0F9840F26C6104
:105C80001AF098FAB4EEC08AF1EE10FAB0EE409A2B
:105C900001D56548EFE70A980023049358B105221F
:105CA00003A91DF00FFF049B2BB1039812F0FEF81F
:105CB00008B95E48DFE70B9F002F04DC40F2E621C5
:105CC00001201AF00DFA23699DF83050DDF840905C
:105CD0009DF84480DDE903BA3BB193F8293013B94C
:105CE000534823F0A5FA00232361E36843B16268B7
:105CF000934202D1112003F07FFB204604F058FBB1
:105D00004C499FED4DAA2C204DF008F83946064627
:105D1000083054F0CCF8002DC6E907BAC6F8249034
:105D200026610CBF1F26FF2606F108004BF026FA5D
:105D30002369586000F1080303608680074601204C
:105D400042F002F943F031FE21693C48FFF7EAFCDA
:105D500068EE8A6A9FED3A7AC6EE877AF6EE009A86
:105D600077EEA97AFCEEE77A17EE906AB6F5803FF7
:105D700001D334487FE736B9F5EEC08AF1EE10FA68
:105D800001DD314877E70E22002106A84BF008FB21
:105D900028EE0A8A9FED2D7AADF81E60C8EE077ACC
:105DA00045F4807545EA880525F0FA05394606A8C8
:105DB000ADF8185029EE0A9A77EEA97AFCEEE77A48
:105DC00017EE903AC9EE077AADF81A3077EEA97A55
:105DD000FCEEE77A17EE903AADF81C3054F022FA58
:105DE000054640B115482169FFF7CEFC0023236129
:105DF000284643F0DAFD206913B0BDEC068BBDE800
:105E0000F08F00BF84220A0000000000CECC4CBE00
:105E10000AD7233B66D62342122109001C21090020
:105E2000513B0900AA38090070330900C247090034
:105E3000EA460900DCB3090000247449597E0600D3
:105E400000401C462D350900BA38090000401C44AA
:105E5000022808B50B46114613D18A0713D10868EA
:105E60000A4A90420FD118790A7990420BD1062242
:105E70000531581D4BF03FFA00280CBF3E201E2074
:105E800008BD0020FCE71E20FAE700BFB4B40900FB
:105E900010B588B0084611461A4603AB0193134B60
:105EA000009302234BF0D5FB05A9039805221DF0B2
:105EB00009FE06984FF4227206211AF023F904987D
:105EC00040F28B23032200214BF0F6FB08490446E5
:105ED0000C204CF023FF059B1A68C0F805209B8816
:105EE000A0F80930047108B010BD00BF34230A00C7
:105EF000B4B409001FB54B7903938B790293CB7926
:105F000001930B7A00934B7A8A7A02494DF01EF97D
:105F100005B000BD232109002DE9F04F97B00DAB6E
:105F20000193344B00930431092301381AF046F8E9
:105F300031490D9840F28D521AF026F92F490890F8
:105F400040F24E620E981AF01FF99DF83C603F2E09
:105F5000834603D940F2FB401AF022F89DF84070C6
:105F6000384644F013F89DF84480404644F00EF85B
:105F7000129C002C04DA40F26E4100201AF0B0F8B6
:105F800014989DF84C500E2804D15DB354B32046AC
:105F90004CF0EFFE0DF12809052249461DF092FD57
:105FA0000B9840F217422146F5B11AF0ABF815985C
:105FB0000E281CD021F0D6FF8246114928204CF033
:105FC000ADFECDE9059ACDE90345CDE90178089903
:105FD00000965B460022099004F052FA099817B027
:105FE000BDE8F08F0748D5E71AF098F8DFE74FF0E3
:105FF000000AE2E7EC220A00BCB3090094B30900EE
:1060000068B40900A462090010B54368044653B19E
:1060100001460648FFF7B8FB0023C4E90333C4E98F
:106020000633636063610E2010BD00BF59980700FE
:1060300070B52DED028B86B0084611461A4603ABAB
:1060400001931F4B009303234BF003FB1D4903985F
:106050004FF43F721AF098F840F20A610646B7EE24
:10606000000A04981AF07EF8059D002DB0EE408AD3
:1060700004DC40F2E62101201AF032F81249242013
:106080004CF04CFE044628464BF078F8DFED0F7AD2
:10609000666028EE278A0023BCEEC88AC4E903059F
:1060A000C4E905330A4884ED028A84F82030E361AC
:1060B0002146FFF737FB204606B0BDEC028B70BDD2
:1060C000C4220A0068B4090044B4090000007A44FC
:1060D0005998070008B501483AF030FDC24D090053
:1060E00010B50446808A43F03BFCE3692BB1BDE860
:1060F0001040D3E9020120F0E5BF014810BD00BF08
:106100007C31090070B58B6804460D4616466BB1AC
:1061100007494DF01BF8A9682046324600F082FE80
:1061200004492046BDE870404DF010B80249F9E737
:106130004B210900352209005B210900F0B50C460E
:1061400085B054F8045B0646A88A174643F008FC5D
:1061500002AB0193084B00933A4602232146701E7E
:1061600019F02CFF28469DF80C209DF8081004F02B
:10617000C9FA0E2005B0F0BDDC220A0008B50148BE
:106180003AF0C0FCD1480900084930B50022882502
:1061900005FB02F463180C5B844204D00132052A2B
:1061A000F6D1002030BD1846FCE700BFA009012051
:1061B0002DE9F04F8BB004AB51F8048B0193784B71
:1061C00000930138012319F0F9FED8F80440204665
:1061D00000F0F6F87348049D2146FFF7A3FA00206B
:1061E00017F010FB0E2D606030D101210AE06268CB
:1061F0009368D26803F18043013B52F82330D98A77
:10620000013189B2002220460BF06CFF0028EED14C
:10621000654F002663689A68964236D321466148E6
:10622000FFF7B2FAD8F80440204600F0C9F86368D6
:10623000D3E9020120F046FFD8F80430044658683C
:106240004CF002FD20460BB0BDE8F08F284606A9B1
:106250001DF0A4FC554E054628461DF063FE00289F
:10626000D6D0830702D10368B34202D050483AF037
:10627000ADFC8388ADF8143005AA83798DF816300B
:10628000012120460BF02EFFE6E7DB6853F826508D
:10629000AB680BB90136BDE7AB8ADFF81C91EA8A1F
:1062A0009A4212D3ADF81830DFF810A1C9F80050A7
:1062B0000023ADF81A203B702088012306A98AF834
:1062C000003053F0B9FF00283DD02B699B68029342
:1062D0000023029A9A42DDD02A69D1685A1C03929F
:1062E000029A51F823B0501E834216BF01EB83017E
:1062F00000234B68DBF8081009B3BBF81410013118
:1063000089B2002B32D09B8A013B1FFA83F9E88ABD
:10631000884214D3494512D8264BADF81810DFF83F
:106320009CA0C3F800B000213970ADF81A9001218B
:106330008AF80010208806A953F080FFD8B1039B8B
:10634000C7E7FAF76DFC9AF80030002BF9D13B78DB
:10635000002BBAD02A699368D26803F18043013BCD
:1063600052F823309B8A01339BB298E7B5F8169018
:10637000CDE7FAF755FC9AF800100029F9D13978E1
:106380000029DCD0DBF81C008168C06801F1804185
:10639000013950F82110898A013189B2B7E700BF6D
:1063A0008C230A0025210400E86E012094B3090023
:1063B000E2380900D4620120D0620120E76E01209A
:1063C00008B543F005FE10B901483AF09BFB08BD43
:1063D000714D090038B544680D4D2046FFF7F0FFB8
:1063E00094F874306BB9B4F86C3000EE103AB8EE33
:1063F000C00AF7EE047ABDE8384020EE270A20F004
:10640000D5BCAB6A002BEED1FAF70AFCE8E700BF77
:10641000F462012010B50446C06D0E2805D1034971
:106420000C204CF07BFC4460E06510BD84B4090096
:1064300030B585B003AB51F8044B0193224B009368
:106440000138012319F0BAFD9DF80C3033B91F480B
:106450004FF4A67240F2DD213AF078FB64681C4DDF
:106460002046FFF7ADFF94F85A30012B01D1AB6AFB
:10647000EBB194F85A30022B22D00123154984F84D
:106480005A302088124D53F0ADFE43F08EFA94F846
:106490005A30012B01D1AB6A63B1AB6A83B994F86E
:1064A0005B1069B1882908D10B4822F0CFFEFAF7BA
:1064B000B7FBD8E7FAF7B4FBE9E7084822F0C6FED5
:1064C0000E2005B030BD00BF94230A000251090020
:1064D000F4620120E8200A00114409006C4409001C
:1064E0002DE9F04796B00FAB01935B4B009304315D
:1064F0000723013819F062FD58490F984FF43F7295
:1065000019F042FE564940F24E620746109819F0C3
:106510003BFE9DF844908246484643F037FD9DF887
:106520004880404643F032FD139E002E04DA40F2CC
:106530006E41002019F0D4FD15989DF850500E289A
:1065400004D14DB346B330464CF013FC052204A9E8
:106550001DF0B8FA059840F217423146F5B119F02E
:10656000D1FD404918204CF0D9FBC0E9017A002345
:106570000446838280F8169080F81780DDE90401D4
:1065800020F068FBE060002D5CD1B6F5007F08DDEF
:10659000354A4FF400715BE03448D7E719F0BEFD8F
:1065A000DFE72682A574FB69002B47D0A368A17D95
:1065B0009A889B798DF80E3085F001050DF1080859
:1065C00045F002050026404605F00705ADF80C2011
:1065D000ADF808608DF80A5042F02DFCE17D0DF118
:1065E000090042F028FC052207A9E0681DF06AFABC
:1065F00003ABCDE90A38089BADF83030238AADF8FB
:10660000343004F11402079BB88A0E930AA9ADF83E
:10661000326053F025FE43F0C8F9154AA18A138869
:10662000F8698B4228BF0B461380124A13888B42AD
:1066300038BF0B46214613804CF0E3FA204616B0D3
:10664000BDE8F087B6F5FF7FABDD0B4A4FF4FF7175
:106650000A483AF0D7FA00BF54230A0068B4090088
:1066600094B3090028B4090015E10800A4620900E8
:10667000A0050120D06A012020E108002D3A090080
:1066800070B58B6804460D4616466BB107494CF051
:106690005DFDA9682046324600F0C4FB044920464F
:1066A000BDE870404CF052BD0249F9E78321090072
:1066B000352209008F2109007FB5044605220846CE
:1066C00001A91DF0FFF9A58A65B163685E68F068ED
:1066D00042F084FCB37901463BB1002301AA28466D
:1066E00042F000FD0E2004B070BDA07C029B228A07
:1066F00020B19A4206D006483AF07CFA9A4201D27A
:106700000448F9E701AA284642F013FDEAE700BF72
:10671000CF430900C4430900022A70B504460E465F
:1067200015460BD140F2722052F031FF014620464F
:106730004CF0FDFC054920464CF0F9FC2A46314658
:106740002046BDE870401EF09FBF00BF0AE1080070
:1067500070B5064686B008460D46144642F02EFC3B
:1067600000234FF400722048019401A9CDE90223CF
:10677000ADF810508DF81430FEF7D4FF00223146EA
:10678000284653F063FD11280446F7D030B116486F
:1067900001A9FEF7F9FF204643F007F99DF81430F0
:1067A000B3B1BDF8100042F009FC01A90E48FEF794
:1067B000EBFFBDF8121089B291B140F20513994276
:1067C00009D040F20F13994208D0084822F030FD5A
:1067D000FAF726FAE2E7064822F038FD0548FBE71B
:1067E000039806B070BD00BF0D7907008144090011
:1067F0001D4B0900144B090008B501483AF0FAF99D
:10680000684909002DE9F04788B0084611461A4644
:1068100005AB01932D4B009303234AF01AFF2C493B
:1068200005984FF43F7219F0AFFC069D002D074606
:1068300004DC40F2E621012019F052FC07980E28F2
:1068400036D17E8A234930204CF068FA40F2FD139D
:106850009E4228BF1E467B68BA7D9B7902F03004B9
:10686000804602F0060213B9134622461C4642B384
:1068700006F1020905FB09F948464AF07FFC054686
:1068800014B330464AF07AFC824630464AF076FC31
:1068900004460023CDE902634046CDE900A44B46FF
:1068A0002A463946F3F790FF404608B0BDE8F08726
:1068B0004FF48E6119F096FC061EC3DC4FF48E6116
:1068C000B9E715469146DBE7A246E2E7CC230A008A
:1068D00068B409000CB4090030B50D4685B0044613
:1068E000406843F038F8062201A928461DF0EAF86E
:1068F000DDE90112204643F0B7FB002803DA4142EC
:1069000003483AF07FF9400040F0010005B030BD87
:10691000D34E090010B58AB002AB0C460193144B5C
:10692000009304310223013819F048FB24686068A1
:1069300043F011F80298052207A91DF0C3F8039847
:1069400000230E28059303D0052204A91DF0BAF8F0
:10695000059B0093DDE90712049B204603F0B8FF76
:1069600020EAE070400040F001000AB010BD00BF16
:10697000BC230A002DE9F041494D4A4B2B6043F0FE
:10698000E6FA002800F08980474B1A78002A00F0C8
:10699000848000221A70454B1A781AB9444A12783A
:1069A000012A2DD1434800241C7003F05FFF424BA5
:1069B0009A8A02B19C82414B9A8A0AB100229A8239
:1069C0003F4C6368BBB13F4B1B78A3B1204603F03B
:1069D00067FF204603F04AFF3B4B9A8A0AB1002228
:1069E0009A823A4B9A8A0AB100229A82384B9A8A42
:1069F0000AB100229A82374B9A8A0AB100229A82FF
:106A0000274803F0F3FCEB6813B1254803F0D0FCF2
:106A10000024AC61304D4FF6FF782E460E272888B3
:106A2000404502D0132153F0EFFB0134052CEF65F4
:106A300005F18805F3D154F0BAFF4FF6FF7704460D
:106A40000D4600231A4636F813104433B94218BFD6
:106A500042F00102B3F5AA7FF5D142B154F0A7FF8D
:106A6000001B61EB0501802871F10001E9D30C489E
:106A7000002103F02FFB4FF42A23184A1B6893428E
:106A800005D14FF43122D2F8FC2F9A4201D000F008
:106A90007BFBBDE8F04135F07DBEBDE8F08100BF75
:106AA00088510120DCB409002C6E0120306E0120D9
:106AB000196F012018500120206801205068012022
:106AC000485001205D6D012050670120A067012022
:106AD000D0670120E85B0120A00901203130444249
:106AE00030B589B003AB51F8045B01930E4B0093B2
:106AF0000138022319F062FA9DF81040039805A9A5
:106B000005221CF0DFFF84F00104E8680094DDE951
:106B10000523D0E9021042F050FB00280CBF1E20D4
:106B20003E2009B030BD00BFAC230A007FB5084647
:106B300011461A4602AB0193114B009302234AF00F
:106B400088FD40F24E6202980E4919F01DFB0E4975
:106B50009DF80C60054618204CF0E7F8044600202C
:106B600016F050FE3246034629462046F3F792FEC1
:106B700042F01BFF054B012220461A7004B070BD85
:106B80009C230A0094B30900BCB309002C6E0120B9
:106B900070B58B6804460D4616466BB107494CF03C
:106BA000D5FAA9682046324600F03CF9044920464F
:106BB000BDE870404CF0CABA0249F9E7B3210900B8
:106BC00035220900BC21090008B5014839F0B6FF9B
:106BD0005547090010B5022888B00B46144624D149
:106BE000A20720D12168124A91421CD19A79012A28
:106BF00009D1A279012A06D19A88A3889A4212D192
:106C00003E2008B010BD1846694643F074FA04A946
:106C1000204643F070FA10220DEB020168464AF05C
:106C20006AFB0028ECD01E20EBE70020E9E700BF5C
:106C300094B3090008B58B7813B9044822F0F8FA28
:106C40000B8883808B78837108BD00BF8B4409005B
:106C50001FB58379012B02D1054839F04BFF6946F6
:106C600043F049FA102168461FF0F4FF05B000BD5B
:106C70009D380900F0B51C4608468FB011464FF00C
:106C8000021219F063F92068C20706D410F003035A
:106C900017D10168414A914213D14BF06CFCA223F9
:106CA0004FF6FF7200214AF007FD3D4905460820D6
:106CB0004CF034F8012304468580837120460FB0E0
:106CC000F0BD384A0240062A05D0002B4DD102689B
:106CD000354B9A4249D101A921F01CF9019B242B83
:106CE00002D0324839F086FF037A2D2BF9D1437B4D
:106CF0002D2BF6D1837C2D2BF3D1C37D2D2BF0D101
:106D0000461E00F12304002516F8017F384639F0AD
:106D1000D1FE28B105F138036B44013503F8207C1E
:106D2000B442F1D1202DDCD106AD0F2402AE28787B
:106D300056F05BF90746687856F057F940EA0710B5
:106D4000A055013C631C05F10205F0D10023144954
:106D5000BDF81450ADF8143008204BF0DFFF02A945
:106D60008580044643F0B1F9A8E7012206A91CF08A
:106D7000A9FE08B90E48B5E70798A222102119F01C
:106D8000C1F9069B02AC03F1100518685968224648
:106D900003C20833AB421446F7D1D7E7C03209002B
:106DA00094B309000F0080FF34310900ED4409005D
:106DB000DE440900F0B589B003AB51F8044B0193F0
:106DC000174B00930138022319F0F8F8062205A9A1
:106DD00003981CF077FE069F0498002140F2B4430C
:106DE0003A464AF069FCA679012E14BF8021102191
:106DF0000546C90840F2E522381A4AF069FC059BAD
:106E0000012E03EB050107D1A2885A55A3881B0A5E
:106E10004B700E2009B0F0BD204643F06CF9F8E746
:106E20006C240A0010B58A79012A92B0044606D172
:106E30008A881F4912B0BDE810404CF087B9084657
:106E40000EA943F058F99DF838300D939DF839306C
:106E50000C939DF83A300B939DF83B300A939DF8C4
:106E60003C3009939DF83D3008939DF83E300793E0
:106E70009DF83F3006939DF8403005939DF84130D2
:106E800004939DF8423003939DF8433002939DF89C
:106E9000443001939DF8453000939DF847209DF8BC
:106EA0004630044920464CF051F912B010BD00BFE5
:106EB000DD210900EA2109002DE9F0472DED048BC1
:106EC00084B002AB0193344B0093022319F076F89F
:106ED000039C0E2C04D14FF480504BF03CFF044631
:106EE0000221204649F01DFA074660B920461EF0EF
:106EF00039FFC3880093294840F257232E2240F2DD
:106F0000F75139F06BFEDDF808809FED258ADFED43
:106F1000258A002507EE905AB8EEE70A07EB851997
:106F200020EE080A1FF042FF00268246B7EE009AC4
:106F300007EE906AB8EEE70A20EE080A1FF036FF67
:106F40005146024640464AF0C3FC1EF081FEB5EEB3
:106F5000C00AF1EE10FA1AD4B4EEC90AF1EE10FA32
:106F600017DC20EE280A30F077FAFCEEC07A17EE34
:106F7000903A09F806300136402ED9D10135402D1E
:106F8000C8D1204604B0BDEC048BBDE8F0870023D7
:106F9000EFE70123EDE700BF042A0A006C51090066
:106FA0002108823C00007C422DE9F04F754C85B0F1
:106FB000002600AFA4F108084FF0880909FB0683FA
:106FC00093F87830002B65D054F0F1FCD4E91E23FF
:106FD000801A61EB0301B0F57A7F71F1000159D39A
:106FE000002134F8080CF9800323BA1D6D4653F0D4
:106FF00045F9002847D1FB8834F8080C0733DB0833
:10700000A5EBC3039D46BA1D03236946EA4653F028
:1070100035F9002837D1B4F8502014F8060C0221B5
:1070200048F0A2FE834660B1FB88C2889A4205D12F
:1070300000F1080168464AF05EF920B3584649F06D
:1070400041FC00233B7214F8063C3A89F888F88129
:1070500043F4007302F0FE0223F0FE0313433B816E
:10706000B4F850307B8134F8083CBB810FF04EF906
:107070000222834607F1080131F05AF8FA88514696
:10708000584656F029FD882303FB06830022AD46AF
:1070900083F8782009FB068393F87930002B41D0E0
:1070A00014F8060C002847D0B4F82EA0524601214F
:1070B00048F05AFE054650B1C288502A04D12146F4
:1070C00008304AF018F940B3284649F0FBFB00208D
:1070D00028F0B4FD054690BB387214F8063C3A8996
:1070E000A7F80AA043F4807302F0FE0223F0FE0327
:1070F000134350253B81284634F8083CBB81FD8171
:107100000FF004F90222824607F1080131F010F86D
:107110002A462146504656F0DFFC09FB0683002232
:1071200083F879200136052E04F188047FF446AFF8
:107130001437BD46BDE8F08FB4F812A0B6E76B78FF
:10714000012B1DD12B7814F8062C03F001039A4271
:1071500016D1B5F806B0BBF1500F11D1062204F1DB
:10716000490105F151004AF0C6F848B95A4621468E
:1071700005F108004AF0BFF810B1284649F0A2FB1B
:107180002846A5E7A809012073B5104D4FF42A241D
:107190004FF00106200B2E7053F08CF808B930F038
:1071A000B7FF04F58054B4F5322FF3D1084B0193A7
:1071B00001A901224FF42A2030F0BAFF054801222C
:1071C00001A930F0B5FF02B070BD00BFFE6E012016
:1071D00031304442FC1F0B00032A05D11E2914BF85
:1071E000044905494BF0A3BF1E2914BF03490449B4
:1071F000F8E700BFB9E00800BEE0080020E10800A1
:1072000015E1080030B587B00C460592D1E901239D
:10721000174904935528CDE90212236809D054F880
:10722000042C02A9184620F0C1FFA4F1080007B001
:1072300030BD184600931EF095FD827B009B82B105
:1072400000EB820002A90569019318460422A847B1
:107250000090F6F721F8DDE9000310B12060204628
:10726000E5E718464BF093F90146024839F0B6FCC1
:10727000885C0900915009002DE9F04F2DED028B3B
:10728000B9B00AAF084611461A4607F150030193F8
:10729000BA4B00931A234AF0DCF93B6D786D3B60E2
:1072A000052207F144011CF00DFC40F2BA21D7F889
:1072B000900056F085F8F863D7F898001EF0C8FCE7
:1072C000D7F868B05A229BFBF2F302FB13B3B0EE7F
:1072D000408A13B1AA4839F08DFC97F8B0A0FE6E31
:1072E000BAF1000F08D0012E06D0A64840F21A22AB
:1072F0004FF4447139F086FCF5F766F9A24B036050
:1073000097F88450B7F960307D6297F888503B63F6
:107310003D62B7F9643097F88C50FB62FD6197F8D5
:1073200070307D6C7B63BD6197F8A030BD6C7D6172
:107330000446B7F8945097F87400FB6097F8A430AF
:1073400097F87CC097F880E0B7F85810B7F85C2041
:10735000D7F8A890B8623D6197F8780097F89C50EC
:10736000BB6397F8AC30BB604FF00008D7F8B4307F
:107370007B6084F8B380CDE904CE0390BB6A0293AE
:107380007B6BB6B2CDE9006304F108001FFA8BF302
:1073900046F0CFFA04F150037B63012E14BF0023A3
:1073A0000AF00103CDE90783CDF82480FB6806933A
:1073B0004FF48073CDE904333B6A03937B6A0293F5
:1073C000FB6A01933B6B0093C5F58075ABB21A461F
:1073D000396804F150000BF0BFF9FB6984F8B23052
:1073E0003B69A4F8AC30BB6BA4F8AE9083F001030A
:1073F00084F8B430BB6884F8B5301FFA89F94FF4CB
:107400007A73B3FBF9F3A4F8B030BB8AFB62C346CE
:10741000FB6A9B4537D35D4BC4F88430FB6BD3B11B
:10742000187943F08DF9B0B100220092BB88F96B56
:1074300004F1840005F078F9002800F08B80544BAB
:10744000C4F88430F96B04F1840042F0B6FEFB6BA3
:10745000187943F08AF9B0EE480A204603F0B6FAEC
:107460004C4991F82A309B0702D4204642F062FE34
:10747000B96B204642F04AFE2046BC37BD46BDEC03
:10748000028BBDE8F08FBB6903EB0B0898F8015045
:10749000786B0BF053F900283AD094F880906BB2D7
:1074A0003B6305F07F05B9F1000F3CD005F10803FF
:1074B00003F0F803E946ADEB030D98F800208DF8D2
:1074C00028200AAB6E1C2A4608F102010DF12900A2
:1074D000BB6249F024FF0096266EBB6A206D012234
:1074E0000021B047CD46786B46F09EF83B6B002BF1
:1074F0002DDA6E1C023518F80500FF2808BF4FF47E
:10750000FA701CF09BFB0BF1020306EB030B7FE709
:10751000F9F786FB204B9B6A002BB9D01F4840F23D
:107520006F3139F03DFB01230093B5EB0902206D6B
:10753000266E434618BF01224946B0470095206D8C
:10754000266E08F102034A460121B047CBE72E46DA
:107550000A20D6E7124BD4F88800C4F884302DF006
:107560004DFF94F88C200F4902F07F0201239340D5
:107570000A5C13430B54D4F8903069E7142D0A00C9
:10758000A04C0900B9510900B4C709005C640900A6
:10759000F4C6090044010120F4620120EC51090005
:1075A00058C00900EB6E0120F0B58DB002AF07F1B5
:1075B00008030C460193264B009304310223013843
:1075C00018F0FCFC206823F037FBD7E9026504467D
:1075D000062207F11C0128461CF074FA94F83A3090
:1075E000102B02D01B4839F005FBA28E386ABA82F4
:1075F00002F00103002103EB52033961B0EB830F6A
:107600007E8206F10106B961FE821ED35209013263
:107610007A607A68FB699200073222F00702ADEBCC
:10762000020D02AA8C467E6888B2864209D807F10C
:10763000100104F1080046F0B2F928462C37BD4687
:10764000F0BD42F820C00131EDE70348CBE700BFB1
:107650007C2E0A00B24C0900CB4E090008B5014847
:1076600039F096FAF44E09007FB502AB0C4601934F
:107670002B4B009304310223013818F09FFC206843
:1076800023F0DAFA039B04460298002BCABF4FF49A
:107690007A764FF0FF3696FBF3F60E2811D04AF0BB
:1076A0006AFF4FF47A7595FBF0F594F8B3305BB14F
:1076B0000023204684F8B43040F09BF93E2004B00B
:1076C00070BD4FF0FF35F0E794F8B430002BEFD1E8
:1076D0006B1CEDD054F06BF92369C31A9E4202D2A1
:1076E000104839F055FAD4F8A020821A9542C4E91E
:1076F000280112D3B3FBF5F205FB1233ED1A54F057
:1077000056F9D4E92832C01A61EB0201A84271F19E
:107710000001CDD2F9F784FAF1E71E20CFE700BFD0
:10772000042D0A00234F090038B50D4623F084FAD2
:10773000044628461EF08CFAB5EEC00AF1EE10FAA7
:1077400006D4B7EE007AB4EEC70AF1EE10FA01DD06
:1077500000F00CF8204603F039F910B9024839F06E
:1077600017FA0E2038BD00BFF44E090008B50348D3
:107770000123002240F2E32139F044FAC25109000A
:1077800008B5014839F0B6F9125009002DE9F04763
:1077900086B0084611461A4602AB0193674B009328
:1077A000042349F056FF40F27A51029855F000FE4A
:1077B00040F27D510546039855F0FAFD60490646B2
:1077C0000C204BF0B2FAFF23DDF8108083722A7987
:1077D00033799A42044603D140F2E34018F0E0FBCB
:1077E00000234360574B1A7A22B11A7E002A40F0D8
:1077F000A280012203EB021363602879012128F0A3
:10780000A5FA0121307928F0A1FA0A2028F0FCFB22
:107810002879002128F09AFA3079002128F096FA88
:10782000032028F0F1FB307928F0E2FA40B93079F2
:107830002EF0E8FE28792EF0E5FE434839F0A8F94D
:10784000287928F0D5FA0028F1D0404B96F804901A
:107850002F79984522D83E4B98458CBF4FF08068D1
:107860004FF0CC7867723079A07201F067FF287909
:10787000384D01F063FF636801221A72666896F85A
:1078800004A0342101FB0AF16B1893F82D2042B1BA
:10789000204603F049F9052039F064F94FF0C86833
:1078A000E0E71F2F9A6083F8302083F82F2083F8B9
:1078B00032205E608ABF07F01F033B46264A2748F6
:1078C000685098BF4FF0A04203F5E073B9F11F0F65
:1078D00040F20C6142F823108CBF09F01F034B46A5
:1078E00003F5E0738CBF1C4A4FF0A04240F20C61DC
:1078F00042F823103368C3F80875C3F80C95C3F831
:107900002485342303FB0AF3EB5853B13068072175
:1079100040F30730F1F71CFC306840F307303FF0CC
:107920000DFA342303FB0A552046012385F82D3038
:1079300006B0BDE8F0870A4839F05CF95C2E0A0011
:1079400098C70900580401203D4909007F1A060024
:107950008FD003001862012000030050DDCD080025
:10796000E04F0900F0B50C468DB054F8045B0646B4
:10797000A87A174641F0D8FF284642F010F808AB25
:1079800001931D4B009321460423701E3A4618F0C4
:1079900015FB062205A909981CF094F89DF81C1007
:1079A0000022402018F04EFC069B0B99B3FBF0F32D
:1079B0000446049304AA0A9B039303A850F0A8FE6C
:1079C000049E40F2E5220121304649F081FE039AEF
:1079D00006FB04F362430392049353B105992846CE
:1079E0000A44BDF8201003F021F910B1404239F0EB
:1079F000B9F80E200DB0F0BD3C2E0A00F0B50C46D3
:107A00008DB054F8045B0646A87A174641F08CFF07
:107A1000284641F0C4FF08AB01931A4B009321465E
:107A200004233A46701E18F0C9FA052205A90998E0
:107A30001CF048F89DF81C100022402018F002FCB1
:107A4000069B0B99B3FBF0F30446049304AA0A9B2C
:107A5000039303A850F05CFE039A049B012100915C
:107A600005996243039263430A442846BDF82010F7
:107A70000493F2F73FFF10B1404239F073F80E2043
:107A80000DB0F0BD1C2E0A002DE9F0410C4694B05B
:107A900054F8046B0546B07A174641F045FF30466E
:107AA00041F07DFF0DAB0193314B00933A46072324
:107AB0002146681E18F082FA05220AA90E981CF0C9
:107AC00001F89DF830100022402018F0BBFB0B9B02
:107AD0001199B3FBF0F30546069306AA109B059394
:107AE00005A850F015FE062207A90F981BF0EAFF23
:107AF0009DF824100022402018F0A4FB089B139945
:107B0000B3FBF0F30446049304AA129B039303A867
:107B100050F0FEFD049F4FF498620121384649F071
:107B2000D7FD0598069BBDF83480002268436B435F
:107B30000092039D0A9A0590654302447C434146A6
:107B40003046079F069303950494F2F7D3FE38B9A5
:107B50004CB123467A194146304603F067F810B11C
:107B6000404238F0FFFF0E2014B0BDE8F08100BFA6
:107B7000E42D0A00F0B50C4687B054F8045B0646C5
:107B8000687A174641F0CAFE284641F008FF02AB6A
:107B90000193184B00932146701E04233A4618F0B7
:107BA0000DFA40F2EC4301220021039849F084FDD4
:107BB00040F2DC43012200210446049849F07CFD98
:107BC0004FF43373064609220598082149F074FDE5
:107BD000C0B2082802D0052038F0C4FF0299F3B2E1
:107BE000E2B2284642F0AFFA0028F4D00E2007B0E7
:107BF000F0BD00BFF42E0A002DE9F04F89B0084611
:107C000011461A4604AB0193744B0093042349F0C8
:107C100020FD40F20531049855F0CAFB40F2944132
:107C20000746059855F0CCFB40F28541044606987E
:107C300055F0C6FB064618B914B9694838F0DAFFA2
:107C400068490C204BF071F89DF81C30FF22054666
:107C5000427223B1644840F2F73138F077FF436055
:107C6000624BD3F8003513F00F0305D0604BD3F807
:107C700000351B0711D101235E4A02EB03136B6031
:107C800097F80480D3F808A085F80980404601F0F1
:107C900055FD24B9FF24AC7206E05748CEE724799D
:107CA000AC72204601F04AFD0EB33679EE723046D2
:107CB00001F044FDD5F804B0504F9BF80490242304
:107CC00003FB09731B7F63B95046F8F7E7FF029087
:107CD000B9F1000F0ED1B0F1206F02D0B0F1A05F6A
:107CE0000BD1284602F0E6FF052038F03BFFFF26C7
:107CF000EE72DFE7B9F1010FF3D1242202FB09F2A2
:107D0000B8180021DBF800A041604046B95028F0C7
:107D100051F8B8F11F0F8BBF08F01F0242463849D7
:107D20004FF0A04102F5E0720120FF2C41F8220043
:107D30004AD0204628F03EF8204628F017F8FF2EBB
:107D400045D000213046039628F000F8039A2421FC
:107D500001FB09F3F918039381F82160FF2681F8EC
:107D600020600221CAF86015029BCAF80885CAF88B
:107D70000C45CAF8102500221146CAF82435504691
:107D800050F0F1FC039BCAF8C065FA5807210AB30A
:107D90004022CAF80423CAF80015DBF8000040F3BB
:107DA0000730F1F7D5F9DBF8000040F307303EF07B
:107DB000C5FF242303FB097700237B772846012393
:107DC0003B7709B0BDE8F08F4FF0FF34B7E74FF0D5
:107DD000FF32BCE7CAF80015EBE700BF142F0A001A
:107DE000D84909007CC709004A52090000F0024046
:107DF0000030024010220A00D04F0900B861012073
:107E00000003005010B50446407A41F087FD6368D6
:107E10001B68D3F82435B3F1805F23D013D8B3F1B6
:107E2000006F21D00BD8B3F1007F1FD01248B3F1FF
:107E3000806F18BF0020400040F0010010BD0F48C7
:107E4000B3F1206FF5E7B3F1804F11D006D8B3F14D
:107E5000A05F0FD00A48B3F1005FEAE70948B3F129
:107E6000004FE6E70848E6E70848E4E70848E2E7A5
:107E70000848E0E70848DEE790D003000024F4005B
:107E800080841E0000127A0040420F0020A10700EB
:107E900048E8010000093D000048E801F0B50C4643
:107EA0008DB054F8045B0646687A174641F036FDFB
:107EB000284641F074FD08AB01931A4B009321460C
:107EC00004233A46701E18F079F8062205A908988E
:107ED0001BF0F8FD9DF81C100022402018F0B2F9AC
:107EE000099B0A9904930446069BB3FBF0F303AA8B
:107EF00004A8039350F00CFC0499039B614303FB1B
:107F000004F20491039252B105989DF82C3001447B
:107F1000284642F037F910B9052038F023FE0E202C
:107F20000DB0F0BDBC2E0A00F0B50C468BB054F875
:107F3000045B0646687A174641F0F0FC284641F09B
:107F40002EFD07AB0193194B0093214603233A46BC
:107F5000701E18F033F8052204A907981BF0B2FD33
:107F60009DF818100022402018F06CF9089B03932C
:107F70000446059B0999B3FBF0F302AA03A80293F8
:107F800050F0C6FB039B029A634362430393029241
:107F900042B104992846194402F030FF10B9052077
:107FA00038F0E0FD0E200BB0F0BD00BFDC2E0A0063
:107FB000F0B50C4693B054F8046B0546707A17463A
:107FC00041F0ACFC304641F0EAFC0CAB01932B4B8A
:107FD000009321460623681E3A4617F0EFFF05225C
:107FE00009A90C981BF06EFD9DF82C100022402072
:107FF00018F028F90E9B0F99059304460A9BB3FBD2
:10800000F0F304AA05A8049350F082FB062206A907
:108010000D981BF057FD9DF820100022402018F00D
:1080200011F9109B119903930546079BB3FBF0F3DD
:1080300002AA03A8029350F06BFB049B039A0298D8
:10804000059963436A4345436143AB4205910493F9
:108050000392029502D00A4838F0CCFD53B106983D
:10806000024409980144304602F090FE10B9052000
:1080700038F078FD0E2013B0F0BD00BF8C2E0A0042
:10808000344109002DE9F04F2DED028B99B00846DF
:1080900011461A460CAB0193594B00930C2349F03F
:1080A000D8FA40F26E510D9855F08AF940F22561E8
:1080B00081460C9855F084F940F26A518246149832
:1080C00055F07EF940F236318046159855F078F932
:1080D00040F265510746169855F072F90546BAF117
:1080E000000F05D1B9F1000F0DD1464838F082FDDF
:1080F000D14518D0C24516D0BA4514D0824512D009
:10810000B9F1000F05D0C1450DD0B9450BD0A94537
:1081100009D0B8F1000F03D0B84504D0A84502D06B
:108120002FB1AF4203D140F2E34017F039FF4FF4D3
:108130003373092205210F9849F0BEFA4FF4A46366
:108140004FF6FF7206460121139849F0B5FA109BCD
:108150002D4A0490934227D02C4A981A4342434117
:108160005B000222012111980393962349F0A4FA9F
:10817000834612981DF06CFDB0EE408A55F056F91A
:108180009DF85C30224905932C204AF0CEFDF6B2D2
:108190000E9B0993082E059B044607D01D48082214
:1081A0004FF4337138F02EFD0123DAE705B913B12E
:1081B000194838F0C3FC4560184D2B68D3F80035DA
:1081C00013F00F0305D0AB68D3F80035190714D1AD
:1081D0000123DE0005EBC30363600593BDF8103097
:1081E000089318464FF4A462012149F05DFA039BFD
:1081F000022B059B18D10A4878E70A4876E700BFAA
:10820000342F0A00A53409003C68090040680900C1
:1082100058C70900C85109005C47090068020120DD
:1082200099480900C14F0900BAF1000F00F0F08031
:108230009AF804200492B9F1000F00F0EC8099F84C
:1082400004200692002F00F0E9803A790792B8F1F5
:10825000000F00F0E68098F804200592039A1B793D
:108260000A93002A18BF0E220A990392804A2423F7
:1082700003FB012393F82030002B40F0D58047EA20
:1082800008035FFA8BFB09980B9310F0C3F9ABF16D
:10829000020C049B0B90DCF1000B4BEB0C0B5A1CFB
:1082A0004FEA0B1B05D0184627F0B2FD049827F0C3
:1082B0005DFD069B581C03D00021184627F046FDA3
:1082C000AB590B9AC3F8242547EA0803002B18BFC3
:1082D0004BF0010B039BAA5943EA0B03DBB2C2F834
:1082E0006C35AB59049AC3F80C25069AC3F81425CB
:1082F00047EA0803B3B1079B591C03D00021184675
:1083000027F024FD059B5A1C05D0184627F080FD58
:10831000059827F02BFDAB59059AC3F80825079A55
:10832000C3F810250A9A5249A8592423534301EB54
:10833000030B504ACC504FF48871CBF8042050F016
:10834000FBF9A8594FF4907150F0F6F9A8594FF481
:10835000927150F0F1F9A8594FF4A27150F0ECF974
:10836000A8594FF4AC7150F0E7F9AB59424AC3F841
:108370000423A859032140F30730F0F7E9FEA85978
:1083800040F307303EF0DAFCAB590822C3F8002571
:108390000023CBE90633CBF8143001238BF82030CF
:1083A000B9F1000F45D1BAF1000F55D09AF8040089
:1083B00084F8260001F0C2F9B8F1000F50D098F807
:1083C000040084F8290001F0B9F9002F4CD0387965
:1083D00084F8280001F0B2F9DFED287A099BA36048
:1083E00028EE278A0023BCEEC88A84F8253060680E
:1083F00084ED038A04F1240128F064F8204B9842AC
:10840000024612D1204619B0BDEC028BBDE8F08FB8
:108410004FF0FF320EE74FF0FF3212E74FF0FF321E
:1084200014E74FF0FF3218E7164A1749174854F07F
:10843000EFFD089904F1100051F039FD28B960688A
:1084400028F0C6F8089838F03FFB99F8040084F843
:10845000270001F073F9A6E7FF2384F82630ABE785
:10846000FF2384F82930B0E7FF2384F82830B3E7EE
:1084700080620120E7CD08001003420000007A442A
:108480000000AD0B0500AD0B213E0900A052090014
:1084900010B522F039FC90F82730FF2B044628D085
:1084A000406828F095F894F826002EF0ABF894F880
:1084B00027002EF0A7F894F829002EF0A3F894F8DE
:1084C00028002EF09FF861680B4A4FF6FF73E38493
:1084D000238591424FF00003C4E90433C4E9073314
:1084E000A36103D00832914203D10123034A002142
:1084F000D1540E2010BD00BF68020120E96E01209A
:1085000010B522F001FC044690F8270041F000FA73
:1085100094ED030ADFED047AB8EE400ABDE810409E
:1085200080EE270A1EF042BC00007A4410B522F00B
:10853000EBFB044690F8270041F0EAF963681868FD
:1085400040F30730002801DBF0F7F2FD0023C4E917
:108550000733A36163681B6843F30733002B08DB11
:108560005909012203F01F0302FA03F3024A42F8F9
:1085700021300E2010BD00BF00E100E038B52DED28
:10858000028B0D4622F0C0FB044690F8270041F014
:10859000BFF928461DF05CFBB0EE408A54F046FF60
:1085A000DFED057A28EE278A0E20BCEEC88A84ED1E
:1085B000038ABDEC028B38BD00007A4407B50A4A35
:1085C00040F29313914208BF4FF4A173019340F21C
:1085D000ED130093054940F2422340F2EA224AF0AB
:1085E000B5FD03B000BD00BF3C680900452209008D
:1085F0002DE9F04715460E461F4622F085FB04463E
:1086000090F8270041F084F91DB900252846BDE8FF
:10861000F08763681B68D3F81435013304D12E4802
:1086200040F26E5138F0EEFA53F0C1F9DFF8B0A025
:1086300080468946A3699D4238D86368186840F32C
:108640000730002844DA2A46314604F1100051F080
:1086500051FC94F82530054693B1012204F1240120
:1086600004F1100051F06DFC04F12401606827F062
:1086700029FF94F8290027F09DFB002384F825307A
:1086800063681B6843F30733002B08DB5909012299
:1086900003F01F0302FA03F3104A42F82130002DC1
:1086A000B4D10B233B604FF0FF35AFE753F07FF9B8
:1086B000E368B0EB080061EB0901984271F1000139
:1086C000BBD2F8F7ADFADAF82830002BB2D09CE72D
:1086D000F0F72EFDB7E700BF9649090000E100E082
:1086E000F462012038B50C462046114606221D468C
:1086F00017F02CFC2CB921460120BDE83840F4F7D6
:1087000093BB2968CB0706D411F0030308D108688E
:10871000144A904204D1012C14D0134838F056FA70
:10872000124A0A40062A04D03BB90A68104B9A4202
:1087300003D1012C01D10F48F0E7BDE838400120FA
:10874000F4F7D2BA084649F016FF0546014620461E
:10875000F4F76AFB2A4604460021C06848F020FE70
:10876000204638BDC0320900353309000F0080FFB4
:10877000343109007F350900012807B50B4606D1C1
:108780000B68009340F61623019302206B460146C6
:10879000002202481FF002FC03B000BD3431090082
:1087A000014601481CF0C0BA04620900014A1CF0ED
:1087B00001BB00BF04620900014A1CF0FBBA00BF04
:1087C0003431090008B508460AB117F0F1FB21B1B0
:1087D0001946BDE8084000F005B8014808BD00BFD3
:1087E000A462090070B50646086810F003038EB055
:1087F0000D4603D10168454A91422AD0444C00EA13
:108800000402062A04D043BB0268424B9A4224D198
:10881000023E012E02D9404838F0D8F90AA91FF0CB
:1088200079FB0646286800EA0403062B13D10009E9
:1088300050F099FE04460A9D24B92946304650F06E
:1088400069FE0446314910204AF068FAC0E9025630
:1088500044600EB070BD4468EDE7012E01D02F4892
:10886000DAE710F0010411D0441002D5002038F0EE
:10887000C1F921460AA855F06FF80C98224600214C
:1088800048F08EFD0AA81EF0EDF9E2E701AA40F2D9
:108890005F211BF09BFF019B2BB101AA21462046C3
:1088A00049F020F8D5E72868324603A91BF00AF9F9
:1088B00020B1DDE903011EF0CDF9CAE728681EF0FA
:1088C0001BF90446B8B91020CDE90A0448F038FC79
:1088D0008DF834400C90286806A91BF05FF9044617
:1088E00020461BF01FFB0028CCD049F044FEFF2897
:1088F00006D90B48BBE741100AA855F01FF8EAE774
:10890000C1B20AA854F066FFEAE700BF046209009A
:108910000F0080FF343109007F350900353309002D
:1089200010410900F0B585B0054617460C461DF00C
:1089300019FA6946064628461FF0ECFA042F054648
:1089400022D1A307009814D12268104B9A4210D16B
:1089500001AA21464AF044FD10B90D4838F0EEF85E
:10896000DDE901123046521A29441EF051FB05B0D0
:10897000F0BD01460023224630461BF0C1F8285CBA
:10898000400040F00100F2E70020F0E7885C0900B9
:10899000E93709002DE9F14F8F0705460C461646C9
:1089A00013D001F00F03022B19D102F0FD06012EA6
:1089B0004FEA111104D001B0BDE8F04F06F0CEBE71
:1089C00001B0BDE8F04F06F0D7BB4968CBB22D2B04
:1089D00000F087800BD8062B0ED02C2B13D0554AD5
:1089E0002146284601B0BDE8F04F06F0C5BE2E2B4B
:1089F00000F08C809D2BF2D1002EF0D104F1080202
:108A0000090A284687E0022A02D0A16806F00AFC7B
:108A1000E768002FE3D017F00309E0D17B68DAB2F2
:108A20008E2AB8460DD1022E4FEA132805D007F141
:108A3000040A08F1FF3BD94515DB08F1010857F896
:108A4000288098F80430312B2BD1022E13D1686A7C
:108A500049F0DCF8686A56226FF0020101B0BDE807
:108A6000F04F45F0E5BC5AF8041F284606F0DAFB43
:108A700009F10109DFE72846D8F8081006F0D2FB13
:108A8000012E686A09D15822022145F0D1FC686A9A
:108A900001B0BDE8F04F49F0E3B856226FF0020193
:108AA000DCE7322B9BD1012E686A0AD148F0FCFF2B
:108AB000D8F80810686A090901B0BDE8F04F48F01D
:108AC000A4BF022E01D149F0A5F8D8F80830686A91
:108AD0001B0918226FF0010101B0BDE8F04F45F00D
:108AE00027BDA268002A3FF47AAF002E7FF477AF4B
:108AF0005168090A022907D1D3682BB1980703D11D
:108B00001B79AC2B3FF46BAF08327AE7002A7FF475
